:020000040800F2
:1080000090AE0020A1810008A98100084DA90008B8
:10801000AD810008AF810008B181000800000000B8
:10802000000000000000000000000000B381000814
:10803000B581000800000000B7810008B981000880
:10804000BB810008BB810008BB810008BB81000820
:10805000BB810008BB810008BB810008BB81000810
:10806000BB810008BB810008BB810008BB81000800
:10807000BB810008BB8100081F97000823970008F8
:10808000BB81000827970008BB810008BB8100085E
:10809000BB810008BB810008BB810008BB810008D0
:1080A000BB810008BB810008BB810008BB810008C0
:1080B000096B0108BB810008BB810008BB81000877
:1080C000BB810008BB810008BB810008BB810008A0
:1080D000BB810008B1720108B5720108B9720108CC
:1080E000EF9A0008BB810008BB810008BB81000833
:1080F000BB810008BB810008BB8100082B970008EA
:10810000BB810008BB810008BB810008BB8100085F
:10811000A9720108AD720108BB810008BB8100088B
:10812000BB810008BB810008BB810008BB8100083F
:10813000BB810008BB810008BB810008BB8100082F
:10814000BB810008BB810008BB810008BB8100081F
:10815000BB8100082F97000833970008BD72010803
:10816000BB810008BB810008BB810008BB810008FF
:10817000BB810008BB810008BB810008BB810008EF
:10818000BB810008BB810008DFF810D000F00CFCB8
:1081900000480047D98F0108AFF3008090AE00205F
:1081A0000648804706480047FEE7FEE7FEE7FEE791
:1081B000FEE7FEE7FEE7FEE7FEE7FEE7AD6A010841
:1081C000898100082DE9F0410024061B254671F144
:1081D000000605DA01240027D0EB070067EB010158
:1081E000161E73F1000605DA0027D2EB07020125FF
:1081F00067EB030300F066FA86460E4617469C4678
:10820000AC4204D00025D0EB050E65EB010624B18D
:108210000020D2EB000760EB030C704631463A4673
:108220006346BDE8F081202A06DBCB17203A41FAED
:1082300002F043EAE07306E041FA02F3D040C2F1F3
:108240002002914008431946704740EA01039B070A
:1082500003D009E008C9121F08C0042AFAD203E0BB
:1082600011F8013B00F8013B521EF9D27047421E43
:1082700012F8013F002BFBD111F8013B02F8013B42
:10828000002BF9D17047421C10F8011B0029FBD1CB
:10829000801A704730B505460020034600E05B1C9D
:1082A000934205D2EC5CC85C201A01D1002CF6D1B7
:1082B00030BD2DE9FE4F804681EA0300C00F0C4619
:1082C000009021F0004123F00045B8EB0200A941E5
:1082D00005D24046214690461C460B46024623F0F6
:1082E0000040104347D0270DC7F30A00C3F30A51DB
:1082F0000290401A019040286BDAC3F3130040F457
:10830000801B0098924620B10023D2EB030A63EB56
:108310000B0B01985946C0F14002504600F003FA99
:1083200006460D4650465946019AFFF77CFF10EB72
:1083300008006141002487EA115284EAE7731A4376
:1083400040D0009A62B3019A012A4FEA075215DC25
:10835000001B61EB02014FF0004202EA0752CDE937
:108360000042001C41F5801132462B4600F08EFA87
:1083700003B0BDE8F08F40462146F9E7001B61EBF2
:108380000201001C41F5801300185B412018A2F582
:10839000001747EB030140EAD570B6196D4111E0B3
:1083A0006D084FEA360645EAC0754FEA0752001BD2
:1083B00061EB0201001C41F5801149084FEA3000D1
:1083C0000019514132462B4603B0BDE8F04F00F092
:1083D0004EBA0098012240000023D0EB020263EB6A
:1083E000E073009821464FEAE074B8EB000061EBBF
:1083F0000401E9E783F000435BE781F0004158E7BF
:108400002DE9FE4F81EA030404F0004421F000410D
:1084100000944FF0000B23F0004350EA01045ED0BB
:1084200052EA03045BD0C3F30A54C1F30A552C4447
:10843000A4F2F3340194A0FB0254C1F3130141F4FC
:108440008011C3F3130343F4801301FB024400FBC8
:10845000034E840A970A44EA815447EA8357A4FBEF
:10846000076802958D0A05FB07854FEA932C04FBEC
:108470000C542705029D4FEA065847EA1637B5EB1C
:1084800008056EEB070C870E920E47EA811742EA49
:108490008312A7FB0201B6EB0B0164EB00042B0D6A
:1084A00043EA0C335E1844EB1C50DA465146E7FBB6
:1084B0000201C5F313044FEA0B3343EA14534FEAA6
:1084C0000432019C43EA0603A4F10C040294009CCC
:1084D000CDE900B400F0DAF903B0BDE8F08F002078
:1084E0000146F9E72DE9F04D81EA030404F0004B61
:1084F00021F0004514464FF0000A23F0004150EAF5
:10850000050220D054EA01021DD0C5F30A570246E5
:10851000C5F31303C1F31300C1F30A5640F48015E9
:1085200043F48013A7EB0608101BD64608F2FD386B
:1085300073EB050002D308F1010801E092185B41DA
:10854000B8F1000F03DA00200146BDE8F08D0020ED
:108550004FF48011064684460EE0171B73EB0507A7
:1085600005D3121B63EB050306434CEA010C4908D3
:108570004FEA300092185B4150EA0107EDD152EA10
:10858000030012D082EA040083EA0501084305D003
:10859000101BAB4106D20122002306E000224FF05F
:1085A000004302E06FF0010253101AEB06004CEB9F
:1085B000085110EB0A0041EB0B01BDE8F04D00F053
:1085C00056B90EB540F2334102910021CDE90011B8
:1085D0000A460B4600F05AF903B000BD3EB5CA1773
:1085E000CB0F002450405140C0186141DA0740F2DF
:1085F00033430094CDE901232246234600F046F997
:1086000003B030BD70B5C1F30A5201F0004500243B
:10861000C1F3130140F2FF3341F480119A4201DAB1
:10862000002070BD40F233439A42A2F2334203DC91
:10863000524200F087F800E090402C43F1D04042D5
:1086400070BD70B5C1F30A5201F000450024C1F3BA
:10865000130140F2FF3341F480119A4202DA002004
:10866000014670BD40F233439A42A2F2334203DC2A
:10867000524200F067F801E000F055F82C43F0D0CA
:108680000023D0EB030063EB010170BD01F0004358
:1086900030B421F0004150EA010206D00A0DA2F5E3
:1086A0006072C1F31301002A02DC30BC0020704765
:1086B000440F44EAC104C100E01830BC00EBC250D2
:1086C00000F09EB82DE9F05F0546002092469B46DB
:1086D00088460646814640241BE0284641464746D8
:1086E000224600F02FF853465A46C01A914110D343
:1086F00011461846224600F016F82D1A67EB0108BD
:108700004F4622460120002100F00DF817EB00092A
:108710004E41201EA4F10104DFDC484631462A46C2
:108720004346BDE8F09F202A04DB203A00FA02F11C
:10873000002070479140C2F1200320FA03F319434F
:1087400090407047202A04DB203A21FA02F00021F1
:10875000704721FA02F3D040C2F120029140084351
:10876000194670470FB4002300B589B00CA90091D9
:108770000B996FF00042CB601E4B06931E4B079384
:108780000423CDE901321D4A089202466B460020BF
:1087900000F0B6F909B05DF814FB70B586B0064676
:1087A0004FF0FF300091CDE90101002015460C4645
:1087B00004903246694604A8FFF7D4FF02460498A5
:1087C000211825B108B1084600E020462860049829
:1087D00000280DD0002A02DD0098884208D0081B2E
:1087E0000094CDE901043246694604A8FFF7BAFFB8
:1087F00006B070BD398D0008578D0008CD8900087E
:108800000029A8BF7047401C490008BF20F00100A4
:10881000704710B4B0FA80FC00FA0CF050EA010482
:1088200004BF10BC704749B1CCF1200421FA04F414
:1088300011FA0CF118BF012121430843A3EB0C01ED
:10884000CB1D4FEA00614FEA102042BF002010BC50
:10885000704700EBC35010440029A4BF10BC704700
:10886000401C490008BF20F0010010BC704710B543
:10887000141E73F1000408DA401C41F10001921843
:108880005B411A4301D120F0010010BD2DE9F04DEC
:1088900092469B4611B1B1FA81F202E0B0FA80F241
:1088A00020329046FFF73FFF04460F4640EA0A0099
:1088B00041EA0B0153465A46084313D0114653EA86
:1088C000010019D0C8F140025046FFF73BFF0546B2
:1088D0000E46504659464246FFF725FF084305D04D
:1088E000012004E020463946BDE8F08D0020054314
:1088F00046EAE0762C4337430A986305E40AA0EB86
:1089000008000022FD0A44EA47540A3002D500203C
:108910000146E9E7010510196941DDE9084500193B
:108920006941BDE8F04DA2E770B521F00043034373
:108930000CD0C1F30A550024D5EB040564EB040305
:10894000D617AD1AB34102DB0020014670BD2018D6
:1089500041EB025170BD0EB5C10F80EAE0700844D2
:10896000CA07002140F233438DE80E000A460B4649
:10897000FFF78CFF03B000BD30B5041E71F1000499
:1089800004DB4FF00044404264EB0101141E73F11C
:10899000000405DB1C464FF00043524263EB040326
:1089A000994208BF904230BD064C074D06E0E06892
:1089B00040F0010394E8070098471034AC42F6D326
:1089C000FFF7E6FBA8B80108C8B80108C0B24FF429
:1089D000F05100F03BBA00002DE9FF4F087883B05A
:1089E0009946FF2805D0491C2D2804D000240020DA
:1089F00008E000200BE00124F9E700EB800003EB26
:108A00004000491C0B78FF2BF7D104B140420023F2
:108A10000293147819461D462D2C01D02B2C04D11D
:108A2000521C2D2C13D000240294AA461478FF2C3B
:108A30000FD00A25A3FB057801FB05814FF0000C40
:108A400003FB0C11521CE3194AEB0101EEE7012470
:108A5000EAE7814453EA010002D019F5C87F06DA3B
:108A600003980021C0E9001107B0BDE8F08F002590
:108A7000AE4E2F46DFF8B882184600F0FBF9CDE97C
:108A80000001B9F1000002DAC9F1000400E0044677
:108A90000023A74A1AEB030B42EB045A12E0E0074B
:108AA00007D02A46334638464146FFF7A9FC074619
:108AB00088462A46334610461946FFF7A1FC05466C
:108AC0000E466410002CEAD1DDE90001B9F1000F77
:108AD0005A46534606DAFFF705FD3A464346FFF786
:108AE00001FD05E0FFF78CFC3A464346FFF788FCA2
:108AF000029A0AB181F00041039AC2E90001B3E78A
:108B00002DE9FF4F1F468DB0D7E901464FF0FF38E2
:108B10002E2045464FF000090B90B9696D1C0E9848
:108B20008847396A824688470028F6D1BAF1FF3F64
:108B30000AD024F4D064002E11DDBAF12B0F08D036
:108B4000BAF12D0F0BD102E0404611B08DE744F48D
:108B50008064B9696D1C0E9888478246761E694606
:108B6000600501D52D2000E02B208DF8000001F1DB
:108B7000010B0DF1200809E0B9696D1C0E988847BA
:108B800082460F9844F40074761E0560002E02DDC4
:108B9000BAF1300FF0D00B998A453ED144F08004F1
:108BA00006E00F99681CA9F1010944F400740860FB
:108BB000B9696D1C761E0E98884782463028F0D021
:108BC0002BE00B998A4505D1200603D444F080049C
:108BD000761E18E050460FF057FE08B30DF1130152
:108BE000761E44F400748B4508D2AAF130000BF8CD
:108BF000010B200607D5A9F1010003E0200602D4ED
:108C000009F101008146A00502D50F99681C086092
:108C1000B9696D1C0E9888478246002ED1DC53E05E
:108C2000002E51DDBAF1650F02D0BAF1450F4BD1DC
:108C3000A00549D5B9696D1C24F44074761E0E98C0
:108C400088478246002E0CDD2B2804D0BAF12D0F68
:108C500007D144F48074B9696D1C0E988847824628
:108C6000761EE00501D52D2100E02B2108F8011B1F
:108C7000CDF82C8021E00DF12901761E44F400741A
:108C800088450CD2AAF1300010F0FF0088F80000EF
:108C900002D10B99884509D908F1010806E0E005E1
:108CA00001D5244801E042F20F708146B9696D1C7C
:108CB0000E98884782460F980560002E04DD5046C6
:108CC0000FF0E2FD0028D6D1F9690E988847FF2001
:108CD0008BF8000088F800000020069007904B46B3
:108CE0006A4608A906A8FFF777FEA00502D46FF030
:108CF00001002AE714F0240F0AD0E00714D1DDE9BF
:108D000006123868031D3B600068C0E900120BE0E2
:108D1000DDE90601FFF7BAFC0146E00704D1386837
:108D2000021D3A600068016028460EE7000014400A
:108D30000000F03FF1D8FFFF426842B1016811F82E
:108D4000013B23B1521EC0E90012184670470121B1
:108D5000C160881E704742685AB1C368016843B950
:108D600083688B4205D0491E521CC0E900120020C6
:108D700070474FF0FF3070472DE9F04D00231A4641
:108D80001B1A8A4103DB00200146BDE8F08DC1F3C8
:108D90000A52C1F3130141F480154FF0000BD107C3
:108DA00002D100186D41521E0027044640F2FF1107
:108DB000384601EB620A3E468046024600204FF4E8
:108DC0008011FFF7BFFCC2197141BB1846EB0100CF
:108DD000B4EB030C75EB000C04D3E41A65EB00054F
:108DE00017460E46241908F101006D4180463428CB
:108DF000E3DDF91946EB0600091BA84103D24FF049
:108E0000FF32134601E0002213461BEB070046EB3E
:108E10000A51BDE8F04DFFF72ABD000030B5041E31
:108E200071F1000404DB4FF00044404264EB0101A7
:108E3000141E73F1000405DB1C464FF00043524240
:108E400063EB04038B4208BF824230BD7F2801D907
:108E5000002208E0064A02EB5002C007127800D157
:108E6000120902F00F0201209040084070470000F4
:108E700068B801080EB540F2334202920022CDE9F3
:108E800000221346FFF702FD03B000BD70B58C1839
:108E900010F8015B15F0070301D110F8013B2A110E
:108EA00006D110F8012B03E010F8016B01F8016BFB
:108EB0005B1EF9D12B0705D40023521E0DD401F8F7
:108EC000013BFAE710F8013BCB1A921C03E013F8C0
:108ED000015B01F8015B521EF9D5A142D8D30020F5
:108EE00070BD027803E010F8013B1A44D2B2491E6B
:108EF00089B2F8D21046704770B5ADF5287D0026CE
:108F00000D46ADF89462ADF8986200EB40012D4833
:108F100000EBC104608AA84251D9ADF898624AE0DA
:108F2000A089228A284481B2274800F0B1F8ADF820
:108F300094626A46208A0BE0BDF894326168C95C8D
:108F4000BDF89432D154BDF89412491CADF8941276
:108F5000BDF894128842EFD8401E81B21046FFF748
:108F6000C0FF1A498870228A0DF1FF31515C81429D
:108F700019D1ADF894620CE0BDF894126068BDF8A8
:108F80009422405CA1688854BDF89402401CADF85E
:108F90009402208ABDF89412401E8842ECDC012025
:108FA0000DF5287D70BD64200FF0A6FEBDF8980277
:108FB000401CADF89802BDF898020628B0D30020F6
:108FC000EEE7000030970108FC6700202212002025
:108FD000F0B50D46064600EB46011C48002200EBAA
:108FE000C104ADF5257D608AA8422BD9694606E00B
:108FF000A0686368805C98548854521C92B2208A9E
:10900000401E9042F4DC208A401E81B26846FFF781
:1090100068FF228A0DF1FF3100275054A089228A6F
:10902000284481B2684600F02FF929463046FFF700
:1090300063FF012807D064200FF05EFE7F1CBFB2E3
:10904000062FEBD300200DF5257DF0BD30970108EC
:1090500038B50025ADF800500CF050F90A4C2070DE
:1090600000F088F820780949242807D0272808D05C
:10907000282802D1022081F8650038BD81F86550AA
:1090800038BD0120F7E7000022120020D412002092
:109090002DE9F041064615460C46012080F3108864
:1090A000254F0020B8800CF009F9000609D40120F2
:1090B0000FF022FEB888401C80B2B880C828F2D3D6
:1090C00035E0B888C82832D21C4F1021384601F04C
:1090D0009EF90821384601F09CF9E82000F030F8AC
:1090E000C4F3871000F02CF8A006000E00F028F85A
:1090F000002000F025F80024002000F021F8641C76
:10910000A4B2042CF8D3002405E0FF2000F018F8E6
:109110003055641CA4B2AC42F7D31021384601F09C
:1091200078F9002080F310880120BDE8F08100204C
:1091300080F31088F9E700002212002000000240AE
:1091400070B50B4C0546022120460CF0D1F90028E1
:10915000F9D0294620460CF0D4F9012120460CF024
:10916000C7F90028F9D020460CF0C9F9C0B270BD8B
:109170000030014010B5012080F310881A4C002007
:10918000A0800CF09BF8000609D401200FF0B4FD7C
:10919000A088401C80B2A080C828F2D320E0A0881C
:1091A000C8281DD2114C1021204601F030F90821A9
:1091B000204601F02EF93D20FFF7C2FF2A20FFF7DD
:1091C000BFFF8020FFF7BCFFA720FFF7B9FF1021EA
:1091D000204601F01EF9002080F31088012010BD08
:1091E000002080F3108810BD2212002000000240F1
:1091F0002DE9F04106460D46012080F31088204CF1
:109200000020A0800CF05AF8000609D401200FF0CD
:1092100073FDA088401C82B2A280C82AF2D32AE043
:10922000A088C82827D2174F1021384601F0EFF840
:109230000821384601F0EDF88420FFF781FF002077
:10924000FFF77EFF0020FFF77BFF0020FFF778FF8E
:10925000002404E0305DFFF773FF641CA4B2AC424D
:10926000F8D31021384601F0D4F8002080F310889C
:109270000120BDE8F081002080F31088F9E70000AC
:10928000221200200000024070B50D46012181F33A
:1092900010881146FFF7ACFF002832D01B4C00208D
:1092A000A0800CF00BF8000609D401200FF024FD7B
:1092B000A088401C80B2A080C828F2D322E0A088F9
:1092C000C8281FD2124C1021204601F0A0F8082116
:1092D000204601F09EF88320FFF732FFC5F3871088
:1092E000FFF72EFFA806000EFFF72AFF0020FFF76A
:1092F00027FF1021204601F08CF8002080F3108811
:10930000012070BD002080F3108870BD2212002063
:109310000000024010B500231A4604E010F8014B8B
:109320006340521CD2B28A42F8D3184610BD0000E6
:1093300010B5044639200FF0DFFEE0B20FF0FCFE5E
:10934000C4F307200FF0F8FEC4F307400FF0F4FE5B
:10935000200E0FF0F1FE4FF48051034801F059F850
:10936000BDE810400EF09CB8000402402DE9F04129
:10937000054614460E463A200FF0BEFEF0B20FF03E
:10938000DBFE300A0FF0D8FE104F4FF48056314606
:10939000384601F03EF8B0463E460EF081F81D28F2
:1093A00011D1284600F0A4F807463B200FF0A4FE98
:1093B0004146304601F02DF83D44002CEDD0208888
:1093C00038442080E9E7BDE8F08100000004024055
:1093D0002DE9F041054614460E463C200FF08CFE68
:1093E000F0B20FF0A9FE300A0FF0A6FE114F4FF4B5
:1093F00080563146384601F00CF80CB10020208030
:10940000B0463E460EF04CF81E2811D1284600F01A
:1094100017F907463D200FF06FFE4146304600F039
:10942000F8FF3D44002CEDD0208838442080E9E747
:10943000BDE8F0810004024010B50BF087FE08B1D2
:1094400000F028F8BDE81040302000F09FB8014639
:10945000362000F089B810B508B100F0A5F8BDE8D5
:109460001040342000F092B810B5044600F09CF88B
:1094700020785C2801D02F2803D10021642000F03F
:10948000FBF8BDE81040322000F080B8682000F002
:109490004BB8000010B522200FF02EFE0FF022FE78
:1094A00004464FF48051024800F0B3FF204610BD3F
:1094B000000402402DE9F0410FF014FE06460FF0C3
:1094C00011FE05460FF00EFE04460FF00BFE074698
:1094D0004FF48051054800F09CFF46EA052040EA21
:1094E000044040EA0760BDE8F0810000000402404B
:1094F00070B5054627200FF0FFFD0FF0F3FD044681
:10950000260007D00FF0EEFD641E05F8010B14F0E5
:10951000FF04F7D14FF48051024800F07AFF304643
:1095200070BD00000004024010B504460C200FF08E
:10953000E3FD20460FF000FEBDE81040FFF7BABF84
:1095400010B504460A200FF0D7FD20460FF0F4FDB9
:109550000FF0C8FD04464FF48051024800F059FF57
:10956000204610BD0004024010B50C460FF0C4FDAB
:1095700020460FF0E1FD4FF48051034800F049FF11
:10958000BDE810400DF08CBF0004024010B50FF094
:10959000B3FD4FF48051034800F03BFFBDE810409D
:1095A0000DF07EBF0004024070B5054601200FF0AB
:1095B000A3FD0FF097FD432828D22B20FFF7C0FF13
:1095C000102823D22F200FF097FD00200FF0B4FDBC
:1095D0003220FFF7DBFF142818D1CF20FFF7B0FFB0
:1095E000040013D04C20FFF79FFF00EB04214C2018
:1095F00000F042F85020FFF797FF00EB04215020C5
:1096000000F03AF80021702000F036F82F200FF01B
:1096100073FD2C7806E015F8014F5C2C01D02F2C3F
:1096200000D1002420460FF087FD002CF3D1BDE8C7
:1096300070404FF48051014800F0EBBE000402403E
:1096400070B505462D200FF057FD0FF04BFD044679
:10965000260007D028780FF06FFD641E6D1C14F0F3
:10966000FF04F7D14FF48051024800F0D2FE30469B
:1096700070BD00000004024070B505460C460D2088
:109680000FF03AFD28460FF057FDE0B20FF054FD01
:10969000C4F307200FF050FDC4F307400FF04CFD5A
:1096A000200E0FF049FDBDE870404FF48051014895
:1096B00000F0AFBE0004024070B5094DFF22134612
:1096C00005F5807605E010F8014B54402A5D5A40BC
:1096D000335D491E89B2F6D242EA032070BD000014
:1096E000C094010870B500221346154605E010F835
:1096F000014BA2186B41491E89B20029F7D1100C09
:1097000040EA034092B2801845EB13414FEA014210
:1097100042EA104108186FEA000080B270BD07F0FD
:1097200053BD07F0F1BC07F0BFBC07F01DBD00F052
:10973000A3BF0AF001BE0000074A904201D20748C9
:1097400001E005481038064A8B0001EA020101D504
:10975000C160704781607047106402400060024041
:109760007D0F7D0F0029016802D041F0010101E069
:1097700021F00101016070472DE9F043016821F0FB
:10978000010101600021016041608160C1600161EF
:10979000212141613C493C4A3D251039904202D18A
:1097A0008D60BDE8F083384A4FF4746618329042F9
:1097B00001D18E60F5E7344A4FF47417303290428D
:1097C00001D18F60EDE7304A4FF0746C483290421F
:1097D00002D1C1F808C0E4E72B4B2C4A6033984211
:1097E00001D1CA60DDE7284C294B7834A04201D171
:1097F000CB60D6E7DFF89080264C08F19008404512
:1098000001D1CC60CDE7DFF880804FF03D5908F101
:10981000A808404502D1C1F80C90C2E71E49DFF804
:1098200078800839404501D10D60BAE71A4D1835E6
:10983000A84201D10E60B4E7174D3035A84201D1DE
:109840000F60AEE7144D4835A84202D1C1F800C000
:10985000A7E7114D10496035091FA84201D10A60E0
:109860009FE70D4A7832904201D10B6099E70A4A8E
:109870009032904201D10C6093E7074AA83290429F
:109880008FD1C1F800908CE7106002403D000020AD
:10989000400F002000003D20106402400B0607D559
:1098A000436912B143F0800301E023F08003436178
:1098B000802908D0002A026801F01E0101D00A4365
:1098C00000E08A430260704730B50368124ACC68F2
:1098D00013400A682243D1E905452C432243CC6951
:1098E00022430C6A22434C6A22438C6A22434C6B0B
:1098F00022438C6B22431A430260426922F0070321
:10990000D1E90B2422431A4342610A6942604A6842
:1099100082608968C16030BD3F801CF02DE9FC4148
:10992000012120200BF01AFC01268DF8046000258F
:109930008DF8065003208DF805001A4C302700974B
:109940008DF807506946204600F00EFD3021204674
:1099500000F05FFD144C84F8F05484F8F25484F85D
:10996000F16484F8F3644FF4FA70C4F8F80400F07A
:109970001DF894F86802802812D16565232084F8C8
:109980006D02052084F86C0284F86B72142084F850
:109990006A02202084F8690284F8685200F048F8CE
:1099A000BDE8FC8100140240D41200207CB50FF009
:1099B00077FAD0200FF044FA0FF0A6FA00200FF04B
:1099C0003FFA0FF0A1FA0FF06BFAD1200FF038FA3E
:1099D0000FF09AFA00246D4601E0062C01D2012016
:1099E00000E000200FF0FCF92855641CE4B2072CBD
:1099F000F3D30FF06FFA0D489DF8061080F86D1242
:109A00009DF8051080F86C129DF8041080F86B1218
:109A10009DF8021080F86A129DF8011080F8691212
:109A20009DF8001080F868127CBD0000D412002060
:109A30007CB51B48002490F868128DF8001090F84F
:109A400069128DF8011090F86A128DF80210012148
:109A50008DF8031090F86B128DF8041090F86C12CA
:109A60008DF8051090F86D028DF806000FF018FAC9
:109A7000D0200FF0E5F90FF047FA00200FF0E0F9E1
:109A80000FF042FA6D46285D0FF0DAF90FF03CFA5C
:109A9000641CE4B2072CF6D30FF01CFA7CBD000066
:109AA000D412002070B5094D0022134605F58076CA
:109AB00005E010F8014B54402A5D5A40335D491EC1
:109AC00089B2F6D242EA032070BD0000C0940108BA
:109AD000072A00D9072240EA002021B1012901D13B
:109AE000D040C0B270479040C0F307207047704725
:109AF000072A00D9072240EA002029B1012902D112
:109B00009040C0F307207047D040C0B270470000BB
:109B100070B5ADF5327D00260D46ADF8BC62ADF8EE
:109B2000C06200EB4001324800EBC104608AA842E9
:109B30005CD9ADF8C06255E0012264212D4800F0E7
:109B4000A9F92C4800788DF80000382842D1228AE3
:109B5000E06802FB0501274800F09CF9ADF8BC6203
:109B60006A46208A0BE0BDF8BC326168C95CBDF86A
:109B7000BC32D154BDF8BC12491CADF8BC12BDF8C2
:109B8000BC128842EFD8401E81B2104600F044FA61
:109B9000228A0DF1FF31515C81421BD1ADF8BC62CC
:109BA0000EE0BDF8BC226168895CA26800FB05205C
:109BB000BDF8BC221154BDF8BC02401CADF8BC027B
:109BC000208ABDF8BC12401E8842EADC01200DF557
:109BD000327D70BD64200FF08FF8BDF8C002401CCC
:109BE000ADF8C002BDF8C0020628A5D30020EEE7FC
:109BF0003C93010820430020F0B50E46074600EBD9
:109C000047012648ADF5317D002500EBC1048DF8F4
:109C1000BC52608AB0423DD900210846FFF778FF68
:109C2000012837D1694609E0A268401E00FB0620E2
:109C30006268285C505548556D1CADB2208AA84218
:109C4000F2D80025208AE16800FB0611401E82B28E
:109C5000134800F09DF9208A401E81B2684600F04A
:109C6000DBF98DF8BC02208AE168012201447043CF
:109C7000401E0144AFA800F08BF931463846FFF78B
:109C800047FF012807D064200FF036F86D1CADB2F5
:109C9000062DD7D300200DF5317DF0BD3C93010892
:109CA00020430020F0B5ADF5317D2C4D00208DF81E
:109CB000BC022B4E288000243FE000206F4607E0C6
:109CC00056F832204968125C0A543A54401C80B25B
:109CD000298801EB410206EBC2010B8A5B1E83421D
:109CE000EEDC288800EB400006EBC000008A401E36
:109CF00081B2384600F090F98DF8BC02288800EB5C
:109D0000400006EBC000C168008A00FB0411401E41
:109D100082B2144800F03CF92888012200EB400090
:109D200006EBC000C168008A01446043401E014444
:109D3000AFA800F02DF9641CA4B2288800EB400005
:109D400006EBC000408AA042B7D82888401C80B2E9
:109D500028800728AFD30DF5317DF0BD100000201D
:109D60003C930108204300207CB5012108460BF0FC
:109D7000F5F901208DF8040002258DF80550002426
:109D80008DF806408DF807001820154E00906946A2
:109D9000304600F0E9FA05221146304600F020FB7B
:109DA00005220621304600F01BFB05220721304624
:109DB00000F016FBA02000908DF8045003208DF8D1
:109DC00005008DF806408DF807406946304600F0E2
:109DD000CBFA402000906946304600F0C5FA7CBDC1
:109DE00000000240F8B5002634460096FFF7BCFF9D
:109DF00000F0A0F82248641C8442FCD3214C0821C6
:109E0000204600F004FB1021204600F002FB062053
:109E100000F076F80821204600F0FBFA08212046E1
:109E200000F0F5FA1021204600F0F3FA012000F0CE
:109E300067F8002000F064F80821204600F0E9FAF5
:109E40001148D0F81C0208B9FFF72CFF0F4D2E80E7
:109E50000F4E002405E0C0B22146FFF759FE641CF6
:109E6000A4B2288800EB400106EBC101498AA14257
:109E7000F1D880B2401C80B228800728E9D3F8BD11
:109E8000FFFF0F00000002400000434210000020CE
:109E90003C9301082DE9F0410546002416460F4683
:109EA000012080F31088DFF854800821404600F03C
:109EB000AEFA1021404600F0ACFA032000F020F882
:109EC000C7F3074000F01CF8C7F3072000F018F8AC
:109ED000F8B200F015F806E0002000F011F8641C5C
:109EE00005F8010BA4B2B442F6D30821404600F0B5
:109EF00090FA002080F31088BDE8F0810000024055
:109F000070B50B4C0546022120460BF0F1FA0028F3
:109F1000F9D0294620460BF0F4FA012120460BF037
:109F2000E7FA0028F9D020460BF0E9FAC0B270BD7C
:109F30000030014010B5012186B008030BF04AF94A
:109F4000124C20460BF0AAFA0021ADF8081060155B
:109F5000ADF80A003820ADF80C000720ADF800106D
:109F6000ADF81000ADF804104FF48270ADF8061093
:109F7000ADF80E10ADF80200694620460BF0C3FAAA
:109F8000012120460BF080FA06B010BD00300140E0
:109F90002DE9F0410546002416460F46012080F3C6
:109FA0001088DFF870800821404600F030FA102158
:109FB000404600F02EFA0620FFF7A2FF0821404697
:109FC00000F027FA0821404600F021FA102140460F
:109FD00000F01FFA0220FFF793FFC7F30740FFF7D7
:109FE0008FFFC7F30720FFF78BFFF8B2FFF788FF5B
:109FF00005E02878FFF784FF641CA4B26D1CB4420E
:10A00000F7D30821404600F004FA002080F31088BE
:10A01000BDE8F08100000240027803E010F8013B47
:10A020001A44D2B2491E89B2F8D2104670470000D5
:10A0300070B51E4A907A012825D1002595721C49D9
:10A040001C480F244E780123F6B14D70D0F82852E9
:10A05000D0F8346245EAC605D0F83062D0F82C0258
:10A06000B60046EA40000543AC43CC708878CC7813
:10A07000A04208D108710C78A04204D0D0710870B9
:10A08000002800D0937170BD4B70D0F82852D0F8E2
:10A09000346245EAC605D0F83062D0F82C02B6002A
:10A0A00046EA40000543AC438C70DFE7D412002041
:10A0B000C9120020000042422DE9F041ADF57C7D3F
:10A0C00000273D46ADF8E873FFF7B6F95F4C14285A
:10A0D00007D084F867520EF04BFF0DF57C7DBDE88C
:10A0E000F0815B48FFF7C0F9594E103E14283070DC
:10A0F00006D042287ED00120FFF7A9F93570ECE7A1
:10A10000FFF7C4F9C6E90205B046BDF8E803FFF75A
:10A110000FF9FAAA4FF4FA716846FFF727F94DA133
:10A1200068460EF089FFB0806E46D0B1E11981F823
:10A13000BC557F1CBFB2282FF8D34746304447A1F7
:10A140000EF07AFF78800021001F08E0BA886318BB
:10A150000A443244D27883F8BC25491C89B2814232
:10A16000F4DB3FA168460EF067FF4746A8F80400FD
:10A17000D0B10021621882F8E455491C89B228291F
:10A18000F8D3304435A10EF057FF7880002109380C
:10A1900008E0BA8863180A443244127A83F8E42546
:10A1A000491C89B28142F4DB30A168460EF044FFBD
:10A1B000B880D0B10021621882F80C56491C89B2CF
:10A1C0001429F8D3304425A10EF036FF7880002101
:10A1D0000D3808E0BA8863180A443244127B83F8C9
:10A1E0000C26491C89B28142F4DB24A168460EF09A
:10A1F00023FF00E025E0B880D0B10021621882F88A
:10A200007655491C89B23229F8D3304413A10EF097
:10A2100013FF78800021C01F08E0BA8863180A4441
:10A220003244927983F87625491C89B28142F4DB65
:10A2300000210320FFF7E0FC0120FFF708F90120CF
:10A240004BE70348FFF707F947E70000D412002067
:10A250003812002041504E3D000000003B0000003D
:10A26000574946494E414D453D0000005749464932
:10A2700050415353574F52443D00000053455256EE
:10A2800045523D002F4910B5884206D101210846AC
:10A290000AF070FF002101204FE02B49884206D1CF
:10A2A000012102200AF066FF0021022045E0274933
:10A2B000884206D1012104200AF05CFF002104201D
:10A2C0003BE02349884206D1012108200AF052FFD1
:10A2D0000021082031E01F49884206D101211020C9
:10A2E0000AF048FF0021102027E01B49884206D1D0
:10A2F000012120200AF03EFF002120201DE0174907
:10A30000884206D1012140200AF034FF002140207C
:10A3100013E01349884206D1012180200AF02AFF68
:10A320000021802009E00F4988420AD184150121CB
:10A3300020460AF01FFF00212046BDE810400AF029
:10A3400019BF10BD00000240000402400008024096
:10A35000000C0240001002400014024000180240AD
:10A36000001C024000200240F0B5002201274FF0FF
:10A37000030C0B6807FA02F52B40AB422CD10668A0
:10A3800053000CFA03F4A64306600E79D0F800E0FF
:10A390009E4046EA0E0606600E79012E01D0022E7E
:10A3A00012D18668A64386604E79D0F808E09E40B8
:10A3B00046EA0E0686604668AE43466045688E797A
:10A3C0009640B6B235434560C568A543C560CC79B3
:10A3D0009C40C3681C43C460521C102AC9D3F0BD02
:10A3E0004B07DB0E9A40C90810B500EB8100016AEB
:10A3F0000F249C40A1430162016A1143016210BD18
:10A400000246002012690A4200D0012070474183B1
:10A4100070470183704700002DE9F04F7548002513
:10A420002DED028B85B001782C4601294FD10026F5
:10A430008246067000F1020898F80000DFF8B89133
:10A440008B46F52804D098F819004F2874D077E08F
:10A4500098F8020098F8011040EA01246548214666
:10A46000801CFFF729F908EB0401497818F804204B
:10A4700041EA022181422AD198F803105F4FF12965
:10A480002AD05F48F2294BD0F32920D180F84860C8
:10A4900080F83CB0F52038707E700520B870F3204D
:10A4A000F8705920387105215448FFF705F9010A61
:10A4B0007971B8715348076052490720083908601C
:10A4C000504801210C38FFF74DF98AF8016005B0BA
:10A4D000BDEC028BBDE8F08F4946481980F8BC6599
:10A4E0006D1CADB2282DF8D30020241F07E008EB27
:10A4F000000212790B1883F8BC25401C80B2A042E0
:10A50000F5DB00210320FFF777FB0028DFD00AF0FE
:10A510006FF8F52038707E700520B870F120BFE725
:10A5200080F848B080F83DB0F52038707E70052086
:10A53000B870F220B4E7FFE798F81A004B281AD059
:10A540002C4831A1801C0EF077FD050002D00221BD
:10A5500089F8021008EB0507B87B41280ED0B87BBC
:10A560005628B4D1C9F8396689F83D66C9F8396604
:10A5700089F83D66ABE789F802B0A8E76E4629196D
:10A5800001EB0800007C3055641CA4B2092CF6D302
:10A5900030460CF0C5FF51EC100BFEF777F800EEDB
:10A5A000100A9FED1A8A1A484146C0EE080AC0ED0B
:10A5B0008D0AB87E4C4689F8380600202A180A44CD
:10A5C000127F3254401C80B20928F7D368460CF041
:10A5D000A7FF51EC100BFEF759F800EE100AC0EE81
:10A5E000080A10EE900AC4F8390697F8270084F894
:10A5F0003D066CE712000020D4120020FC0300206E
:10A60000D4420020AC640240524D43000000C842D6
:10A61000D416002070B5144C40F224463146204632
:10A620000CF0B1FE00281ED0314620460CF048FE4A
:10A630000E4D00212846FFF795F8314620460CF0D4
:10A640003FFE0B492846FFF777F82088201D008839
:10A65000291D4FF47A70086001212846FFF782F81F
:10A6600004490120087070BD0014014028640240B4
:10A67000008800101200002010B5104C0E49204632
:10A68000FFF75AF800212046FFF76CF80C4C4021E8
:10A6900020460CF071FE0028F9D0084C0949783C9E
:10A6A0002046FFF749F801212046FFF75BF80649ED
:10A6B0000120487010BD000000802020A0640240EE
:10A6C0000014014000880010120000202DE9F04322
:10A6D00001218FB088050AF041FDDFF88C904846D3
:10A6E000FFF74AF84020050103900024CDE9054515
:10A6F000C60207940894CDE909461C4F0B944FF00D
:10A700002068CDE900870C940D94694648460E9464
:10A71000FFF7DAF8012210214846FFF7BFF8DFF80B
:10A720004890A9F178094846FFF726F84FF47A7067
:10A73000CDE90340CDE9054507940894CDE90946E4
:10A740000B480B940C940D94CDF800800E94CDE939
:10A75000017069464846FFF7B7F801214846FFF700
:10A7600001F80FB0BDE8F083A0640240041401407A
:10A77000140000207CB5012104200AF0EFFC164EE5
:10A78000082206213046FFF72BFE0822072130461B
:10A79000FFF726FE02218DF8051000258DF80650E2
:10A7A0000124C0208DF8074000908DF80410694600
:10A7B0003046FFF7D9FD600200908DF804408DF817
:10A7C000065003208DF805008DF807406946304695
:10A7D000FFF7CAFD7CBD0000000802402DE9F047EC
:10A7E000FFF7C8FF4FF4E13000F07AF8FFF76EFF93
:10A7F00000F058F8264D002685F8286685F82A6668
:10A80000012085F8290685F82B0642F21070C5F85C
:10A810003006214F1F483860DFF87C800E21A8F1F8
:10A820000808C8F80010A8F1040901214846FEF7FD
:10A8300099FF1A4C667060780028FCD04FF4FA70CB
:10A840000EF05AFA4FF4165000F04AF81149002061
:10A85000134A103101EB000C135C401CC0B28CF8A1
:10A8600008300A28F6D300202A1892F8B8250B18C9
:10A87000401CC0B2DA740428F6D339601921C8F834
:10A88000001001214846FEF76DFF6670BDE8F087B5
:10A89000D4120020E4070020AC6402401200002023
:10A8A0004891010838B545208DF8000002208DF848
:10A8B000010001248DF802408DF80340684607F03E
:10A8C0009FF947208DF800008DF8014000208DF899
:10A8D00002008DF80340684607F092F938BD000089
:10A8E0001FB50446012120200AF074FC0020ADF8B9
:10A8F00004000094ADF80600ADF80800ADF80C00B7
:10A900000C200D4CADF80A00694620460CF072FD93
:10A91000012120460CF0D7FC012240F224412046C0
:10A920000CF050FD102120460CF0CAFC0122C02181
:10A9300020460CF0D2FC1FBD001401400249C8792A
:10A940000022CA7170470000D4120020024800683B
:10A95000C00700D000BEFEE7F0ED00E002494AF675
:10A96000AA200860704700000030004010B50EF0CB
:10A97000FFFABDE8104064200EF0BEB92DE9F04F9B
:10A9800083466BA0ADF57D7D002400689A460E4697
:10A990002746FB90ADF8E843042A26D8DFF89491C7
:10A9A00099F86C1202EBC20505EB0215624A3023DE
:10A9B000154403EB1111297199F86C1201F00F0184
:10A9C0003031697199F86B1203EB1111A97199F883
:10A9D0006B0200F00F003030E871FEF72DFD1428F7
:10A9E00007D089F867720EF0C3FA0DF57D7DBDE8DA
:10A9F000F08FDFF84481A8F1240898F800001428AB
:10AA00000ED02846FEF730FD88F80000142807D045
:10AA100042287DD00120FEF71AFD88F80070E4E797
:10AA20004FF47A70864200D90646FEF72FFD454660
:10AA3000C5E90207FEF77CFC99F86B2248463021F5
:10AA400001EB12128DF8002099F86B2202F00F0230
:10AA500030328DF8012099F86A2201EB12128DF83C
:10AA6000022099F86A2202F00F0230328DF803209A
:10AA700099F8692201EB12128DF8042090F86922EE
:10AA800002F00F0230328DF8052090F8682201EBB9
:10AA900012118DF8061090F8680200F00F003030A7
:10AAA0008DF80700BAF1000F03D0BAF1010F02D000
:10AAB00004E0542000E052208DF808003A208DF880
:10AAC00009000A23EC4618E00BEB54021078000949
:10AAD000B0FBF3F1C1EBC10108440CEB04013030D1
:10AAE0008872107800F00F00B0FBF3F2C2EBC202E4
:10AAF00010443030A41CC872A4B2B4EB460FE3D3A8
:10AB000003EB460081B2FAAA6046FEF761FC00E062
:10AB100009E0FAAA0221FBA8FEF75AFC0120FEF781
:10AB200096FC2F7061E72846FEF795FC5DE7000074
:10AB30000D0A0000D41200204C1200202DE9F04F25
:10AB400000252DED028BA1B08DF838508DF8005006
:10AB50008DF82050CDE91255CDE900558DF80850FB
:10AB60008DF80C508DF810508DF81450ADF8185029
:10AB70009FEDF80AF8488DED0D0A00F500572530D5
:10AB80000124DFF8D8A34FF47A7BD526DFF8D083F1
:10AB900007909CE0DFF8C09399F8720918B389F820
:10ABA0007259B7F8F81FDAF88C205046C2F57A725D
:10ABB000914218D1D0F88C00C0F57A70A7F8F00F48
:10ABC000E64800218830FEF7CDFDE448E5498830AD
:10ABD000FEF7B2FD88F80040CAF88CB0DF480121CA
:10ABE0008830FEF7BFFD99F87E0910B389F87E59C9
:10ABF000B7F8FA1FDAF844205046C2F57A7291424B
:10AC000017D1406CC0F57A70A7F8F20FD348002135
:10AC10004030FEF7A7FDD148D3494030FEF78CFD08
:10AC200088F80140CAF844B0CC4801214030FEF712
:10AC300099FD99F88A0910B389F88A59B7F8FC1F69
:10AC4000DAF814205046C2F57A72914217D1406961
:10AC5000C0F57A70A7F8F40FC04800211030FEF755
:10AC600081FDBE48C1491030FEF766FD88F80240FC
:10AC7000CAF814B0B94801211030FEF773FD99F8F5
:10AC80009619484619B380F89659B7F8FE1FDAF8B6
:10AC90002C205046C2F57A72914218D1C06AD14632
:10ACA000C0F57A70A7F8F60FAC4800212830FEF7FF
:10ACB00059FDAA48AE492830FEF73EFD88F803400A
:10ACC000C9F82CB0A54801212830FEF74BFDA24859
:10ACD00090F8721990F87E29114490F88A2990F81A
:10ACE00096091044C1427FF455AF04F0DABF0178F1
:10ACF00019B105708DF8085010E0417819B1457010
:10AD00008DF808400AE0817811B18570022003E0D7
:10AD1000C17819B1C57003208DF808009DF80800AE
:10AD2000DFF8348200EB400101EB001008EB00106B
:10AD300090F8161A9DF80800DFF838B200EB4002D0
:10AD4000C2EBC0121BF83200C1280AD19DF80800DE
:10AD500000EB4002C2EBC0120BEBC2008078082867
:10AD60000CD0082984F06987DFE811F0F01A280078
:10AD7000090989111F199A1AD61DFC207E4880F8EE
:10AD800048409DF8080030B1012807D002280FD0B4
:10AD9000032808D10FE04FF4804101E04FF4005147
:10ADA0007648FFF734FB7648C0F8885204F045BF78
:10ADB0004FF48051F4E74FF40061F1E79DF808008B
:10ADC00000EB4001C1EBC0110BEBC100407800214A
:10ADD00006F09EF88DF810008DF82050C14619E05D
:10ADE0009DF8080000EB400101EB00109DF82010D9
:10ADF00009EB001000EB011090F8410A9DF81010CB
:10AE000088429DF8200002D18DF8100010E0401C0F
:10AE10008DF820009DF8080000EB400101EB0010C8
:10AE200009EB001090F8170A9DF820108842D7D837
:10AE30009DF8080000EB4001C1EBC0100BEBC00017
:10AE400080780A22B2EB101F9DF8080000EB400248
:10AE5000C2EBC0100BEBC000807801D100F00F00F6
:10AE60008DF80C009DF80C0010B910208DF80C0026
:10AE70009DF808009DF80C1000EB4002C2EBC012D8
:10AE80005F460BEBC20008444078ADF818009DF80F
:10AE9000080000EB4001C1EBC0110BEBC1009DF8B5
:10AEA0000C10491C06F017FC8DF800009DF80800F6
:10AEB00000EB4001C1EBC01107EBC1009DF80C1085
:10AEC000084480789DF80010884244F0B6869DF8CA
:10AED000080000EB4001C1EBC01107EBC10138468F
:10AEE0004978002904F0A9869DF8081001EB410279
:10AEF000C2EBC11100EBC1029DF80C101144CA78DD
:10AF00009DF8081001EBC10303EB012109EBC1031C
:10AF10009DF8101001EB411103EB810181F8142F12
:10AF20009DF8081009EB01129DF81010114481F8EA
:10AF3000D059BDF81810CE292AD02ADCB9297CD0E6
:10AF400020DC5A29CED0B22978D0B529F7D0B6293D
:10AF5000BBD1FDE300000000D412002000600240DD
:10AF600010080020008800200080201020800010A1
:10AF7000008800106C500020D442002000180240CD
:10AF800000004242C3297CD0C5297BD0CA299CD16C
:10AF9000F5E3E129FCD004F3C880D52908D0D729EE
:10AFA000A0D0D92991D17EE2E7298ED104F061BEEB
:10AFB0009DF8081001EB4102C2EBC11107EBC10083
:10AFC000C07889F862009DF8080000EB400101EBB1
:10AFD00000109DF8101009EB001000EB011099F81B
:10AFE0006210A4EBD11290F8421A62F3000180F8CB
:10AFF000421A9DF8080000EB400101EB00109DF89B
:10B00000101009EB001000EB011099F862104A09CA
:10B0100090F8421A62F3410180F8421A9DF8080044
:10B0200000EB400101EB001009EB00119DF810004E
:10B0300001EB001090F8420A01E0F2E3F2E3C0F302
:10B0400040019DF8080000EBC00202EB002009EB74
:10B05000C0029DF8100000EB401002EB800090F859
:10B06000F00EC0F3400081424CD09DF808004A46E3
:10B0700000EBC00101EB002009EBC0019DF81000BE
:10B0800001E0D0E3FAE300EB401001EB80019DF812
:10B09000080000EB400303EB00109DF8103009EBB3
:10B0A000001000EB031090F8420A430891F8F00EEC
:10B0B00063F3410081F8F00E9DF8080000EB4001B9
:10B0C00001EB00109DF8101002EB001000EB0110D6
:10B0D00090F8420A800716D59DF80800D92100EBA8
:10B0E000C00303EB002009EBC0029DF8100000EB49
:10B0F000401002EB800080F8DD1E9DF80810022051
:10B10000FEF77AFD42E09DF8080000EBC00101EB7C
:10B11000002002EBC0019DF8100000EB401001EB95
:10B12000800080F8E54E9DF80800D92100EBC003AF
:10B1300003EB002002EBC0039DF8100000EB401071
:10B1400003EB800080F8DD1E9DF8080000EB400155
:10B1500001EB001002EB00119DF8100001EB001153
:10B1600091F8420A20F0200381F8423A9DF8080045
:10B1700000EBC00101EB002009EBC0019DF81000BD
:10B1800000EB401001EB800080F8164F9DF808009E
:10B1900000EB400101EB001009EB00119DF81000DD
:10B1A00001EB001090F8420A00F001019DF8080040
:10B1B00000EBC00202EB002009EBC0029DF810007A
:10B1C00000EB401002EB800090F8F00E00F0010060
:10B1D000814204F003829DF8080000EBC00101EBFE
:10B1E00000209DF8101009EBC00001EB411100EBAD
:10B1F00081009DF8081001EB410202EB01119DF85E
:10B20000102009EB011101EB021191F8421A90F89C
:10B21000F02E61F3000280F8F02E9DF8080000EB9C
:10B22000400101EB00109DF8101009EB001000EB3D
:10B23000011090F8420AC00739D09DF808004F4627
:10B2400000EBC00101EB002009EBC0019DF81000EC
:10B2500000EB401001EB800090F8160F00289DF8DD
:10B26000080000EBC00101EB002009EBC0019DF8D4
:10B27000100000EB401001EB80003BD080F8155F20
:10B280009DF8080000EB400101EB001007EB0011F6
:10B290009DF8100001EB001191F8420A20F0010224
:10B2A00081F8422A97F8210638B304F097B99DF83F
:10B2B000080000EB400101EB00109DF8101009EBB5
:10B2C000001000EB011090F8421A21F0200180F8E4
:10B2D000421A9DF8080000EBC00101EB002009EBC9
:10B2E000C0019DF8100000EB401001EB800080F8D9
:10B2F000155FDAE780F8154FD4E7387D0128D4D1FF
:10B30000786DF98A8842D0D29DF8080000EBC00120
:10B3100001EB002007EBC0019DF8100000EB40108E
:10B3200001EB800090F8150F0128BED19DF80800B0
:10B3300000EBC00101EB002007EBC0019DF81000FD
:10B3400000EB401001EB800090F8490F0028ACD1D1
:10B350009DF8080000EB400101EB001007EB001125
:10B360009DF8100001EB001090F8401A9DF80800BD
:10B3700000EBC00202EB002007EBC00080F8D11EFA
:10B380009DF80800C32100EBC00202EB002007EB90
:10B39000C0029DF8100000EB401002EB800080F826
:10B3A000DD1E9DF8080000EB400101EB001007EBEB
:10B3B00000119DF8100001EB0010C0F8445A9DF8F0
:10B3C00008100220FEF718FC8DF8385017E09DF8A1
:10B3D000080000EBC00101EB002007EBC0019DF865
:10B3E000100000EB401001EB80019DF8380008448C
:10B3F00080F8175F9DF83810491C8DF838109DF8BB
:10B4000038001428E3D38DF8385017E09DF8080071
:10B4100000EBC00101EB002007EBC0019DF810001C
:10B4200000EB401001EB80009DF83810084480F8D4
:10B43000335F9DF83800401C8DF838009DF83800C7
:10B440000A28E3D331E79DF8080000EBC00101EBC7
:10B45000002009EBC0019DF8100000EB401001EB4B
:10B46000800090F8D80E012844F0E7839DF808008A
:10B4700000EBC00101EB002009EBC00080F8D35EB7
:10B480009DF80800022100EBC00202EB002009EB4E
:10B49000C0029DF8100000EB401002EB800080F825
:10B4A000D81EB6217BE29DF8081001EB410202EBA9
:10B4B000011109EB011191F81C1A00299DF80C10DB
:10B4C00002D00A29D0D191E00829CDD18DF8385089
:10B4D00024E09DF8081001EB4102C2EBC1119DF878
:10B4E000382000EBC1011144C97801F00F0109298E
:10B4F00018D89DF8081001EB4102C2EBC1119DF86C
:10B50000382000EBC1011144C97801F0F001902905
:10B5100008D89DF83810491C8DF838109DF838105F
:10B520000629D6D39DF838100629C4F086839DF8E5
:10B53000081001EB4102C2EBC11100EBC101C97857
:10B540000B049DF8081001EB4102C2EBC11100EBA6
:10B55000C10109799DF8082043EA012102EB420369
:10B56000C3EBC21200EBC202527911439DF80820CE
:10B5700002EBC20303EB022209EBC2039DF8102089
:10B5800002EB421203EB8202C2F8F11E9DF8081092
:10B5900001EB4102C2EBC11100EBC10189790B043F
:10B5A0009DF8081001EB4102C2EBC11100EBC10193
:10B5B000C97943EA01239DF8081001EB4102C2EB6F
:10B5C000C11100EBC100007A03439DF8080000EBB5
:10B5D000C00101EB002009EBC0019DF8100000EB59
:10B5E000401001EB8000C0F8F53EA4E08DF8385023
:10B5F00024E09DF8081001EB4102C2EBC1119DF857
:10B60000382000EBC1011144C97801F00F0109296C
:10B6100018D89DF8081001EB4102C2EBC1119DF84A
:10B62000382000EBC1011144C97801F0F0019029E4
:10B6300008D89DF83810491C8DF838109DF838103E
:10B640000829D6D39DF838100829C4F0F6829DF851
:10B65000081001EB4102C2EBC11100EBC1018A7974
:10B660009DF8081001EB4103C3EBC11100EBC101D0
:10B67000C97842EA01629DF8081001EB4103C3EB6F
:10B68000C11100EBC10109790B049DF8081001EB11
:10B690004107C7EBC11100EBC101497943EA012120
:10B6A0000A439DF8081001EBC10303EB012109EBEC
:10B6B000C1039DF8101001EB411103EB8101C1F8AA
:10B6C000F12E9DF8081001EB4102C2EBC11100EB15
:10B6D000C1018A7A9DF8081001EB4103C3EBC11147
:10B6E00000EBC101C97942EA01629DF8081001EB43
:10B6F0004103C3EBC11100EBC101097A0B049DF8B2
:10B70000081001EB4107C7EBC11100EBC100407A03
:10B7100043EA002002439DF8080000EBC00101EB62
:10B72000002009EBC0039DF8100000EB401003EB74
:10B730008000C0F8F52E9DF8080000EBC00101EB79
:10B74000002009EBC0019DF8100000EB401000E064
:10B75000A1E001EB800090F8D80E03289DF80800C6
:10B760000ED000EB400101EB00109DF8101009EB2A
:10B77000001000EB011090F8420A80072DD51AE066
:10B7800000EBC00101EB002009EBC00080F8D35EA4
:10B790009DF80800042100EBC00202EB002009EB39
:10B7A000C0029DF8100000EB401002EB800080F812
:10B7B000D81EC521F3E09DF8080000EBC00101EBA5
:10B7C000002009EBC0019DF8100000EB401001EBD8
:10B7D000800080F8DD6E04F030BA9DF8080000EBC0
:10B7E000C00101EB002009EBC0019DF8100000EB47
:10B7F000401001EB800090F8E60E0128EBD19DF897
:10B80000080000EBC00101EB002009EBC0019DF82E
:10B81000100000EB401001EB800080F8E65EB621DE
:10B8200088E02CE0CFE09DF8080000EBC00101EBC0
:10B83000002009EBC0029DF8100000EB401002EB65
:10B84000800080F8DD6E9DF8080000EBC00101EB80
:10B85000002009EBC00080F8D34E9DF8080000EBF3
:10B86000400101EB00109DF8101009EB001000EBF7
:10B87000011090F8421A41F02002C7E0C9E09DF89B
:10B88000080000EBC00101EB002009EBC00080F8CC
:10B89000D35EC32183E09DF8081001EB410202EB67
:10B8A000011109EB011191F81C1A00299DF80810EB
:10B8B00001EB4102C2EBC11100EBC10103F0528761
:10B8C000C9780A049DF8081001EB4103C3EBC111CC
:10B8D00000EBC101097942EA01229DF8081001EB51
:10B8E0004103C3EBC11107EBC100407902439DF84E
:10B8F000080000EBC00101EB002009EBC0039DF83C
:10B90000100000EB401003EB8000C0F80C2F9DF8F6
:10B91000080000EBC00101EB002009EBC0019DF81D
:10B92000100000EB401001EB800090F8D80E0228C8
:10B9300019D0C5219DF8080000EBC00202EB0020E1
:10B9400009EBC0029DF8100000EB401002EB8000F4
:10B9500080F8DD1E9DF8080000EBC00101EB00201F
:10B9600009EBC0002CE09DF8080000EBC00101EBE2
:10B97000002009EBC00080F8D35E9DF80800032189
:10B9800000EBC00202EB002009EBC0029DF81000A2
:10B9900000EB401002EB800080F8D81ED9219DF802
:10B9A000080000EBC00202EB002009EBC0029DF88A
:10B9B000100000EB401002EB800080F8DD1E0AE76B
:10B9C00080F8D35E07E79DF8080000EBC00101EBAB
:10B9D000002009EBC00080F8D34E9DF8080000EB72
:10B9E000C00101EB002009EBC0029DF8100000EB44
:10B9F000401002EB800080F8DD6E9DF8080000EB3F
:10BA0000400101EB001009EB0010FCE380F8422A32
:10BA1000E1E69DF8081001EB410202EB011109EB90
:10BA2000011191F81C1A00299DF80C1002D00E2962
:10BA3000C5D19CE00C29C2D18DF8385024E09DF886
:10BA400008109DF8383001EB4102C2EBC11100EB48
:10BA5000C102D118C97801F00F01092918D89DF841
:10BA6000082002EB4203C3EBC21100EBC1029DF8B8
:10BA700038101144C97801F0F001902908D89DF8D8
:10BA80003810491C8DF838109DF838100A29D6D383
:10BA90009DF838100A2992D30022CDE900222946C8
:10BAA0008DF83850BC461FE0DDE90002120242EA80
:10BAB00010620002CDE900029DF8080000EB400290
:10BAC000C2EBC0109DF838200CEBC0001044C078C9
:10BAD000DDE90023104341EA0302CDE900029DF8AD
:10BAE0003800401C8DF838009DF838000528DBD35D
:10BAF000DDE900239DF8080000EBC00707EB0020FC
:10BB000009EBC0079DF8100000EB401007EB800028
:10BB1000C0F8F92EC0F8FD3E0022CDE900228DF8D4
:10BB200038101FE0DDE90002120242EA1062000252
:10BB3000CDE900029DF8080000EB4002C2EBC01006
:10BB40009DF838200CEBC0001044007ADDE900239A
:10BB5000104341EA0302CDE900029DF83800401C81
:10BB60008DF838009DF838000528DBD399E08DF872
:10BB7000385024E09DF808109DF8383001EB410260
:10BB8000C2EBC11100EBC102D118C97801F00F015D
:10BB9000092918D89DF8082002EB4203C3EBC21113
:10BBA00000EBC1029DF838101144C97801F0F00192
:10BBB000902908D89DF83810491C8DF838109DF848
:10BBC00038100C29D6D39DF838100C29C4F03580D4
:10BBD0000022CDE90022134629468DF838501EE098
:10BBE000009A1B0243EA12631202CDE900239DF87A
:10BBF000082002EB4203C3EBC2129DF8383000EB81
:10BC0000C2021A44D278DDE900371A4341EA070339
:10BC1000CDE900239DF83820521C8DF838209DF87E
:10BC20003820062ADCD3DDE900379DF8082002EB36
:10BC3000C20A0AEB022209EBC20A9DF8102002EBAD
:10BC400042120AEB8202C2F8F93EC2F8FD7E0023DE
:10BC5000CDE900338DF838101FE0DDE900231B0229
:10BC600043EA12631202CDE900239DF8082002EB9B
:10BC70004203C3EBC2129DF8383000EBC2021A44F3
:10BC8000527ADDE900371A4341EA0703CDE9002380
:10BC90009DF83820521C8DF838209DF83820062A4F
:10BCA000DBD3DDE900129DF8080000EBC00303EBD5
:10BCB000002009EBC0039DF8100000EB401003EBDF
:10BCC0008000C0F8011FC0F8052F9DF8080000EBA8
:10BCD000C00101EB002009EBC0019DF8100000EB52
:10BCE000401001EB800090F8D81E9DF8080000EB92
:10BCF000C00202EB002009EBC00090F8D40E814294
:10BD00007ED199F821064F46B8B19DF8080000EBA6
:10BD1000400101EB00109DF8101009EB001000EB42
:10BD2000011090F8421A41F0080280F8422A9DF86A
:10BD300008100220FDF760FF88E0C7F835509DF835
:10BD4000080000EBC00101EB002007EBC0019DF8EB
:10BD50001000102200EB401001EB800101F6F961A8
:10BD60000798FCF772FA9DF8080000EBC00101EBA0
:10BD7000002007EBC0019DF8100000EB401001EB24
:10BD80008000D0F8F11EC7F81910D0F8F50EC7F8EA
:10BD90001D009DF8080000EB400101EB001007EBCF
:10BDA00000119DF8100001EB001090F8400A387661
:10BDB000F448D0F86812C7F83910B0F86C02A7F848
:10BDC0003D009DF8080000EBC00101EB002007EBEF
:10BDD000C0019DF8100000EB401001EB8000D0F88E
:10BDE0000C0FC7F821009DF8080000EB400101EBA3
:10BDF000001007EB00119DF8100001EB001000E0AF
:10BE000012E0D0F8440AC7F83F00786D81B20220F2
:10BE1000FDF7DEF800210620FDF7EEFE786D401CF0
:10BE200078650021052085E79DF8080000EB4001BA
:10BE300001EB00109DF8101009EB001000EB011051
:10BE400090F8421A41F0040180F8421A9DF8080067
:10BE500000EBC00101EB002009EBC0019DF81000D0
:10BE600000EB401001EB800080F8165F9DF80800A1
:10BE700000EBC00101EB002009EBC0019DF81000B0
:10BE800000EB401001EB800080F8DD6E9DF80800AB
:10BE900000EBC00101EB002009EBC0019DF8100090
:10BEA00000EB401001EB800090F8D80E042843F01E
:10BEB000C4869DF8080000EB400101EB00109DF8DE
:10BEC000101009EB001000EB011090F8421A41F03D
:10BED000800280F8422A9DF8080000EBC00101EBC7
:10BEE000002009EBC00080F8D34E9DF80800052221
:10BEF00000EBC00101EB002009EBC0039DF810002E
:10BF000000EB401003EB800080F8D82E63E409EBCF
:10BF1000C0019DF8100000EB401001EB800090F88C
:10BF2000DA0EB228F2D19DF8080000EBC00101EB57
:10BF3000002009EBC00080F8D35E9DF80800B22114
:10BF400000EBC00202EB002009EBC0029DF81000DC
:10BF500000EB401002EB800080F8DD1E9DF8080029
:10BF600000EBC00101EB002009EBC0019DF81000BF
:10BF700000EB401001EB800080F8DA5E2BE49DF8C6
:10BF8000080000EB4001C1EBC01059461BF830001F
:10BF9000042809D09DF8080000EB4002C2EBC01055
:10BFA00011F83000152801D1ADF818009DF80800EF
:10BFB0005F4600EB4002C2EBC01001EBC0004278CC
:10BFC0009DF8080000EB4003C3EBC01011F83000EF
:10BFD00042EA0020A0F58051303922D09DF80800B7
:10BFE00000EB4001C1EBC01007EBC00039464278BE
:10BFF0009DF8080000EB4003C3EBC01017F83000B9
:10C0000042EA0020A0F58052313A0CD09DF8080099
:10C0100000EB4002C2EBC01011F83000022804D03F
:10C0200019E0A62015E0A72013E09DF8080000EB1A
:10C030004002C2EBC01001EBC00002799DF808007D
:10C0400000EB4003C3EBC01007EBC000C07842EA2E
:10C050000020ADF818009DF8080000EBC00101EBCE
:10C06000002008EBC00090F8D21E8DF810109DF84B
:10C07000080008EB00119DF81000084480F8D05922
:10C08000BDF8180043F23002811A90427CD009DCDE
:10C0900004287AD0152879D0A6280DD0A72843F0F7
:10C0A000CC85CAE0B1F5C06F71D0A1F5C06101398E
:10C0B0006ED00429F3D1FDE39DF8080000EBC00128
:10C0C00001EB002008EBC00080F8D35E9DF808006B
:10C0D00000EBC00101EB002008EBC0019DF810004F
:10C0E00000EB401001EB800090F8D80E032836D00A
:10C0F0009DF8080000EBC00101EB002008EBC00137
:10C100009DF8100000EB401001EB800090F8D80E75
:10C1100008283ED09DF8080000EBC00101EB00208C
:10C1200008EBC0019DF8100000EB401001EB80000F
:10C1300090F8D80E0D2836D09DF8080000EBC0010D
:10C1400001EB002008EBC0019DF8100000EB40104F
:10C1500001EB800090F8DD0EA5282ED03FE09DF881
:10C160000800042100EBC00202EB002008EBC00233
:10C170009DF8100000EB401002EB800080F8D81E04
:10C18000A821FCE3D4120020D3E039E1AAE2CBE2FB
:10C19000F9E29DF80800092100EBC00202EB002043
:10C1A00008EBC002ECE39DF808000E2100EBC00292
:10C1B00002EB002008EBC002FEE39DF8080000EB54
:10C1C000400101EB00109DF8101008EB001000EB8F
:10C1D000011090F8421A41F0040180F8421A9DF8CB
:10C1E000080000EBC00101EB002008EBC0019DF846
:10C1F000100000EB401001EB800090F8DA0EA1284F
:10C2000003F01B8500E0FDE39DF8080000EBC00192
:10C2100001EB002008EBC0019DF8100000EB40107E
:10C2200001EB800090F8DA1E9DF8080000EBC002D8
:10C2300002EB002008EBC002E5E39DF8080000EBEC
:10C24000C00101EB002008EBC00080F8D35E9DF830
:10C25000080000EBC00101EB002008EBC0019DF8D5
:10C26000100000EB401001EB800090F8D80E05287C
:10C270009DF8080000EBC00101EB00200CD008EB9A
:10C28000C0019DF8100000EB401001EB800090F819
:10C29000D80E092806D016E008EBC00080F8D35E5F
:10C2A000062100E00A219DF8080000EBC00202EB25
:10C2B000002008EBC0029DF8100000EB401002EBDC
:10C2C000800080F8D81E9DF8080000EBC00101EB4B
:10C2D000002008EBC0019DF8100000EB401001EBBE
:10C2E000800090F8DD0EA42821D19DF8080000EB15
:10C2F000400101EB00109DF8101008EB001000EB5E
:10C30000011090F8421A41F0200180F8421A9DF87D
:10C31000080000EBC00101EB002008EBC0019DF814
:10C32000100000EB401001EB800080F8155FA121A8
:10C3300027E78DF8385014A83B4613E09DF8081005
:10C3400001EB4102C2EBC1119DF8382003EBC101A2
:10C350001144C9789DF8382081549DF83810491C43
:10C360008DF838109DF838100629E7D306210CF017
:10C37000D9FCCDE91205129B000AC0182F4645EBE7
:10C3800007014FF480720023FBF71CFF9DF80800A3
:10C3900000EBC00101EB002008EBC0039DF810008A
:10C3A00000EB401003EB800080F8DC2E9DF80800C5
:10C3B00000EBC00101EB002008EBC00080F8D37E49
:10C3C0009DF8080000EBC00101EB002008EBC00263
:10C3D0009DF8100000EB401002EB800080F8D84E72
:10C3E0009DF80800A72200EBC00101EB002008EB3C
:10C3F000C0039DF8100000EB401003EB8000FCE34D
:10C400009DF8080000EBC00101EB002008EBC00123
:10C410009DF8100000EB401001EB800090F8D80E62
:10C4200006282BD19DF8080000EBC00101EB00208D
:10C4300008EBC00080F8D35E9DF80800072100EBF0
:10C44000C00202EB002008EBC0029DF8100000EBD8
:10C45000401002EB800080F8D81E9DF80800A7214C
:10C4600000EBC00202EB002008EBC0029DF81000B8
:10C4700000EB401002EB800080F8DD1E9DF8080004
:10C4800000EBC00101EB002008EBC0019DF810009B
:10C4900000EB401001EB800090F8D80E01289DF8C9
:10C4A000080000EBC00101EB002054D008EBC001F4
:10C4B0009DF8100000EB401001EB800090F8D80EC2
:10C4C00007289DF8080000EBC00101EB002048D0D0
:10C4D00008EBC0019DF8100000EB401001EB80005C
:10C4E00090F8D80E0B289DF8080000EBC00101EB76
:10C4F00000203CD008EBC0019DF8100000EB40107C
:10C5000001EB800090F8D80E0C289DF8080000EB95
:10C51000C00101EB002040D008EBC0019DF81000E5
:10C5200000EB401001EB800090F8D80E0E284BD0A5
:10C530009DF8080000EBC00101EB002008EBC001F2
:10C540009DF8100000EB401001EB800090F8D80E31
:10C550000F287CD0DAE408EBC00080F8D35E02211B
:10C5600020E008EBC00080F8D35E08211AE008EB59
:10C57000C00080F8D35E9DF808000C2100EBC002DB
:10C5800002EB002008EBC0029DF8100000EB401009
:10C5900002EB800080F8D81EC9E608EBC00080F8E6
:10C5A000D35E0D219DF8080000EBC00202EB0020D5
:10C5B00008EBC0029DF8100000EB401002EB800079
:10C5C00080F8D81EA321DCE59DF808000F2100EBC0
:10C5D000C00202EB002008EBC0039DF8100000EB46
:10C5E000401003EB800080F8D81E9DF80800A121C0
:10C5F00000EBC00202EB002008EBC0039DF8100026
:10C6000000EB401003EB800080F8DD1E9DF8080071
:10C6100000EBC00202EB002008EBC0039DF8100005
:10C6200000EB401003EB800080F8DA1E9DF8080054
:10C6300000EB400101EB00109DF8101008EB00101A
:10C6400000EB011090F8421A41F0800100E013E085
:10C6500080F8421A9DF8080000EB400101EB001041
:10C660009DF8101008EB001000EB011090F8421A32
:10C6700041F0040103F073B89DF8080000EBC0011D
:10C6800001EB002008EBC0019DF8100000EB40100A
:10C6900001EB800090F8DA0EA12819D09DF808006F
:10C6A000A32100EBC00202EB002008EBC0029DF8C2
:10C6B000100000EB401002EB800080F8DD1E9DF8BA
:10C6C000080000EBC00101EB002008EBC001F6E31D
:10C6D0009DF80800A12100EBC00202EB002008EB4E
:10C6E000C002EDE39DF80800A12100EBC00202EBBF
:10C6F000002008EBC0029DF8100000EB401002EB98
:10C70000800080F8DA1E9DF8080000EBC00202EB02
:10C71000002008EBC0029DF8100000EB401002EB77
:10C72000800080F8DD1EFDE39DF8080000EBC001ED
:10C7300001EB002008EBC0019DF8100000EB401059
:10C7400001EB800090F8D80E062843F076829DF821
:10C75000080000EBC00101EB002008EBC00080F8EE
:10C76000D35E9DF80800072100EBC00202EB002019
:10C7700008EBC0029DF8100000EB401002EB8000B7
:10C7800080F8D81EFEE39DF8080000EBC00101EB25
:10C79000002008EBC00080F8D35E9DF80800A721B8
:10C7A00000EBC00202EB002008EBC0029DF8100075
:10C7B00000EB401002EB800080F8DD1E9DF80800C1
:10C7C0003B4600EB4001C1EBC01007EBC0004079D5
:10C7D00030289DF8080000EB400146D0C1EBC010A6
:10C7E00003EBC000407931289DF808007ED000EBB3
:10C7F0004001C1EBC01003EBC000407933289DF825
:10C80000080000EB400172D0C1EBC01003EBC00088
:10C81000407934289DF8080000EB400101EB00103E
:10C820009DF8101008EB001000EB011090F8421A70
:10C8300075D021F0010180F8421A9DF8080000EB44
:10C84000400101EB001008EB00119DF8100001EB16
:10C85000001191F8420A20F0020281F8422A0020D9
:10C86000CDE900008DF83850D3E101EB00109DF8C0
:10C87000101008EB001000EB011090F8421A21F0A4
:10C88000010180F8421A9DF8080000EB400101EB1D
:10C8900000109DF8101008EB001000EB011090F84C
:10C8A000421A21F0020180F8421A9DF8080000EBBC
:10C8B000C00100E06AE201EB002008EBC0019DF836
:10C8C000100000EB401001EB800090F8DB0E3128E7
:10C8D000C5D19DF8080000EB400101EB00109DF868
:10C8E000101008EB001000EB011001E018E023E14C
:10C8F00090F8421A21F0200180F8421A9DF80800B1
:10C9000000EBC00101EB002008EBC0019DF8100016
:10C9100000EB401001EB800080F8155F9FE72DE1F0
:10C9200000EBC00101EB002008EBC0019DF81000F6
:10C9300000EB401001EB800090F8160F00289DF8E6
:10C94000080000EBC00101EB002008EBC0019DF8DE
:10C95000100000EB401001EB80007CD080F8155FE8
:10C960009DF8080000EB400101EB001008EB0011FE
:10C970009DF8100001EB001191F8420A01E0FCE380
:10C98000FCE320F0010281F8422A9DF8080000EB48
:10C99000400101EB00109DF8101008EB001000EBB7
:10C9A000011090F8421A21F0020180F8421A98F81A
:10C9B00021060028B2D100E0F3E398F81400012822
:10C9C000ACD1D8F85400B8F816108842A6D29DF819
:10C9D000080000EBC00101EB00209DF8101008EBEF
:10C9E000C00001EB411100EB810090F8150F012808
:10C9F00094D19DF8080000EBC00101EB002008EB8A
:10CA0000C00101E0FDE3FDE39DF8100000EB4010E4
:10CA100001EB800090F8490F0028CBD19DF8080069
:10CA20004FF0104100EBC00202EB002008EBC00207
:10CA30009DF8100000EB401002EB8000C0F8E01EF3
:10CA40009DF8080000EB400101EB001008EB00111D
:10CA50009DF8100000E05CE001EB001090F8401A37
:10CA60009DF8080000EBC00202EB002008EBC000BC
:10CA700080F8D11E9DF8080000EBC00101EB0020FA
:10CA800008EBC0019DF8100000EB401001EB8000A6
:10CA900090F8D81E9DF8080000EBC00202EB0020C1
:10CAA00008EBC00090F8D40E814289D19DF80800AF
:10CAB00000EBC00101EB002008EBC0019DF8100065
:10CAC00000EB401001EB800080F8DE5E9DF808006E
:10CAD000A42100EBC00202EB002008EBC0029DF88D
:10CAE000100000EB401002EB800080F8DA1E9DF889
:10CAF0000800A32100EBC00202EB002008EBC002FB
:10CB00009DF8100000EB401002EB800080F8DD1E65
:10CB1000A5E680F8154F9DF8080000EB400101EBF9
:10CB2000001008EB00119DF8100001EB001191F8C6
:10CB3000420A40F0010226E701EB00109DF81010B8
:10CB400008EB001000EB011090F8421A41F00101CF
:10CB500080F8421A9DF8080000EB400101EB00103C
:10CB60009DF8101008EB001000EB011090F8421A2D
:10CB700041F0020180F8421AA22116E021F02001C2
:10CB800080F8421A9DF8080000EB400101EB00100C
:10CB90009DF8101008EB001000EB011090F8421AFD
:10CBA00021F0020180F8421AA9219DF8080000EB4B
:10CBB000C00202EB00209DF8102008EBC00002EB41
:10CBC000421200EB820080F8DA1E48E6DDE9001030
:10CBD000000140EA11700901CDE900109DF808003C
:10CBE00000EB4001C1EBC0109DF8381003EBC00012
:10CBF000084480793038C11700E0FDE3DDE9002703
:10CC000010433943CDE900019DF83800401C8DF8F0
:10CC100038009DF838000628D8D39DF80800009900
:10CC200000EBC00202EB002008EBC0029DF81000F0
:10CC300000EB401002EB8000C0F8F11E0021CDE9AE
:10CC400000118DF8385020E0DDE90010000140EAC5
:10CC500011700901CDE900109DF8080000EB4001BA
:10CC6000C1EBC0109DF8381003EBC0000844407BB6
:10CC7000DDE900273038C11710433943CDE9000101
:10CC80009DF83800401C8DF838009DF838000428C5
:10CC9000DAD39DF80800009900EBC00202EB0020F7
:10CCA00008EBC0029DF8100000EB401002EB800082
:10CCB000C0F80C1F0022CDE9002211468DF8385033
:10CCC0001FE00098090141EA10710001CDE900015F
:10CCD0009DF8080000EB4001C1EBC0109DF8381032
:10CCE00003EBC0000844407CDDE900273038C11761
:10CCF00010433943CDE900019DF83800401C8DF800
:10CD000038009DF838000628DBD39DF8080000990C
:10CD100000EBC00202EB002008EBC0029DF81000FF
:10CD200000EB401002EB8000C0F8F51E9DF80800F3
:10CD300000EB4001C1EBC01003EBC00041799DF84E
:10CD4000080000EBC00202EB002008EBC0029DF8D7
:10CD5000100000EB401002EB800080F8DB1E9DF815
:10CD6000080000EB400101EB001008EB00119DF8FA
:10CD7000100001EB001090F8421A9DF8080000EB3B
:10CD8000C00202EB002008EBC002F8E39DF80800A7
:10CD900000EBC00101EB002008EBC00080F8D35E7F
:10CDA0009DF8080000EBC00101EB002008EBC0017A
:10CDB0009DF8100000EB401001EB800090F8D80EB9
:10CDC0000A286AD09DF8080000EBC00101EB0020A2
:10CDD0009DF8101008EBC00001EB411100EB810041
:10CDE00090F8D81E9DF8080000EBC00202EB00206E
:10CDF00008EBC00090F8D40E814214D198F82106B7
:10CE0000F0B39DF8080000EB400101EB00109DF825
:10CE1000101008EB001000EB011090F8421A41F0DE
:10CE2000080280F8422A9DF80800A72100EBC00202
:10CE300002EB002008EBC0029DF8100000EB401050
:10CE400002EB800080F8DD1E9DF80800A22100EBB7
:10CE5000C00202EB002008EBC0029DF8100000EBBE
:10CE6000401002EB800080F8DA1E9DF8080000EB0D
:10CE7000C00101EB002008EBC0019DF8100000E0AC
:10CE80001FE000EB401001EB800080F8165F0021EE
:10CE9000CDE900118DF83850A3E09DF808000B2172
:10CEA00000EBC00202EB002008EBC0029DF810006E
:10CEB00000EB401002EB800080F8D81EB3E78AE355
:10CEC000A7E3C8F835509DF8080000EBC00101EB5E
:10CED000002008EBC0019DF81000102200EB40106C
:10CEE00001EB800101F6F9610798FBF7AEF99DF8B7
:10CEF000080000EBC00101EB002008EBC0019DF829
:10CF0000100000EB401001EB8000D0F8F11EC8F8D3
:10CF10001910D0F8F50EC8F81D009DF8080000EBB8
:10CF2000400100E062E301EB001008EB00119DF806
:10CF3000100001EB001090F8400A88F818009DF8E6
:10CF4000080000EBC00101EB002008EBC0019DF8D8
:10CF5000100000EB401001EB8000D0F80C0FC8F877
:10CF60002100FE48D0F86812C8F83910B0F86C02F9
:10CF7000A8F83D00D8F8540081B20220FCF728F848
:10CF8000002100E047E10620FCF736FED8F8540007
:10CF9000401CC8F8540000210520FCF72DFE42E794
:10CFA000DDE90010000140EA11700901CDE900102F
:10CFB0009DF8080000EB4001C1EBC0109DF838104F
:10CFC00007EBC0000844C07ADDE900233038C11700
:10CFD00010431943CDE900019DF83800401C8DF83D
:10CFE00038009DF838000A28DAD3DDE900129DF8F0
:10CFF000080000EBC00303EB002008EBC0039DF822
:10D00000100000EB401003EB8000C0F8F91EC0F8E0
:10D01000FD2E0021CDE900118DF8385020E0DDE92A
:10D020000001090141EA10710001CDE900019DF8FC
:10D03000080000EB4001C1EBC0109DF8381007EB71
:10D04000C0000844407DDDE900233038C11710439B
:10D050001943CDE900019DF83800401C8DF83800D7
:10D060009DF838000A28DAD3DDE900129DF808009F
:10D0700000EBC00303EB002008EBC003FEE39DF8C8
:10D08000080000EB4001C1EBC01059461BF830000E
:10D09000042809D09DF8080000EB4002C2EBC01044
:10D0A00011F83000152801D1ADF818009DF80800DE
:10D0B000D94600EB4002C2EBC01001EBC000427841
:10D0C0009DF8080000EB4003C3EBC01011F83000DE
:10D0D00042EA0020A0F58051303922D09DF80800A6
:10D0E00000EB4001C1EBC01009EBC000494642789B
:10D0F0009DF8080000EB4003C3EBC01019F83000A6
:10D1000042EA0020A0F58052313A0CD09DF8080088
:10D1100000EB4002C2EBC01011F83000022804D02E
:10D1200019E0A62015E0A72013E09DF8080000EB09
:10D130004002C2EBC01001EBC00002799DF808006C
:10D1400000EB4003C3EBC01009EBC000C07842EA1B
:10D150000020ADF818009DF80800474600EBC0011C
:10D1600001EB002008EBC00090F8D21E8DF81010E3
:10D170009DF8080008EB001101E0FCE39CE09DF83D
:10D180001000084480F8D059BDF81800A7287DD0B9
:10D1900008DC04287BD015287AD0A62842F04D85DB
:10D1A0003BE09CE000F51D60B0F5804004D0112804
:10D1B0006FD01228F2D1FDE39DF8080000EBC0010A
:10D1C00001EB002007EBC0019DF8100000EB4010C0
:10D1D00001EB800090F8D80E0028DFD19DF8080000
:10D1E00000EBC00101EB002007EBC00080F8D35E2C
:10D1F0009DF8080000EBC00101EB002007EBC00127
:10D2000001E0B2E1B6E09DF8100000EB401001EB48
:10D21000800080F8D84EA721ADE39DF8080000EB10
:10D22000C00101EB002007EBC00080F8D35E9DF841
:10D23000080000EBC00101EB002007EBC0019DF8E6
:10D24000100000EB401001EB800090F8D80E02288F
:10D2500029D09DF8080000EBC00101EB002007EB8E
:10D26000C0019DF8100000EB401001EB800090F829
:10D27000D80E05282AD09DF8080000EBC00101EB6C
:10D28000002007EBC0019DF8100003E08DE0CEE028
:10D29000D2E1F3E100EB401001EB800090F8DD0EED
:10D2A000A52826D037E09DF80800032100EBC00236
:10D2B00002EB002007EBC0029DF8100000EB4010CD
:10D2C00002EB800080F8D81EA92154E39DF80800E5
:10D2D000062100EBC00202EB002007EBC0029DF824
:10D2E000100000EB401002EB800080F8D81EA22155
:10D2F00041E39DF8080000EB400101EB00109DF8B0
:10D30000101007EB001000EB011090F8421A41F0EA
:10D31000040180F8421A9DF8080000EBC00101EBFF
:10D32000002007EBC0019DF8100000EB401001EB5E
:10D33000800090F8DA0EA12802F07F849DF80800A2
:10D3400000EBC00101EB002007EBC0019DF81000CD
:10D3500000EB401001EB800002E00000D41200203E
:10D3600090F8DA1E9DF8080000EBC00202EB0020E6
:10D3700007EBC0029DF8100000EB401002EB8000AC
:10D3800080F8DD1EA1219DF8080000EBC00202EB31
:10D39000002008EBC0029DF8100000EB401002EBEB
:10D3A000800080F8DA1E02F048BC9DF8080000EB0F
:10D3B000C00101EB002007EBC0019DF8100000EB5D
:10D3C000401001EB800090F8DD0EA42823D19DF8D9
:10D3D000080000EB400101EB00109DF8101007EB76
:10D3E000001000EB011090F8421A41F0200180F883
:10D3F000421A9DF8080000E0FDE300EBC00101EBDC
:10D40000002007EBC0019DF8100000EB401001EB7D
:10D41000800080F8155F9DF8080000EBC00101EB6B
:10D42000002007EBC00080F8D35EFEF780BF9DF8B8
:10D43000080000EBC00101EB002007EBC0019DF8E4
:10D44000100000EB401001EB800090F8D80E01288E
:10D450009DF8080000EBC00101EB002030D007EB85
:10D46000C0019DF8100000EB401001EB800090F827
:10D47000D80E04289DF8080000EBC00101EB002045
:10D4800024D007EBC0019DF8100000EB401001EB29
:10D49000800090F8D80E06289DF8080000EBC00127
:10D4A00001EB002021D007EBC0019DF8100000EB3C
:10D4B000401001EB800090F8D80E072860D072E78A
:10D4C00007EBC00080F8D35E022104E007EBC00048
:10D4D00080F8D35E05219DF8080000EBC00202EB46
:10D4E000002007EBC002FFF765B807EBC00080F82B
:10D4F000D35E9DF80800072200EBC00101EB00207D
:10D5000007EBC0039DF8100000EB401003EB800018
:10D5100080F8D82E9DF80800A12200EBC00101EB95
:10D52000002007EBC0039DF8100000EB401003EB58
:10D53000800080F8DD2E9DF8080000EB400101EB33
:10D5400000109DF8101007EB001000EB011090F890
:10D55000421A41F0800280F8422A9DF8080000EB50
:10D56000400101EB001008EB00109DF8101000EBDB
:10D57000011090F8421A41F00402FEF747BA91E315
:10D580009DF8080000EBC00101EB002007EBC00193
:10D590009DF8100000EB401001EB800090F8DA0ECF
:10D5A000A1282DD09DF80800A32100EBC00202EBBA
:10D5B000002007EBC0029DF8100000EB401002EBCA
:10D5C000800080F8DD1E9DF8080000EBC00101EB33
:10D5D000002007EBC0019DF8100000EB401001EBAC
:10D5E000800090F8DA0EA22802F027839DF8080048
:10D5F00000EBC00101EB002008EBC000FEF7E0B932
:10D600009DF80800A12100EBC00202EB002007EB0F
:10D61000C0029DF8100000EB401002EB800080F883
:10D62000DD1E9DF8080000EBC00101EB002008EBB7
:10D63000C00080F8D34EB6E69DF80800A12100EBAB
:10D64000C00202EB002007EBC0029DF8100000EBC7
:10D65000401002EB800080F8DD1E9DF8080000EB12
:10D66000C00202EB002007EBC0029DF8100000EBA7
:10D67000401002EB800080F8DA1EB7E79DF8080042
:10D6800000EBC00101EB002007EBC00080F8D35E87
:10D690009DF80800A72100EBC00202EB002007EB79
:10D6A000C0029DF8100000EB401002EB800080F8F3
:10D6B000DD1E9DF808004B4600EB4001C1EBC01099
:10D6C00009EBC000407930289DF8080000EB4001CC
:10D6D00051D0C1EBC01003EBC000407931289DF858
:10D6E00008007DD000EB4001C1EBC01003EBC0008F
:10D6F000407933289DF8080000EB400171D0C1EB60
:10D70000C01003EBC000407934289DF8080000EBFE
:10D71000400167D0C1EBC01003EBC0004079352851
:10D7200072D09DF8080000EB400101EB00109DF85D
:10D73000101007EB001000EB011090F8421A21F0D6
:10D74000010180F8421A9DF8080000EB400101EB4E
:10D75000001007EB00119DF8100001EB001191F88B
:10D76000420A20F0020281F8422A0020CDE900009E
:10D770008DF83850D6E101EB00109DF8101007EB42
:10D78000001000EB011090F8421A21F0010180F81E
:10D79000421A9DF8080000EB400101EB00109DF8D3
:10D7A000101007EB001000EB011090F8421A21F066
:10D7B000020180F8421A9DF8080000EBC00101EB5D
:10D7C000002007EBC0019DF8100000EB401001EBBA
:10D7D000800090F8DB0E3128C7D19DF8080002E0E8
:10D7E00013E019E13AE100EB400101EB00109DF874
:10D7F000101007EB001000EB011090F8421A21F016
:10D80000200180F8421AB0E758E100EBC00101EBBB
:10D81000002007EBC0019DF8100000EB401001EB69
:10D82000800090F8160F00289DF8080000EBC0015A
:10D8300001EB002007EBC0019DF8100000EB401049
:10D8400001EB80007DD080F8155F9DF8080000EBAB
:10D85000400101EB001007EB00119DF8100001EBF7
:10D86000001191F8420A20F0010281F8422A9DF845
:10D87000080000EB400101EB001000E08AE39DF896
:10D88000101007EB001000EB011090F8421A21F085
:10D89000020180F8421A97F821060028B3D1387D9A
:10D8A0000128B0D1786DF98A8842ACD29DF8080081
:10D8B00000EBC00101EB00209DF8101007EBC00049
:10D8C00001EB411100EB810090F8150F01289AD16E
:10D8D0009DF8080000EBC00101EB002007EBC00140
:10D8E0009DF8100000EB401001EB800090F8490F0C
:10D8F000002888D19DF808004FF0104100EBC002CD
:10D9000002EB002007EBC0029DF8100000EB401076
:10D9100002EB8000C0F8E01E9DF8080000EB40011B
:10D9200001EB001007EB00119DF8100001EB001057
:10D9300090F8401A9DF8080000EBC00202EB0020AE
:10D9400000E056E007EBC00080F8D11E9DF808000B
:10D9500000EBC00101EB002007EBC0019DF81000B7
:10D9600000EB401001EB800090F8D81E9DF80800F5
:10D9700000EBC00200E09BE302EB002007EBC000DD
:10D9800090F8D40E814289D19DF8080000EBC001C7
:10D9900001EB002007EBC0019DF8100000EB4010E8
:10D9A00001EB800080F8DE5E9DF80800A42100EB0A
:10D9B000C00200E07FE102EB002007EBC0029DF80F
:10D9C000100000EB401002EB800080F8DA1E9DF89A
:10D9D0000800A32100EBC00202EB002007EBC0020D
:10D9E0009DF8100000EB401002EB800080F8DD1E77
:10D9F000BBE680F8154F9DF8080000EB400101EBF5
:10DA0000001007EB00119DF8100001EB001191F8D8
:10DA1000420A40F0010228E701EB00109DF81010C7
:10DA200007EB001000EB011090F8421A41F00101E1
:10DA300080F8421A9DF8080000EB400101EB00104D
:10DA40009DF8101007EB001000EB011090F8421A3F
:10DA500041F0020180F8421AA22120E001EB0010FF
:10DA60009DF8101007EB001000EB011090F8421A1F
:10DA700021F0200180F8421A9DF8080000EB4001D7
:10DA800001EB00109DF8101007EB001000EB0110E7
:10DA900090F8421A21F0020180F8421AA9219DF85B
:10DAA000080000EBC00202EB00209DF8102007EBFD
:10DAB000C00002EB421200EB82000EE09DF808006D
:10DAC000A12100EBC00202EB002007EBC0029DF891
:10DAD000100000EB401002EB800080F8DA1E44E6F4
:10DAE000DDE90010000140EA11700901CDE90010E4
:10DAF0009DF8080000EB4001C1EBC0109DF8381004
:10DB000003EBC00008448079DDE9002C3038C117F0
:10DB1000104341EA0C01CDE900019DF83800401C9A
:10DB20008DF838009DF838000828D9D39DF80800F2
:10DB3000009900EBC00202EB002007EBC0029DF849
:10DB4000100000EB401002EB8000C0F8F11E002135
:10DB5000CDE900118DF8385021E0DDE90010000119
:10DB600040EA11700901CDE900109DF8080000EBB2
:10DB70004001C1EBC0109DF8381003EBC000084411
:10DB8000C07BDDE9002C3038C117104341EA0C019D
:10DB9000CDE900019DF83800401C8DF838009DF853
:10DBA00038000628D9D39DF80800009900EBC00280
:10DBB00002EB002007EBC0029DF8100000EB4010C4
:10DBC00002EB8000C0F80C1F0021CDE900118DF898
:10DBD000385023E0DDE90001090141EA107100013C
:10DBE000CDE900019DF8080000EB4001C1EBC01039
:10DBF00003EBC00000E050E39DF838100844407D7E
:10DC0000DDE9002C3038C117104341EA0C01CDE9A1
:10DC100000019DF83800401C8DF838009DF8380050
:10DC20000828D7D39DF80800009900EBC00202EB4A
:10DC3000002007EBC0029DF8100000EB401002EB43
:10DC40008000C0F8F51E9DF8080000EB4001C1EB14
:10DC5000C01003EBC00041799DF8080000EBC00242
:10DC600002EB002007EBC0029DF8100000EB401013
:10DC700002EB800080F8DB1E9DF8080000EB4001FD
:10DC800001EB001007EB00119DF8100001EB0010F4
:10DC900090F8421A9DF8080000EBC00202EB002049
:10DCA00007EBC0029DF8100000EB401002EB800073
:10DCB00080F8F01EBFE49DF8080000EBC00101EB06
:10DCC000002007EBC00080F8D35E9DF8080000EB51
:10DCD000C00101EB002007EBC0019DF8100000EB34
:10DCE000401001EB800090F8D80E03286BD09DF80F
:10DCF000080000EBC00101EB00209DF8101007EBBD
:10DD0000C00001EB411100EB810090F8D81E9DF896
:10DD1000080000EBC00202EB002007EBC00090F807
:10DD2000D40E814214D197F82106E0B39DF8080083
:10DD300000EB400101EB00109DF8101007EB001004
:10DD400000EB011090F8421A41F0080280F8422AD4
:10DD50009DF8080000EBC00101EB002007EBC001BB
:10DD60009DF8100000EB401001EB800080F8165F7A
:10DD70009DF80800A72100EBC00202EB002007EB92
:10DD8000C0029DF8100000EB401002EB800080F80C
:10DD9000DD1E9DF80800A22100EBC00202EB00206E
:10DDA00007EBC00200E020E09DF8100000EB4010FF
:10DDB00002EB800080F8DA1E0021CDE900118DF819
:10DDC0003850CC4699E09DF80800042100EBC002D1
:10DDD00002EB002007EBC0029DF8100000EB4010A2
:10DDE00002EB800080F8D81EB2E7C7F835509DF8E6
:10DDF000080000EBC00101EB002007EBC0019DF81B
:10DE00001000102200EB401001EB800101F6F961D7
:10DE10000798FAF71AFA9DF8080000EBC00101EB29
:10DE2000002007EBC0019DF8100000EB401001EB53
:10DE30008000D0F8F11EC7F81910D0F8F50EC7F819
:10DE40001D009DF8080000EB400101EB001007EBFE
:10DE500000119DF8100001EB001090F8400A387690
:10DE60009DF8080000EBC00101EB002007EBC001AA
:10DE70009DF8100000EB401001EB8000D0F80C0F73
:10DE8000C7F82100FE48D0F86812C7F83910B0F87A
:10DE90006C02A7F83D00786D81B20220FBF798F87C
:10DEA00000210620FBF7A8FE786D401C7865002154
:10DEB0000520FBF7A1FE4BE7DDE90010000140EA79
:10DEC00011700901CDE900109DF8080000EB400138
:10DED000C1EBC0109DF838100CEBC0000844C07AAC
:10DEE000DDE900233038C11710431943CDE90001A3
:10DEF0009DF83800401C8DF838009DF838000C283B
:10DF0000DAD3DDE900129DF8080000EBC00303EB53
:10DF1000002007EBC0039DF8100000EB401003EB5E
:10DF20008000C0F8F91EC0F8FD2E0021CDE90011D7
:10DF30008DF8385020E0DDE90001090141EA107157
:10DF40000001CDE900019DF8080000EB4001C1EBA4
:10DF5000C0109DF838100CEBC0000844C07DDDE90E
:10DF600000233038C11710431943CDE900019DF853
:10DF70003800401C8DF838009DF838000C28DAD3A2
:10DF8000DDE900129DF8080000EBC00303EB002060
:10DF900007EBC0039DF8100000EB401003EB80007E
:10DFA000C0F8011FC0F8052F84E69DF8080043461D
:10DFB0009DF8101008EB0010084480F8D0599DF827
:10DFC0000800DC4600EB4001C1EBC0100BEBC000C9
:10DFD000407870280AD19DF8080000EB4001C1EBA1
:10DFE000C0100CEBC0008078FA2830D09DF80800F3
:10DFF00000EB4001C1EBC0100CEBC00040789DF875
:10E00000080000EB4001C1EBC0101CF830009DF887
:10E01000080000EBC00101EB002003EBC00090F80A
:10E02000D21E8DF810109DF8080003EB00119DF82A
:10E030001000084480F8D059BDF81800012841D0DC
:10E0400065287DD0B128AFD0B628ADD103E0B1208E
:10E05000ADF81800DBE79DF8080000EBC00101EB0C
:10E06000002003EBC0019DF8100000EB401001EB15
:10E07000800090F8D80E012896D19DF8080000EB9A
:10E08000C00101EB002003EBC00080F8D35E9DF8D7
:10E09000080000EBC00101EB002003EBC0019DF87C
:10E0A000100000EB401001EB800080F8D84EB12149
:10E0B0009DF8080000EBC00202EB002008EBC00254
:10E0C000FDF775BC9DF8080000EB4001C1EBC010E6
:10E0D0000BEBC00000790128B5D00228B3D003288B
:10E0E000B1D00528B1D19DF8080000EBC00101EBCB
:10E0F000002003EBC0019DF8100000EB401001EB85
:10E10000800090F8D80E00289FD19DF8080000EB01
:10E11000C00101EB002003EBC00080F8D35E9DF846
:10E12000080000EBC00101EB002003EBC0019DF8EB
:10E13000100000EB401001EB800080F8D84E00E0AA
:10E1400013E09DF80800B62100EBC00202EB0020AE
:10E1500003EBC0029DF8100000EB401002EB8000C2
:10E1600080F8DD1EB221FFF70EB99DF8080000EB24
:10E170004001C1EBC0100CEBC0000079B922ADF832
:10E1800018209DF8080000EB4001C1EBC0100CEB1B
:10E19000C000007900F00F018DF814108DF8385090
:10E1A0001DE09DF8080000EB400101EB001003EBBF
:10E1B00000119DF8380001EB001090F8411A9DF80D
:10E1C000080000EB4007C7EBC0101CF830005038C7
:10E1D000814212D09DF83800401C8DF838009DF81F
:10E1E000080000EB400101EB001003EB001090F879
:10E1F000170A9DF838108842D3D89DF838009DF84A
:10E20000141008448DF810009DF8080000EBC001C0
:10E2100001EB002003EBC0079DF8100000EB40105D
:10E2200007EB800090F8D80E012811D09DF8080067
:10E2300000EBC00101EB002003EBC0019DF81000D2
:10E2400000EB401001EB800090F8D80E01287DD142
:10E250009DF8080000EBC00101EB002003EBC000BB
:10E2600080F8D35E9DF80800022100EBC00707EBA1
:10E27000002003EBC0079DF8100000EB401001E008
:10E28000D412002007EB800080F8D81E9DF808000B
:10E2900000EBC00101EB0020FCE380F8DD2E09E576
:10E2A0009DF8080000EB400101EB001008EB0010A6
:10E2B00090F81C0A20B101287DD00228EFD166E237
:10E2C0009DF8080008EB400000F50050B0F8F00F92
:10E2D000801F81B29DF808005F4600EB4002C2EB50
:10E2E000C0120BEBC200401CFBF7FCF9CDE9120594
:10E2F0009DF8080008EB400000F50050B0F8F01F52
:10E300009DF80800394400EB4002C2EBC0106FF0EA
:10E31000040202EBC0000844042107F0FFF9DDE924
:10E320001223C117CDE90001504059400843B6D12E
:10E330009DF8080008EB001080F8D0599DF80800FF
:10E34000B94600EB4001C1EBC01100E0CAE207EBA7
:10E35000C1000079ADF81800BDF8180031289ED131
:10E360009DF8080008EB400000F50050B0F8F00FF1
:10E370004121183890FBF1F0C217CDE9000288F86E
:10E3800004048DF838502F46BBE09DF8080000EBE0
:10E390004001C1EBC0119DF8380009EBC10100EB51
:10E3A00080100844007D9DF83810414481F8050430
:10E3B0009DF8080000E0AEE000EB4001C1EBC011A9
:10E3C0009DF8380009EBC10100EB801008440821DA
:10E3D0001A3007F06FF98DED0D0A10EE100A9DF856
:10E3E000381008EB0111C1F815049DF8080000EB86
:10E3F0004001C1EBC01109EBC1009DF8381001EBE1
:10E40000811108440821323007F054F98DED0D0ACE
:10E4100010EE100A9DF8381008EB0111C1F8110434
:10E420009DF8080000EB4001C1EBC01109EBC100F1
:10E430009DF8381001EB8111084408213A3007F0AB
:10E4400039F98DED0D0A10EE100A9DF8381008EB21
:10E450000111C1F819049DF8080000EB4001C1EB5F
:10E46000C0119DF8380009EBC10100EB8010084491
:10E470000821423007F01EF98DED0D0A10EE100A4A
:10E480009DF8381008EB0111C1F81D049DF8080033
:10E4900000EB400101EB00109DF8381008EB001074
:10E4A00000EB011090F8421A41F0800180F8421A06
:10E4B0009DF8080008EB400000F50050B0F8F01F90
:10E4C0009DF80800494400EB4002C2EBC0104FF039
:10E4D000FF3202EBC000095C9DF8080000EBC002AF
:10E4E00002EB002008EBC0039DF8100000EB401089
:10E4F00003EB800080F8141F9DF83800401C8DF855
:10E5000038009DF83800DDE90012401A77EB020070
:10E51000FFF63BAF48E59DF808005F4600EB400181
:10E52000C1EBC0100BEBC000437D9DF8080000EB71
:10E530004002C2EBC0100BEBC000807D43EA00201C
:10E54000C317CDE900039DF80800152100EB400238
:10E55000C2EBC0100BEBC000FBF7AEF8CDE9120523
:10E56000DDE90001129B694058400843D2D19DF873
:10E57000080000EB4001C1EBC011384617F831200C
:10E58000521E8DF810209DF8081008EB01129DF81E
:10E590001010114481F8D0599DF81010414481F8B1
:10E5A00005549DF8101008EB0111C1F815549DF8A1
:10E5B000081001EB4102C2EBC11100EBC1018A79E5
:10E5C0009DF8081001EB4103C3EBC11100EBC10141
:10E5D000497942EA012100EE101AF8EE400A9FED57
:10E5E000FA0A9DF8081080EE801A01EB4102C2EB96
:10E5F000C11100EBC1010A799DF8081001EB41033C
:10E60000C3EBC11100EBC101C97842EA012100EE60
:10E61000901A9DF81010F8EE600A71EE200A10EEC4
:10E62000902A08EB0111C1F811249DF8081001EBA4
:10E630004102C2EBC11100EBC1018A7A9DF80810BA
:10E6400001EB4103C3EBC11100EBC101497A42EA7E
:10E65000012100EE901A9DF80810B8EE601AC1EE84
:10E66000000A01EB4102C2EBC11100EBC1010A7AC1
:10E670009DF8081001EB4103C3EBC11100EBC10190
:10E68000C97942EA012100EE101A9DF81010B8EE87
:10E69000400A30EE800A10EE102A08EB0111C1F892
:10E6A00019249DF8081001EB4102C2EBC11100EBE7
:10E6B000C100C07A00069DF8080000EB4001C1EBE4
:10E6C000C01018D407EBC000027B9DF8080000EBD7
:10E6D0004003C3EBC01007EBC000C07A42EA002041
:10E6E00000EE100AB8EE400ADFEDB80A20EE200A6C
:10E6F00010EE100A19E007EBC000037B9DF808003C
:10E7000000EB4001C1EBC01007EBC000C07A43EA48
:10E710000020404280B2F9F754FF9FEDAD1B53EC4F
:10E72000112BF9F76DFEF9F7B1FF9DF8101008EB0A
:10E730000111C1F81D049DF8080000EB400101EB38
:10E7400000109DF8101008EB001000EB011090F87D
:10E75000421A41F0800180F8421A9DF8080000EB4F
:10E760004001C1EBC01107EBC100C17D9DF808005D
:10E7700000EBC00202EB002008EBC0029DF8100085
:10E7800000EB401002EB800080F8141FB7E09DF80A
:10E7900008005F4600EB4001C1EBC0100BEBC0006E
:10E7A000C3799DF8080000EB4002C2EBC0100BEBF0
:10E7B000C000007A43EA0020C317CDE900039DF8AA
:10E7C0000800072100EB4002C2EBC0100BEBC000B9
:10E7D000FAF772FFCDE91205DDE90001129B6940ED
:10E7E000584008437ED19DF8080000EB4001C1EB82
:10E7F000C01117F83100401E8DF810009DF8080078
:10E8000008EB001080F8D0599DF81000404480F8C3
:10E8100005549DF8080000EB4001C1EBC01107EB67
:10E82000C1008079F9F7CDFE41EC110B9FED6A0B29
:10E8300009F00EF99DF80800B0EE408AF0EE608A0B
:10E8400000EB4001C1EBC01107EBC10002799DF85C
:10E85000080000EB4001C1EBC01107EBC100C0781C
:10E8600042EA0020F9F7ADFE53EC182BF9F73AFE17
:10E87000F9F70CFF9DF8101008EB0111C1F8150411
:10E880009DF8100008EB0010C0F811549DF810001E
:10E8900008EB0010C0F819549DF8100008EB0010A8
:10E8A000C0F81D549DF8080000EB400101EB00107A
:10E8B00008EB00129DF8100002EB001090F8421ACD
:10E8C00041F0800280F8422A9DF8080000EB4001E8
:10E8D000C1EBC01107EBC100427A9DF8080000EBC4
:10E8E000C00100E05DE201EB002008EBC0039DF8F1
:10E8F000100000EB401003EB800080F8142F9DF80F
:10E90000080000EB400101EB001008EB001090F84C
:10E91000170A88F8040444E29DF8080000EB40015F
:10E92000C1EBC0100BEBC0005946C3789DF808003E
:10E9300000EB4002C2EBC0100BEBC000807843EA52
:10E9400000208DF80C009DF8080000EB4002C2EB9F
:10E95000C0109DF80C200BEBC000104443789DF8CC
:10E96000080000EB4002C2EBC0109DF80C2001EB48
:10E97000C000805C43EA0020C317CDE900039DF886
:10E9800008009DF80C1000EB4002C2EBC0100BEB2E
:10E99000C000FAF791FECDE91205DDE90001129BF6
:10E9A000694058400843B6D19DF808005B4600EB2B
:10E9B0004001C1EBC0100BEBC00040788DF8100097
:10E9C0008DF83850414625E000FF7F470000803D2C
:10E9D000000000000000B0BF000000000000244064
:10E9E0009DF8080000EB400202EB00109DF8382073
:10E9F00001EB001000EB021090F8410A9DF8102086
:10EA000090429DF8380002D18DF8100010E0401CB3
:10EA10008DF838009DF8080000EB400202EB001072
:10EA200001EB001090F8170A9DF838209042D7D8D3
:10EA30009DF8080000EB400202EB00109DF810204A
:10EA400001EB001000EB021090F8422A42F0800225
:10EA500080F8422A9DF8080000EB4002C2EBC0108B
:10EA600003EBC0000279ADF818209DF8080001EB17
:10EA700000129DF81000104480F8D059BDF818001D
:10EA8000F32806D007DC052873D0F12808D0F22837
:10EA900089D187E18DE1F4286CD0F628F8D18BE19B
:10EAA0009DF8080000EBC00202EB002001EBC00261
:10EAB0009DF8100000EB401002EB800090F8D80E9B
:10EAC00000289DF8080020D000EB400202EB001067
:10EAD0009DF8102001EB001000EB021090F8490A9D
:10EAE000C00711D09DF8080000EBC00202EB002027
:10EAF00001EBC0029DF8100000EB401002EB80001B
:10EB000090F8580FC00720D0A8E000EBC00202EB3D
:10EB1000002001EBC0029DF8100000EB401002EB5A
:10EB2000800080F8D84E9DF80800F42200EBC00762
:10EB300007EB002001EBC0079DF8100000EB401030
:10EB400007EB800080F8DD2E88E09DF8080000EBE0
:10EB5000C00202EB002001EBC0029DF8100000EBA8
:10EB6000401002EB800090F84A0F98B38DF83850AF
:10EB700028E091E132E19DF8080000EBC00202EBD1
:10EB800000209DF8102001EBC00002EB421200EBC8
:10EB900082009DF83820104490F84B2F9DF8080013
:10EBA00000EB400707EB00109DF8387001EB0010F8
:10EBB000384490F81E0A824208D19DF83800401C63
:10EBC0008DF838009DF838000428D4D39DF838001B
:10EBD000042825D042E09DF8080000EBC00202EBBB
:10EBE000002001EBC0029DF8100000EB401002EB8A
:10EBF00080009DF83820104490F84B0F9DF80820B5
:10EC000002EB420707EB02129DF8387001EB02128B
:10EC10003A4492F81E2A904208D19DF83800401CD0
:10EC20008DF838009DF838000A28D4D39DF83800B4
:10EC30000A2813D09DF8080000EBC00202EB002068
:10EC400001EBC0029DF8100000EB401002EB8000C9
:10EC500090F8582F42F0010280F8582F9DF80C00D0
:10EC600011289DF8080000EB400202EB00109DF80F
:10EC7000102001EB001000EB021090F8422A36D071
:10EC800022F0080280F8422A9DF8080000EBC0023A
:10EC900002EB002001EBC0029DF8100000EB4010D9
:10ECA00002EB800090F8580FC0077AD09DF808005A
:10ECB00000EBC00202EB002001EBC0029DF8100047
:10ECC00000EB401002EB8000A0F8565F9DF80800B2
:10ECD000052200EBC00303EB002001EBC0019DF80F
:10ECE000100000EB401001EB8000FFF7D6BA42F0B5
:10ECF000080280F8422A8DF8385023E09DF8080079
:10ED000000EB4002C2EBC01003EBC0029DF83800DC
:10ED1000104442799DF8080000EBC00707EB002083
:10ED200001EBC0079DF8100000EB401007EB8007D7
:10ED30009DF83800384480F8172F9DF83820521C71
:10ED40008DF838209DF838000A28D7D38DF8385030
:10ED500023E09DF8080000EB4002C2EBC0109DF8D4
:10ED6000382003EBC0001044C27B9DF8080000EB84
:10ED7000C00707EB002001EBC0079DF8100000EB77
:10ED8000401007EB80009DF83870384480F8302F31
:10ED90009DF83800401C8DF838009DF83800022896
:10EDA000D7D3DBE19DF80800F12200EBC00303EBB1
:10EDB000002008EBC00192E79DF80800032200EB59
:10EDC000C00303EB002001EBC0039DF8100000EB33
:10EDD000401003EB800080F8D82EE3E79DF8082070
:10EDE000022002EBC20707EB022201EBC2079DF8EB
:10EDF000102002EB421207EB820282F8D80E9DF837
:10EE00000800F62700EBC00202EB00209DF810205E
:10EE100001EBC00002EB421200EB820080F8DD7EC5
:10EE20009DF8080000EBC00202EB00209DF81020C6
:10EE300001EBC00002EB421200EB820080F84A4F67
:10EE40008DF8385023E09DF8080000EB4002C2EB3B
:10EE5000C0109DF8382003EBC000104442799DF8A3
:10EE6000080000EBC00707EB002001EBC0079DF88E
:10EE7000100000EB401007EB80009DF8387038441C
:10EE800080F84B2F9DF83800401C8DF838009DF815
:10EE900038000A28D7D361E19DF8080000EB400252
:10EEA000C2EBC01003EBC00082799DF8080000EBB4
:10EEB0004007C7EBC0100BEBC000407942EA0022CC
:10EEC0009DF8080000EBC00303EB002001EBC0033A
:10EED0009DF8100000EB401003EB8000A0F8562FC7
:10EEE0009DF8080000EBC00202EB002001EBC0021D
:10EEF0009DF8100000EB401002EB8000B0F8562F98
:10EF00009DF8080000EB400303EB001001EB00103C
:10EF1000B0F82A0A8242BED39DF80800F12200EB25
:10EF2000C00303EB002001EBC0079DF8100000EBCD
:10EF3000401007EB800080F8DD2E9DF8080000EB04
:10EF4000C00202EB002008EBC0019DF8100000EBAE
:10EF5000401001EB800090F8581F21F0010180F86B
:10EF6000581FFBE09DF808005A4600EB4001C1EB3A
:10EF7000C0100BEBC00000798DF810008DF8205008
:10EF8000C14619E09DF8080000EB400101EB0010BC
:10EF90009DF8201009EB001000EB011090F8410AD9
:10EFA0009DF8101088429DF8200002D18DF81000C5
:10EFB00010E0401C8DF820009DF8080000EB400197
:10EFC00001EB001009EB001090F8170A9DF82010D3
:10EFD0008842D7D89DF8080000EB4001C1EBC01073
:10EFE00002EBC000C078ADF81800BDF81800182872
:10EFF00012D2DFE800F0110C0E118E8E868E881171
:10F0000011118A8E8E8E8E8C11118E118E8E1A2079
:10F0100000E00D208DF80C009DF80C00001FC1B21F
:10F020009DF808005F4600EB4003C3EBC0130BEBF9
:10F03000C300C01CFAF76EF98DF800009DF80800B7
:10F0400000EB4001C1EBC01107EBC1009DF80C10B3
:10F05000084410F8010C9DF8001088427ED19DF8FC
:10F06000080000EB4001C1EBC01107EBC1013846BD
:10F070004978002972D09DF8081001EB4102C2EBDB
:10F08000C11100EBC1029DF80C101144CA789DF823
:10F09000081001EBC10303EB012109EBC1039DF84B
:10F0A000101001EB411103EB810181F8142F9DF841
:10F0B000081009EB01129DF81010114481F8D05985
:10F0C000BDF81810CE293CF476AB24DCB9293CF409
:10F0D000D6AB7BF736AFC3297DD0C5297BF456AFBD
:10F0E0009DF8081001EB410202EB011109EB01113F
:10F0F00091F81C1A00299DF80C106DD00E29ADD185
:10F10000DBE3072086E7082084E70C2082E70A205B
:10F1100080E706207EE7E129D5D006DCD5293AD064
:10F12000D729A7D0D92999D17CE2E5297BF43CAF36
:10F1300089F860459DF8080000EBC00101EB002054
:10F1400009EBC0019DF8100000EB401001EB8000BE
:10F1500090F8D80E00289DF8080000E0F0E200EBDF
:10F16000C00101EB00207CF4D2AE09EBC00080F8B6
:10F17000D35E9DF8080000EBC00101EB002009EB15
:10F18000C0019DF8100000EB401001EB800080F8FA
:10F19000D84EFCF710BB9DF8081001EB4102C2EB02
:10F1A000C11107EBC100C07889F862009DF8080022
:10F1B00000EB400101EB00109DF8101009EB00106E
:10F1C00000EB011099F86210A4EBD11290F8421AEA
:10F1D00062F3000101E096E2D2E280F8421A9DF863
:10F1E000080000EB400101EB00109DF8101009EB46
:10F1F000001000EB011099F862104A0990F8421AC9
:10F2000062F3410180F8421A9DF8080000EB4001CA
:10F2100001EB00109DF8101009EB001000EB01103D
:10F2200090F8420AC0F340019DF8080000EBC002CC
:10F2300002EB00209DF8102009EBC00002EB421207
:10F2400000EB820090F8F00EC0F34000814249D0FC
:10F250009DF8080000EBC00101EB002009EBC002A3
:10F260009DF81000494600EB401002EB80009DF82D
:10F27000082002EB420303EB02129DF8103009EB69
:10F28000021202EB031292F8422A530890F8F02E71
:10F2900063F3410280F8F02E9DF8080000EB400275
:10F2A00002EB00109DF8102001EB001000EB0210A3
:10F2B00090F8420A800716D59DF80800D92200EB85
:10F2C000C00303EB002009EBC0019DF8100000EB28
:10F2D000401001EB800080F8DD2E9DF80810022020
:10F2E000FAF78AFC42E09DF8080000EBC00202EB4E
:10F2F000002001EBC0029DF8100000EB401002EB73
:10F30000800080F8E54E9DF80800D92200EBC0038C
:10F3100003EB002001EBC0039DF8100000EB401050
:10F3200003EB800080F8DD2E9DF8080000EB400222
:10F3300002EB001001EB00129DF8100002EB00122E
:10F3400092F8420A20F0200382F8423A9DF8080021
:10F3500000EBC00202EB002009EBC0019DF8100099
:10F3600000EB401001EB800080F8164F9DF808007C
:10F3700000EB400101EB001009EB00119DF81000BB
:10F3800001EB001090F8420A00F001019DF808001E
:10F3900000EBC00202EB002009EBC0029DF8100058
:10F3A00000EB401002EB800090F8F00E00F001003E
:10F3B00081426AD09DF8080000EBC00101EB0020FB
:10F3C0009DF8101009EBC00001EB411100EB81002A
:10F3D0009DF8081001EB410202EB01119DF810208D
:10F3E00009EB011101EB021191F8421A90F8F02E8D
:10F3F00061F3000280F8F02E9DF8080000EB400158
:10F4000001EB00109DF8101009EB001000EB01104B
:10F4100090F8420AC0073BF44AAF9DF808004F46F7
:10F4200000EBC00101EB002009EBC0019DF81000CA
:10F4300000EB401001EB800090F8160F00289DF8BB
:10F44000080000EBC00101EB002009EBC0019DF8B2
:10F45000100000EB401001EB800017D080F8155F22
:10F460009DF8080000EB400101EB001007EB0011D4
:10F470009DF8100001EB001191F8420A20F0010202
:10F4800081F8422A97F8210618B1A7E080F8154FB5
:10F49000F8E7387D012865D1786DF98A884261D214
:10F4A0009DF8080000EBC00101EB002007EBC00154
:10F4B0009DF8100000EB401001EB800090F8150F54
:10F4C00001284FD19DF8080000EBC00101EB00209E
:10F4D00007EBC0019DF8100000EB401001EB80002D
:10F4E00090F8490FF0BB9DF8080000EB400101EBDC
:10F4F000001007EB00119DF8100001EB001090F8D0
:10F50000401A9DF8080000EBC00202EB002007EB58
:10F51000C00080F8D11E9DF80800C32100EBC00296
:10F5200002EB002007EBC0029DF8100000EB40103A
:10F5300002EB800080F8DD1E9DF8080000EB400122
:10F5400001EB001007EB00119DF8100001EB00101B
:10F55000C0F8445A9DF808100220FAF74DFB8DF8C8
:10F56000385018E03AE09DF8080000EBC00101EBCC
:10F57000002007EBC0019DF8100000EB401001EBEC
:10F5800080019DF83800084480F8175F9DF8381016
:10F59000491C8DF838109DF838001428E3D38DF8F5
:10F5A000385017E09DF8080000EBC00101EB002087
:10F5B00007EBC0019DF8100000EB401001EB80004C
:10F5C0009DF83810084480F8335F9DF83800401CDF
:10F5D0008DF838009DF838000A28E3D39DF808001C
:10F5E00000EB400101EB00109DF8101009EB00103A
:10F5F00000EB011090F8420A80077BF524AF9DF8DC
:10F600000800D92100EBC00202EB002009EBC00288
:10F610009DF8100000EB401002EB800080F8DD1E2A
:10F62000FBF711BF9DF8081001EB410202EB01113D
:10F6300009EB011191F81C1A00299DF80C1002D059
:10F640000A297DD130E008297AD18DF8385025E09B
:10F650009DF8081001EB4102C2EBC1119DF8382062
:10F6600000EBC1011144C97801F00F0109293BF6F3
:10F6700059AF9DF8081001EB4102C2EBC1119DF892
:10F68000382000EBC1011144C97801F0F001902944
:10F69000EDD89DF83810491C8DF838109DF83810B9
:10F6A0000629D5D3FBF73EBF8DF8385025E09DF8ED
:10F6B000081001EB4102C2EBC1119DF8382000EBAC
:10F6C000C1011144C97801F00F0109293BF6BAAF15
:10F6D0009DF8081001EB4102C2EBC1119DF83820E2
:10F6E00000EBC1011144C97801F0F0019029EDD877
:10F6F0009DF83810491C8DF838109DF838100829ED
:10F70000D5D3FBF79FBF9DF8080000EBC00101EBCC
:10F71000002009EBC0019DF8100000EB401001EB48
:10F72000800080F8DD6E9DF8080000EBC00101EB61
:10F73000002009EBC00080F8D34E9DF8080000E0DF
:10F7400095E000EB400101EB001009EB00119DF882
:10F75000100001EB001090F8421A41F0200180F8EF
:10F76000421A6AE20A799DF8081001EB4103C3EBE3
:10F77000C11107EBC100C07842EA0022FCF7B7B81C
:10F780000C2974D18DF8385024E09DF808109DF8AC
:10F79000383001EB4102C2EBC11100EBC102D118BC
:10F7A000C97801F00F01092918D89DF8082002EB4B
:10F7B0004203C3EBC21100EBC1029DF838101144A3
:10F7C000C97801F0F001902908D89DF83810491C3B
:10F7D0008DF838109DF838100A29D6D39DF83810C6
:10F7E0000A2944D30022CDE90022134629468DF888
:10F7F00038501EE0009A1B0243EA12631202CDE960
:10F8000000239DF8082002EB4203C3EBC2129DF8CF
:10F81000383000EBC2021A44D278DDE900371A43CF
:10F8200041EA0703CDE900239DF83820521C8DF8EA
:10F8300038209DF83820052ADCD3DDE900379DF813
:10F84000082002EBC20C0CEB022209EBC20C9DF863
:10F85000102002EB42120CEB8202C2F8F93EC2F811
:10F86000FD7E0023CDE900338DF8381020E0D3E091
:10F87000DDE900231B0243EA12631202CDE90023F3
:10F880009DF8082002EB4203C3EBC2129DF838300A
:10F8900000EBC2021A44127ADDE900371A4341EA4A
:10F8A0000703CDE900239DF83820521C8DF838203D
:10F8B0009DF83820052ADBD399E08DF8385024E0F4
:10F8C0009DF808109DF8383001EB4102C2EBC111E0
:10F8D00000EBC102D118C97801F00F01092918D82D
:10F8E0009DF8082002EB4203C3EBC21100EBC102FA
:10F8F0009DF838101144C97801F0F001902908D81A
:10F900009DF83810491C8DF838109DF838100C29D6
:10F91000D6D39DF838100C297ED30022CDE90022E1
:10F9200029468DF83850BC461FE0DDE9000212027E
:10F9300042EA10620002CDE900029DF8080000EBE7
:10F940004002C2EBC0109DF838200CEBC000104400
:10F95000C078DDE90023104341EA0302CDE900024B
:10F960009DF83800401C8DF838009DF838000628B6
:10F97000DBD3DDE900239DF8080000EBC00707EBAF
:10F98000002009EBC0079DF8100000EB401007EBCA
:10F990008000C0F8F92EC0F8FD3E0022CDE900221B
:10F9A0008DF838101FE0DDE90002120242EA106211
:10F9B0000002CDE900029DF8080000EB4002C2EB16
:10F9C000C0109DF838200CEBC0001044407ADDE9EF
:10F9D0000023104341EA0302CDE900029DF83800FC
:10F9E000401C8DF838009DF838000628DBD3DDE98F
:10F9F00000129DF8080000EBC00303EB002009EBA8
:10FA0000C0039DF8100000EB401003EB8000C0F82D
:10FA1000011FC0F8052F00E00FE19DF8080000EB82
:10FA2000C00101EB002009EBC0019DF8100000EBC4
:10FA3000401001EB800090F8D81E9DF8080000EB04
:10FA4000C00202EB002009EBC00090F8D40E814206
:10FA50007ED199F821064F46B8B19DF8080000EB19
:10FA6000400101EB00109DF8101009EB001000EBB5
:10FA7000011090F8421A41F0080280F8422A9DF8DD
:10FA800008100220FAF7B8F878E0C7F835509DF86A
:10FA9000080000EBC00101EB002007EBC0019DF85E
:10FAA0001000102200EB401001EB800101F6F9611B
:10FAB0000798F8F7CAFB9DF8080000EBC00101EBBE
:10FAC000002007EBC0019DF8100000EB401001EB97
:10FAD0008000D0F8F11EC7F81910D0F8F50EC7F85D
:10FAE0001D009DF8080000EB400101EB001007EB42
:10FAF00000119DF8100001EB001090F8400A3876D4
:10FB00009DF8080000EBC00101EB002007EBC001ED
:10FB10009DF8100000EB401001EB8000D0F80C0FB6
:10FB2000C7F821006648D0F86812C7F83910B0F855
:10FB30006C02A7F83D00786D81B20220F9F748FA0F
:10FB400000210620FAF758F8786D401C786500E02F
:10FB500002E00021052095E79DF8080000EB400138
:10FB600001EB00109DF8101009EB001000EB0110E4
:10FB700090F8421A41F0040180F8421A9DF80800FA
:10FB800000EBC00101EB002009EBC0019DF8100063
:10FB900000EB401001EB800080F8165F9DF8080034
:10FBA00000EBC00101EB002009EBC0019DF8100043
:10FBB00000EB401001EB800080F8DD6E9DF808003E
:10FBC00000EBC00101EB002009EBC0019DF8100023
:10FBD00000EB401001EB800090F8D80E04282CD1E7
:10FBE0009DF8080000EB400101EB00109DF810109B
:10FBF00009EB001000EB011090F8421A41F080016F
:10FC000080F8421A9DF8080000EBC00101EB0020CB
:10FC100009EBC00080F8D34E9DF80800052100EBE9
:10FC2000C00202EB002009EBC0029DF8100000EBBF
:10FC3000401002EB800080F8D81E98F86702A0B14F
:10FC40009DF8080008EB400000F50050B0F8F01FE8
:10FC50009DF80800012300EB4002C2EBC0120BEB41
:10FC6000C2009DF80820FAF789FE8DF838505946F1
:10FC700013E089F86055FBF79EBD9DF8080000EB86
:10FC80004002C2EBC0109DF8382001EBC000855443
:10FC90009DF83800401C8DF838009DF83800142875
:10FCA000EBD3084801784278114482781144C27835
:10FCB000D1427BF41CA821B0BDEC028BBDE8F08FD3
:10FCC000D4120020100800202DE9F74F8EB000203C
:10FCD000ADF80000ADF80C00ADF80C00ADF80C006C
:10FCE0008DF810008DF814008DF81800CDE908008B
:10FCF000CDE90800ADF83400FEA2D2E90032CDE92A
:10FD00000132FEA2D2E90032CDE90A32FD4A107179
:10FD10000E9800EB400202EB0010FB4A02EB0010D1
:10FD2000804690F8160A8DF810000E9802EB00102D
:10FD300003900844814690F8D0290E9808EB0117EB
:10FD400000EBC00303EB0020EF4B042A03EBC00AD7
:10FD500001EB41130AEB83051FD1052289F8D02955
:10FD6000002085F8D80E97F8420A20F0800087F826
:10FD7000420A98F8162AA120072A0ED2DFE802F0DC
:10FD80000D040B0B06080A00E52004E0B12002E098
:10FD9000312000E0F12085F8DD0E9DF810C00E9BAB
:10FDA00010980222D94EC3EB0313A1384FF0030B76
:10FDB0004FF0410E03EB8304BCF1070F7CD2DFE868
:10FDC0001CF07B0007008A02E7036A053D06B006C7
:10FDD00097F8410A4FF0000B594601F04BFD8DF8A2
:10FDE000140095F8D81E9AF8D40E814202D1012150
:10FDF0008AF8D31E99F8D009401C89F8D009109BC5
:10FE0000A221A620CE2B7DD012DC4FF0A502B92B6B
:10FE100079D006DCB22B77D0B52B35D0B62B4BD1B1
:10FE200013E1C32B71D0C52B70D0CA2BF7D101E1E0
:10FE3000E12B6CD006DCD52B09D0D72B68D0D92B81
:10FE4000EDD10FE0E52B72D0E72BE8D12DE2F520C4
:10FE500006F834009DF8140006EBC4056870A9701C
:10FE6000D52009E0F52006F834009DF8140006EBD3
:10FE7000C4056870A970D920E8702846032101F0F4
:10FE80002AFC2871052004E2F52106F834109DF8BB
:10FE9000141006EBC407797098F81C1A4FF0B508D7
:10FEA00059B1D5F8E01EB1F1104F39D34FF01041E0
:10FEB0000022CDE9081237E097E2D5F8E00EB0F560
:10FEC000100F05D34FF410000021CDE9080103E025
:10FED000D5F8E00ECDE9080BBA7058460FE0BDF832
:10FEE0000000C0F10200C200DDE90801F8F79BF94B
:10FEF000BDF800103944C870BDF80000401CADF8D2
:10FF0000000006E03BE12AE0AAE088E02CE102E103
:10FF1000D6E1BDF800000328E1D387F80680E4E0CD
:10FF2000D5F8E01ECDE9081BB870584610E0B1E1E5
:10FF3000BDF80000C0F10300C200DDE90801F8F7D8
:10FF400072F9BDF800103944C870BDF80000401CBB
:10FF5000ADF80000BDF800000428E9D35DE0F5210C
:10FF600006F834109DF8141006EBC407797098F861
:10FF70001C1A4FF0B90859B1D5F8E01EB1F1104F75
:10FF80002FD0D5F8E01ECDE9081BB87058463EE0EA
:10FF9000D5F8E00EB0F5100F06D0D5F8E01ECDE98B
:10FFA000081BBA70584615E04FF410000021CDE947
:10FFB0000801F6E7BDF80000C0F10200C200DDE96B
:10FFC0000801F8F730F9BDF800103944C870BDF8E1
:10FFD0000000401CADF80000BDF800000328E9D384
:10FFE0009BE74FF010410022CDE90812CDE7BDF8A4
:10FFF0000000C0F10300C200DDE90801F8F713F9C1
:020000040801F1
:10000000BDF800103944C870BDF80000401CADF8C0
:100010000000BDF800000428E9D340469CE0F5202C
:1000200006F834009DF8140006EBC4056870A9704A
:10003000C32021E7F52006F834009DF8140006EBF4
:10004000C4056870A970CA2016E7F52006F83400C8
:100050009DF8140006EBC4056870A970B6200BE784
:10006000F52006F834009DF8140006EBC4077870FC
:1000700098F81C0AB22110B1BA7058462EE0A4209C
:10008000B87058460EE0D5F80C0FBDF80020C2F14C
:100090000102D200D040BDF800203A44D070BDF833
:1000A0000000401CADF80000BDF800000228EAD3B3
:1000B00079713846052101F00EFBB87175E1D5F86C
:1000C0000C0FBDF80020C2F10202D200D040BDF8F2
:1000D00000203A44D070BDF80000401CADF800008C
:1000E000BDF800000328EAD3B9713846062101F0B3
:1000F000F2FA0DE0016932303130300001693230FE
:100100004530300010080020D41200200C47002099
:10011000F8710820BDE0F52106F834109DF81410A0
:1001200006EBC4077970B87058460EE0D5F8100F8A
:10013000BDF80010C1F10301C900C840BDF80010AE
:100140003944C870BDF80000401CADF80000BDF88F
:1001500000000428EAD3E120F8713846072101F0B5
:10016000BAFA3872092094E0F52006F834009DF8B8
:10017000140006EBC4056870A970C5207CE6F52064
:1001800006F834009DF8140006EBC407787098F860
:100190001C0A4FF0CE0818B1AE20B870584650E097
:1001A000AC20B870584611E0D5F8F90ED5F8FD1E10
:1001B000BDF80020C2F10402D200F8F734F8BDF80F
:1001C00000103944C870BDF80000401CADF80000B4
:1001D000BDF800000528E7D3584611E0D5F8010F17
:1001E000D5F8051FBDF80020C2F10402D200F8F7CF
:1001F0001AF8BDF8001039440872BDF80000401C20
:10020000ADF80000BDF800000528E7D387F80D80A1
:1002100038460D2101F05FFAB8730F2039E0D5F8A8
:10022000F90ED5F8FD1EBDF80020C2F10502D2007E
:10023000F7F7F9FFBDF800103944C870BDF80000A9
:10024000401CADF80000BDF800000628E7D3584672
:1002500011E0D5F8010FD5F8051FBDF80020C2F157
:100260000502D200F7F7DFFFBDF8001039444872ED
:10027000BDF80000401CADF80000BDF800000628E5
:10028000E7D387F80F8038460F2101F024FA38743D
:100290001120ADE2F52006F834009DF8140006EBBD
:1002A000C4056870A970E520E6E5F52006F834007D
:1002B0009DF8140006EBC4056870A970E720DBE523
:1002C000F52006F834009DF8140006EBC4056870AC
:1002D000A970D720D0E597F8411A8DF8141095F839
:1002E000D83E9AF8D41E8B4202D101238AF8D33E1D
:1002F00099F8D019491C89F8D0199DF8141021B12A
:100300009DF81410491E8DF814100A286DD2DFE8EC
:1003100000F041F3568CF4F1F005EF6D06F834204F
:100320009DF8140006EBC4074030787087F802E0AF
:100330003020F870387195F8DC0E00097871787902
:100340000A28787901D2303000E03730787195F89A
:10035000DC0E00F00F00B871B8790A28B87901D224
:10036000303000E03730B87187F807B0781C0721CB
:10037000F8F7D0FF38720920ADF8340095F8D80EA0
:10038000042802D1052085F8D80E00208AF8D30E63
:10039000062028E0042206F834209DF8141006EB0D
:1003A000C4004031417051213CE1072020E2287116
:1003B00085F805B0681C0521F8F7ACFFFDE30422C1
:1003C00006F834209DF8141006EBC400403141704B
:1003D00080F802E00521C170ADF8342095F8D80E00
:1003E000022802D1584685F8D80E20E106F83420BC
:1003F0009DF8140006EBC4054030687085F802E0F3
:100400003120E8703220287185F805B0681C05217C
:10041000F8F780FFA8710720ADF8340097F8420A7A
:1004200020F0200087F8420A01E106F834209DF808
:10043000140006EBC4074030787087F802E03121E1
:10044000F97030203871D5F8E02EB2F5100F00D2D7
:100450003220787195F8DE0E012803D095F8DE0E73
:1004600010B103E0B97101E03220B8710021ADF89C
:10047000001013E0D5F8E00EBDF80020C2F105022F
:100480009200D040BDF8002000F00F003A44303018
:10049000D071BDF80000401CADF80000BDF80000B0
:1004A0000628E7D332207873ADF8001013E0D5F8B2
:1004B0000C0FBDF80010C1F103018900C840BDF860
:1004C000001000F00F00394430308873BDF8000090
:1004D000401CADF80000BDF800000428E7D387F801
:1004E00012B0781C1221F8F715FFF8741420D2E32B
:1004F00080E063E163E100E06EE006F834209DF8FF
:10050000140006EBC4074030787087F802E0322010
:10051000F870312139717871B8710021ADF800108F
:1005200013E0D5F80C0FBDF80020C2F103029200D1
:10053000D040BDF8002000F00F003A443030D071B8
:10054000BDF80000401CADF80000BDF80000042814
:10055000E7D3ADF80010302008E0BDF800103944B2
:10056000C872BDF80010491CADF80010BDF80010AD
:100570001929F2D387F824B0781C2421F8F7CAFE91
:1005800087F82500262086E306EBC40148704CE07E
:1005900097F8411A8DF8141095F8D83E9AF8D41EA1
:1005A0008B4202D101238AF8D33E99F8D019491C15
:1005B00089F8D0199DF8141021B19DF81410491E26
:1005C0008DF814100A2832D2DFE800F00506224E1A
:1005D000FAF9F8311432DDE606F834209DF81400FB
:1005E00006EBC4054030687085F802E03120E87001
:1005F0003520DCE606F834209DF8140006EBC4052F
:100600004030687085F802E03220E8703020CEE695
:10061000042206F834209DF8141006EBC400403183
:100620004170714681700521C170ADF8342034E30A
:1006300006F834209DF8140006EBC40540306870BD
:1006400085F802E03120E8703220287185F805B085
:10065000681C0521F8F75EFEA87197F8420A20F0A1
:10066000200087F8420AA0E606F834209DF814001E
:1006700006EBC4074030787087F802E03121F9704A
:1006800087F804E0D5F8E00EB0F1104F09D0322021
:10069000787195F8DE0E012805D095F8DE0E20B1B0
:1006A00005E03020F4E7B97101E03220B871002292
:1006B000ADF8002013E0D5F8E00EBDF80010C1F150
:1006C00007018900C840BDF8001000F00F00394450
:1006D0003030C871BDF80000401CADF80000BDF816
:1006E00000000828E7D33220F873ADF8002013E0AB
:1006F000D5F80C0FBDF80010C1F105018900C84004
:10070000BDF8001000F00F00394430300874BDF817
:100710000000401CADF80000BDF800000628E7D33B
:100720003021B975ADF8002008E0BDF8000038446C
:10073000C175BDF80000401CADF80000BDF8000018
:100740000628F2D37977ADF8002008E0BDF8000064
:1007500038448177BDF80000401CADF80000BDF8BA
:1007600000000628F2D387F82410ADF8002009E035
:10077000BDF80000384480F82510BDF80000401C8A
:10078000ADF80000BDF800000628F1D387F82B1063
:10079000ADF8002009E0BDF80000384480F82C10C6
:1007A000BDF80000401CADF80000BDF800000628B0
:1007B000F1D387F83210ADF800200CE066E060E07D
:1007C00017E0BDF80000384480F83310BDF8000091
:1007D000401CADF80000BDF800000628F1D387F8F2
:1007E00039B0781C3921F8F795FD87F83A003B209D
:1007F00051E206F834209DF8140006EBC40740309F
:10080000787087F802E03220F87031213971332195
:100810007971B8710021ADF8001013E0D5F80C0F14
:10082000BDF80020C2F105029200D040BDF80020C2
:1008300000F00F003A443030D071BDF80000401C89
:10084000ADF80000BDF800000628E7D3ADF80010B1
:10085000302008E0BDF8001039444873BDF800109E
:10086000491CADF80010BDF800101929F2D387F823
:1008700026B0781C2621F8F74DFD87F827002820A0
:1008800009E2102006F8340030207DE6102006F83A
:100890003400312078E697F8410A8DF81400BDF84D
:1008A000000000EB40100AEB800090F8D82E9AF878
:1008B000D40E824202D101228AF8D32E99F8D0298F
:1008C000521C89F8D0290027ADF800700EE0BDF861
:1008D000002008EB021090F8410A9DF81420904285
:1008E0000AD0BDF80000401CADF8000098F8170AC7
:1008F000BDF800209042EAD8BDF8002008EB0210B5
:1009000090F8400A081A401C8DF818009DF8140051
:1009100020B19DF81400401E8DF8140095F8D90EF2
:100920000F2805D295F8D90E401C85F8D90E01E0A4
:1009300085F8D97E10996520B1394FF0FA08092958
:100940007BD2DFE801F0050C437A7A647A1D2F0030
:100950009DF81400503006F83400202166E09DF820
:100960001400503006F8340095F8D90E06EBC40593
:1009700040F0300068700120A870E8702F7136E0F8
:100980009DF81410503106F8341095F8D91E06EB76
:10099000C40541F030016970A8700120E8709DF82D
:1009A000180023E09DF81410503106F8341095F823
:1009B000D91E06EBC40541F030016970A870012012
:1009C000E8709DF8180040F010000FE09DF814004A
:1009D000503006F8340095F8D90E06EBC40540F007
:1009E000300068700120A870E87005202871284642
:1009F0000521F9F757F8CDE9080768710898000A4A
:100A0000A87185F807B085F80880FFF7ABBB95F8AB
:100A1000DA0E85F8DD0E85F8DA7E9DF81400503088
:100A200006F8340095F8D90E40F0C00106EBC4007A
:100A3000417080F8028058462DE187E0BDF8003013
:100A40000398184490F8D0395B1C80F8D03998F896
:100A50001C0A30B1491CC9B2012836D0022875D110
:100A600044E01098312802D045286FD116E00020CC
:100A7000ADF8000001A90CE0BDF80000BDF80030A1
:100A800006EBC402085CD054BDF80000401CADF871
:100A90000000BDF800000728EED386E40020ADF882
:100AA00000000AA90CE0BDF80000BDF8003006EB1C
:100AB000C402085CD054BDF80000401CADF8000032
:100AC000BDF800000728EED36FE48DF814109DF8F0
:100AD000140006F8340006EBC40585F801B00027C1
:100AE000AF70EA702F71092068710EE08DF8141054
:100AF0009DF8140006F8340006EBC40585F801B033
:100B00000027AF70EF702F716A7128460621F8F741
:100B1000D3FDCDE90807000AE8710898A871FFF72E
:100B2000F8BAF74999F8D009401C89F8D00997F824
:100B3000410A8DF814001098F32878D007DC0528B6
:100B400076D0F12808D0F22800D113E072E0F42822
:100B50006FD0F6286ED1D8E0F52006F834009DF865
:100B6000140006EBC40568700027AF700520E8701C
:100B7000F120FEE0F52006F834009DF8140006EBA5
:100B8000C40778704FF0000887F80280F2203871AF
:100B900095F8480F787195F8480F012813D095F80B
:100BA000480F20285BD00620ADF83400BDF8340093
:100BB000F8703846BDF8341000E0E4E0F8F77CFD4A
:100BC000CDE9080848E12520ADF834004146ADF8EC
:100BD00000800DE0BDF80000284490F8210FBDF81A
:100BE00000203A449071BDF80000401CADF80000B0
:100BF000BDF800000F28EDD3ADF800100DE0BDF8F2
:100C00000000284490F8330FBDF800203A44507596
:100C1000BDF80000401CADF80000BDF800000A2837
:100C2000EDD395F8420FF877ADF8001012E03FE0F1
:100C3000AEE091E031E0BDF80000284490F8430FA9
:100C4000BDF80010394481F82000BDF80000401CB8
:100C5000ADF80000BDF800000528ECD3A6E70A2097
:100C6000ADF8340040460BE0BDF80000284490F891
:100C7000430FBDF8001039448871BDF80000401CD6
:100C8000ADF80000BDF800000428EDD38EE74870F1
:100C9000BDF83400801CADF834009A489A4D0E9986
:100CA00091B3012971D0022970D003296FD107E1D6
:100CB000F52006F834009DF8140006EBC4077870A0
:100CC0004FF00008404687F80280F321397195F80B
:100CD000481F79710C21ADF8341095F8421FB97195
:100CE0000BE0BDF80000284490F8430FBDF8001059
:100CF0003944C871BDF80000401CADF80000BDF8D3
:100D000000000528EDD351E7AFE00620ADF8340030
:100D1000F52006F834009DF8140006EBC405687051
:100D20004FF0000885F80280BDF83400E870F62026
:100D3000287197F8480A68712846BDF83410F8F70A
:100D4000BBFCCDE90808BDF83410000A6854BDF8B2
:100D50003410089829449AE7F52006F834009DF8E5
:100D6000140006EBC40568700027AF700520E8701A
:100D7000F420287128460521F8F79EFCCDE90807E4
:100D8000000A68710898A8716DE47CE088E0A6E02C
:100D900040F21320ADF83400F52006F834009DF839
:100DA000140006EBC4077870BDF83400000AB87070
:100DB000BDF83400F870052038714FF0000948463E
:100DC0000CE0BDF8002008EB020090F81E0ABDF808
:100DD00000203A445071BDF80000401CADF80000FE
:100DE000BDF800000A28ECD3B8F82A0A8A46000A9F
:100DF000F873B8F82A0A3874B5F8560F000A7874F0
:100E0000B5F8560FB874B5F8561F0E9801EB802050
:100E100081B20320F8F770F84D46ADF800905046C7
:100E20004FF400720DE0BDF80010014491F8661017
:100E3000BDF800303B44D974BDF80010491CADF832
:100E40000010BDF800109142EDD33846BDF83410C3
:100E5000F8F732FCCDE90805BDF83410000A7854E3
:100E6000BDF834100898394411E7BDF83410B1B317
:100E70008021F9F7CCFABDF83400C5F8A400224867
:100E80000121A03029E0BDF8341041B30821F9F761
:100E9000BEFABDF8340068671B48012170301CE0C1
:100EA000BDF83400D8B14FF480711848F9F7AFFAA3
:100EB000BDF83400C5F8BC0013480121B8300CE07F
:100EC000BDF8341059B14FF48061F9F7A0FABDF8BC
:100ED0003400E8650C4801215830F8F743FC084815
:100EE00090F86702002807D006EBC4000023BDF885
:100EF00034100E9AF9F742FD11B0BDE8F08F0000F2
:100F0000D4120020000C02400060024000000240A9
:100F10002DE9F04700242DED048B804689469FED96
:100F20001E9B25462646E20040464946F7F77BF9D8
:100F3000C7B22046F7F745FB41EC110BB0EE490A6A
:100F4000F0EE690A06F084FD380907F00F0100EBA6
:100F50008000B0EE408AF0EE608A01EB4000F7F7C7
:100F600030FB53EC182BF7F74BFA41EC180B2846E3
:100F70003146F7F733FB53EC182BF7F79AF9F7F7ED
:100F800060FB641CE4B205460E46082CCBD3BDECD6
:100F9000048BBDE8F087000000000000000059400D
:100FA00070B50F4D40F224442146284606F0EBF977
:100FB000012813D1298828462A1D1188214606F0C8
:100FC0007FF90849012081F871090748D0F88C00A1
:100FD00001F50051C0F57A70A1F8F80F70BD00005E
:100FE00000440040D41200200060024010B50C4CB8
:100FF00040F22441204606F0C6F901280ED120888F
:10100000201D00880749012081F87D090648406CB1
:1010100001F50051C0F57A70A1F8FA0F10BD00007B
:10102000004C0040D41200200060024010B50B4C70
:1010300040F22441204606F0A6F901280DD120886F
:10104000A0880749012081F889090648406901F50F
:101050000051C0F57A70A1F8FC0F10BD005000409F
:10106000D41200200060024010B50C4C40F2244124
:10107000204606F088F901280ED12088201D00881E
:101080000749012081F895090648C06A01F5005119
:10109000C0F57A70A1F8FE0F10BD000000480040B6
:1010A000D41200200060024010B5124C10492046B6
:1010B000F8F742FB00212046F8F754FB0E4C402184
:1010C000204606F059F90028F9D080210B48F9F79D
:1010D000A0F9084C0A49183C2046F8F72DFB0121DD
:1010E0002046F8F73FFB07490120087110BD0000BA
:1010F00000802020A060024000440040000C02401C
:10110000008800201008002010B5124C104920461D
:10111000F8F712FB00212046F8F724FB0E4C402183
:10112000204606F029F90028F9D008210B48F9F7E4
:1011300070F9084C0A49303C2046F8F7FDFA0121C5
:101140002046F8F70FFB07490120087110BD000089
:101150002080002070600240004C0040000C0240E3
:10116000008020101008002010B5124C10492046B5
:10117000F8F7E2FA00212046F8F7F4FA0E4C402185
:10118000204606F0F9F80028F9D04FF480710B489A
:10119000F9F73FF9074C0A49A83C2046F8F7CCFA82
:1011A00001212046F8F7DEFA06490120087110BD3A
:1011B00000800028B860024000500040000002405B
:1011C000208000101008002010B5124C1049204655
:1011D000F8F7B2FA00212046F8F7C4FA0E4C402185
:1011E000204606F0C9F80028F9D04FF480610B487A
:1011F000F9F70FF9074C0A49303C2046F8F79CFAFA
:1012000001212046F8F7AEFA06490120087110BD09
:10121000008000185860024000480040000C024066
:1012200000880010100800202DE9F047012190B03F
:10123000480503F093FF8648F8F79EFA40273801E7
:101240000024CDE90540C50107940894CDE909457E
:1012500046040C940D94DFF8FC917F480B94CDE983
:101260000207CDE9006969460E947948F8F72CFB2E
:10127000012210217648F8F711FBDFF8D4A1AAF17A
:10128000180A5046F8F778FA4FF47A78CDE903480F
:10129000E811CDE9054007940894CDE909456F4868
:1012A0000B940C940D9400960E94CDE90190694630
:1012B0005046F8F709FB01215046F8F753FADFF8DA
:1012C00090A1AAF1300A5046F8F756FAE811CDE994
:1012D000054007940894CDE909450C940D94DFF876
:1012E000809160480B94CDE90207CDE90069694619
:1012F0000E945046F8F7E8FA012210215046F8F70C
:10130000CDFADFF84CA1AAF1600A5046F8F734FA9A
:10131000CDE90348E811CDE9054007940894CDE9EB
:10132000094551480B940C940D9400960E94CDE908
:10133000019069465046F8F7C7FA01215046F8F780
:1013400011FADFF80CA10AF1180A5046F8F714FA5E
:10135000E811CDE9054007940894CDE909450C94BE
:101360000D94DFF8089142480B94CDE90207CDE9CE
:10137000006969460E945046F8F7A6FA012210213A
:101380005046F8F78BFADFF8C8A0AAF1900A504649
:10139000F8F7F2F9CDE90348E811CDE905400794E3
:1013A0000894CDE9094533480B940C940D940096AC
:1013B0000E94CDE9019069465046F8F785FA01216F
:1013C0005046F8F7CFF9DFF88890A9F14809484668
:1013D000F8F7D2F90397E811CDE90540079408948E
:1013E000CDE9094525480B940C940D94224F0096A5
:1013F0000E94CDE9017069464846F8F765FA012276
:1014000010214846F8F74AFADFF84490A9F1780924
:101410004846F8F7B1F9CDE90348E811CDE90540B0
:1014200007940894CDE9094515480B940C940D9444
:1014300000960E94CDE9017069464846F8F744FAE3
:1014400001214846F8F78EF910B0BDE8F08700009A
:10145000A0600240044400400C4700206C50002073
:10146000044C0040644900205454002004500040C3
:10147000BC4B00203C58002004480040144E002083
:10148000245C00202DE9FC410121084603F066FEA2
:101490000121042003F062FE0121082003F05EFE1A
:1014A0000121402003F05AFEDFF8FC8007220521CD
:1014B0004046F8F795FF072206214046F8F790FFCF
:1014C000072208214046F8F78BFF072209214046F2
:1014D000F8F786FF354F08220A213846F8F780FFD3
:1014E00008220B213846F8F77BFF082202214046EC
:1014F000F8F776FF08220C213846F8F771FF02262C
:101500008DF8056000244FF459708DF806400125D0
:1015100000908DF807508DF8046069464046F8F752
:1015200023FF8DF805604FF4E0508DF806400090E1
:101530008DF807508DF8046069463846F8F714FFB7
:101540004FF4916000908DF806408DF80450694684
:101550004046F8F709FF280200908DF806408DF804
:10156000045069461248F8F7FFFE8DF806404FF424
:10157000F040104C00908DF8045069462046F8F772
:10158000F3FEA9032046F8F742FF69032046F8F767
:101590003EFFA1142046F8F73AFFE1142046F8F781
:1015A00036FFBDE8FC810000000C0240000802404C
:1015B000000002400018024070B50024FFF762FFEF
:1015C000FFF732FE00F022F80E4D002185F86C196D
:1015D000012285F86C290C48017081704170C2703D
:1015E0004FF47A718160042085F86C0904E020468C
:1015F00000F062F9641CE4B295F86C09A042F6D8D8
:1016000070BD0000D412002010430020F8B5112056
:101610008DF8000002258DF8015001248DF802405C
:101620008DF80340684600F0EBFA26208DF80000A4
:101630008DF8014000268DF802608DF80340684661
:1016400000F0DEFA0E208DF800008DF801508DF8C4
:1016500002408DF80340684600F0D2FA27208DF84A
:1016600000008DF801408DF802608DF80340684657
:1016700000F0C6FA0F208DF800008DF801508DF8AB
:1016800002408DF80340684600F0BAFA34208DF825
:1016900000008DF801408DF802608DF80340684627
:1016A00000F0AEFA2F208DF800008DF801508DF873
:1016B00002408DF80340684600F0A2FA35208DF80C
:1016C00000008DF801408DF802608DF803406846F7
:1016D00000F096FAF8BD01B9102110F8012B10F8AE
:1016E000013B491E5A400904090CF8D102F07F0061
:1016F000704700002DE9FF5F14460F464FF48056F7
:101700004FF480684FF4C0694FF00C0A40F2244B4C
:10171000002580B1012830D0022851D0032871D192
:101720000121880403F03EFD0097012C6DD0022CAE
:1017300070D094B377E00121480403F033FD0097A3
:10174000012C03D0022C06D054B10DE0ADF804609A
:10175000ADF8088008E0ADF80460ADF8089003E04B
:10176000ADF80450ADF80850ADF80650ADF80C5087
:10177000ADF80AA069463B4C5DE00121C80403F0C6
:1017800011FD0097012C03D0022C07D05CB10EE0B4
:10179000ADF80460ADF8088009E040E0ADF8046001
:1017A000ADF8089003E0ADF80450ADF80850ADF87E
:1017B0000650ADF80C50ADF80AA069462A4C3AE044
:1017C0000121080503F0EEFC0097012C03D0022C48
:1017D00006D054B10DE0ADF80460ADF8088008E023
:1017E000ADF80460ADF8089003E0ADF80450ADF832
:1017F0000850ADF80650ADF80C50ADF80AA0694697
:101800001A4C18E02CE000E004E0ADF80460ADF8FC
:10181000088008E0ADF80460ADF8089003E0ADF88A
:101820000450ADF80850124CADF80650ADF80C500D
:10183000ADF80AA06946204605F0DCFD01212046EE
:1018400005F041FD01225946204605F0BBFD10215F
:10185000204605F035FD0122C021204605F03DFD62
:10186000BDE8FF9F00440040004C00400050004095
:10187000004800402DE9FC410024CDE900446F46BA
:1018800064220023F6F79EFC0E46054610461946D4
:101890000A220023F6F796FC010102F00F00081857
:1018A000385504F10104E4B228463146082CE7D348
:1018B000DDE90001BDE8FC812DE9F05F644F4FF0E8
:1018C000040A0646002587F86CA900EB460000EBE9
:1018D000061007EB001494F81D0A012803D100211B
:1018E000304600F0B7F806EB4602B84607EB820731
:1018F0004FF0000B87F870B987F872B987F871B9A3
:1019000087F873B94FF00509C7F8789987F8A0B937
:1019100087F8A2B9012087F8A10987F8A309D4F8AC
:10192000180A00EB80004000C7F8A80994F8152AAF
:10193000D4F8101A3046FFF7DDFE94F8160A06EBCD
:10194000C601434A01EB062102EBC106072815D266
:10195000DFE800F01404060A0C0E1800484600E008
:101960000F2086F8D40E09E00720FAE75046F8E782
:10197000D4F8180A64214843C7F8A8094FF0A10A0F
:10198000C1465EE00320ECE705EB451006EB800066
:1019900080F8E4BE012380F8E63E80F8E5BE80F8DA
:1019A000E7BE4FF47A73C0F8EC3E04EB051383F8FE
:1019B00042BA80F8D8BE94F8161A07293FD2DFE859
:1019C00001F03E0408080A0C0E00E52180F8DD1E37
:1019D00035E05146FAE7B121F8E73121F6E7F12188
:1019E00080F8DD1E002125E001EBC10707EB012790
:1019F00001EB410C02EBC7070CEB011C002009EBCB
:101A00000C1211E002EB001C9CF840CA93F8488AC3
:101A1000C44507D193F840CA00EB401807EB88088B
:101A200088F849CF401CC0B292F817CA8445E9D85B
:101A3000491CC9B299F86C094A468842D4D86D1C31
:101A4000EDB294F8170AA8429ED8BDE8F09F0000B6
:101A5000D41200202DE9F041054661484FF4804240
:101A6000531006685F488414C71439B1C5B1012DFD
:101A700018D0022D18D0032D1BD117E035B1012D40
:101A800006D0022D06D0032D13D105E0114604E047
:101A9000194602E0214600E03946F8F7BAFC08E0B2
:101AA000114604E0194602E0214600E03946F8F705
:101AB000AEFC642007F020F900224FF416512846AE
:101AC000FFF718FEDFF8208105EB450008EB8000EA
:101AD000002280F8A229C0F8A42905EB450000EBFC
:101AE000051008EB0011D1F8183A08F5405043648E
:101AF000012380F83D3091F8161A3C4C962305EBF3
:101B00008500204406290AD2DFE801F00903050513
:101B10000733762102E0837001E06E218170C5EB0E
:101B20000511334B01EB8101C02403F8314003EB75
:101B3000C10462700821A170E27006F00F0105EB8C
:101B4000051211442171807860712020A071E1712B
:101B5000802020724C2060725420A0722548264FAD
:101B60000B2645B1012D0FD0022D24D0032D14D109
:101B70002CE06621D2E78021F8F749FCC7F8A46081
:101B80001D480121A03006E00821F8F740FC7E67DF
:101B9000194801217030F7F7E5FD98F8670228B180
:101BA000204600232A460B21F8F7E8FEBDE8F04165
:101BB000642007F0A1B84FF480711048F8F727FCB3
:101BC000C7F8BC600C480121B830E4E74FF48061ED
:101BD000F8F71DFCFE65084801215830DBE70000DE
:101BE000187AFF1F00180240D41200200C60002059
:101BF0000C470020000C0240006002400000024040
:101C000030B50F23C27801780125FAB1144A126861
:101C100001F1E02102F4E062C2F5E062C2F30722C2
:101C2000C2F10404D3404278A24084781C4014439B
:101C3000220181F80024007800F01F018D40400946
:101C4000800000F1E020C0F8005130BD01F01F001D
:101C500085404809800000F1E020C0F8805130BD87
:101C60000CED00E0024A1140014302480160704758
:101C700080FFFF1F08ED00E0BFF34F8F04480168AD
:101C8000044A01F4E06111430160BFF34F8FFEE7A6
:101C90000CED00E00400FA0510B50021074B0A46E0
:101CA000002003EBC004401CC0B262548028F8D36B
:101CB000491CC9B20829F3D310BD00000F6A0020E7
:101CC0002DE9FE4F0026171A8146701E3546A3EBFC
:101CD000010A8846002F02DD4FF0010102E003D126
:101CE0004FF00001019102E0C7F100070190BAF145
:101CF000000F02DD4FF0010002E003D14FF00000C1
:101D0000009002E0C7F1000A00905046574501DDFF
:101D10003C4600E00446601C4FF0000B029016E0C9
:101D200008F0FF0109F0FF000C9A00F015F83E449E
:101D30005544A64202DD0199361B8944A54202DDC5
:101D400000992D1B88440BF101001FFA80FB0299BA
:101D50008B45E5DBBDE8FE8F30B5CC0801F007030D
:101D600001259D40EBB2064D05EBC005C808285C77
:101D70000AB1184302E063EA0000C043285530BDB1
:101D80000F6A00202DE9FC4101210A2003F0E6F949
:101D900001248DF8044000264FF4C0508DF80660F1
:101DA000032700908DF805708DF807406946464876
:101DB000F8F7DAFA8DF804408DF806608DF80570B2
:101DC000A5028DF80740414C009569462046F8F77A
:101DD000CBFAC82006F090FF29462046F8F717FBFB
:101DE000C82006F089FF29462046F8F712FBC820D4
:101DF00006F082FF0021FD2000F024FA00211220CD
:101E000000F020FA0021AE2000F01CFA0021D520BD
:101E100000F018FA0021A02000F014FA0021A820F8
:101E200000F010FA00213F2000F00CFA0021D3202E
:101E300000F008FA0021084600F004FA00214020D2
:101E400000F000FA0021A02000F0FCF90021C020E1
:101E500000F0F8F90021DA2000F0F4F90021122056
:101E600000F0F0F90021812000F0ECF900217F2042
:101E700000F0E8F90021D92000F0E4F900218220E7
:101E800000F0E0F90021DB2000F0DCF90021342033
:101E900000F0D8F90021A42000F0D4F90021A620F8
:101EA00000F0D0F90021202000F0CCF900210846F4
:101EB00000F0C8F9FFF7F0FE0021AF2000F0C2F9F2
:101EC00000F054F8BDE8FC81000C02400004024020
:101ED0000346012000E05843491EC9B2FBD27047B7
:101EE0002DE9F84F82460A980D4650436421B0FB15
:101EF000F1F0984600F0FF0B4FF001090AEB0207E2
:101F00002B4600245046FAB21946CDF80090FFF750
:101F1000D7FE05EB0806F3B2FAB2F1B25046CDF89F
:101F20000090FFF7CDFE5246F3B229461046CDF899
:101F30000090FFF7C5FEF3B2FAB2F8B22946CDF829
:101F40000090FFF7BDFE4F460AEB0B0609E028198B
:101F5000C3B2C1B2F2B250460097FFF7B1FE641CA3
:101F6000E4B24445F3D3BDE8F88F000070B5002516
:101F7000B020294600F066F90021084600F062F919
:101F80000021102000F05EF9084E002406EBC4008A
:101F90000121405D00F056F9641CE4B2802CF5D3B9
:101FA0006D1CEDB2082DF0D370BD00000F6A00204B
:101FB00070B50B4C05460221204603F099FA002823
:101FC000F9D02946204603F09CFA0121204603F06F
:101FD0008FFA0028F9D0204603F091FAC0B270BD04
:101FE000003800402DE9FC4F1D46884681468B464F
:101FF0000090082B0ED0680700D0012000EBD50020
:10200000690810FB01F0C0B2203A02F0FF0A002676
:10201000019046E00620F7E7082D10D00C2D14D0D3
:10202000102D16D0182D3FD121490AEBCA0001EB23
:1020300080000027845DE0070FD00B9A10E01D4957
:102040000AEB4A0001EB4000F3E70AEB4A001A49A9
:10205000EDE71A4901EB0A10EBE70B9830B30022C9
:1020600041464846FFF778FE7F1C640808F10100EE
:10207000FFB200F0FF08082FDDD309F1010000F0E6
:10208000FF09082D0AD00099A9EB0100B0EB550F0C
:1020900004D10BF10800894600F0FF0B761CD846EE
:1020A000F6B201988642B7D3BDE8FC8F0122D7E78C
:1020B0009CA5010810990108389B0108AC9F0108F4
:1020C0002DE9F84F1D00DDE90A7992468B468046DE
:1020D0004FF0000611D11046F6F773FA41EC100BE1
:1020E00005F01EFC9FED1C1B51EC100B53EC112B4B
:1020F000F6F7DFF8F6F786FAC5B2082F00D1022608
:1021000000241CE0281B401EC1B20A20FFF7E0FE9D
:10211000BAFBF0F00A21B0FBF1F201FB1200CDF89E
:10212000009088B13030C2B206EB570101FB048049
:10213000C0B23B465946FFF755FF641CE4B2AC42BF
:10214000E0D32846BDE8F88F06EB570101FB048079
:10215000C0B23B463022EDE7000000000000F03F37
:102160002DE9FF4F81B0064600900F464FF0000A60
:102170008946580700D0012000EBD30004900020CE
:1021800032E0002029E00E98002410F80A500AF1ED
:1021900001001FFA80FAE80701D00F9A02E00F98B9
:1021A00048B3002239463046FFF7D6FD7F1C641C39
:1021B0006D08E4B2FFB2082CEDD3761C0098F6B29D
:1021C000311A0398814204D109F10800009E00F001
:1021D000FF0908F101004F46C0B2039980468842CA
:1021E000D1D30BF10100C0B2049983468842C8D311
:1021F00005B0BDE8F08F0122D4E72DE9F8431D4674
:10220000DDE908781646894604460EE03B46494615
:102210002046CDF80080FFF7E5FE082F0ED004EB36
:102220005700C4B26D1EEDB2761C002D04D032787A
:10223000202A01D37E2AE9D9BDE8F883A41DE4B29F
:10224000F0E700002DE9F041114C06464FF400651F
:1022500000292946204602D0F8F7DBF801E0F8F71C
:10226000D6F84FF4805739462046F8F7D0F839466B
:102270000848F8F7CEF83046FFF79AFE3946204670
:10228000F8F7C7F829462046BDE8F041F8F7C1B88D
:10229000000C0240000402402DE9F04F87B00027F7
:1022A000ADF80C70ADF80470ADF80870ADF81470AE
:1022B000ADF81070ADF800704FF0F20B4FF0A30ABC
:1022C000FC4EDFF8F483FCE394F82306022802D1E5
:1022D0000720ADF80000BDF8000030448079BDF85B
:1022E00000103144C97840EA0160BDF80010314463
:1022F0000979BDF8002009043244527941EA0221EB
:102300000843EE494A68904277D04860BDF8000023
:1023100030448078BDF800103144497840EA012506
:10232000B4F8EA14BDF800002844801C814264D34C
:10233000B4F8EA04BDF80010401B401A801EA4F84F
:10234000EA04BDF8000029463044F7F7B5F9BDF8B6
:102350000010294431444978BDF800202A44B25C79
:1023600041EA0221814279D194F86702A04640B146
:10237000A81C81B2BDF80000012330440422F8F704
:10238000FDFABDF800003044007900F0010004902F
:10239000BDF80000304480790024C0F34209EB1FEF
:1023A0000DE020443044C0794A460499F7F790FB89
:1023B000BDF8001021443144C871641CA4B2BDF8BA
:1023C00000009C42EDDB3044C079012188F82116E1
:1023D0004FF00009C8F8289588F82695B84A82F881
:1023E0003290C2F83490ADF8149011287ED00DDCF4
:1023F000A0F10B00062815D200E0FCE3DFE810F0A6
:1024000007086D08A5089F089F0A1D00A2286FD025
:1024100004DC12286DD0A12804D1F5E2A32869D0EC
:10242000A42868D000204946BDF800200244B154D9
:10243000401C80B20528F7D3F2E3ADF80C90444677
:10244000D2E1BDF80C0000EB400101EB001004EB01
:10245000001090F8160A07287DD200E0F3E3DFE8C9
:1024600000F07A040404047A9B00484682E0BDF838
:102470000000BDF8141008443044007AB8B30128B5
:1024800002D002286ED112E0BDF80C0000EB400132
:1024900001EB0010BDF8041004EB001000EB01107C
:1024A00090F8421A21F0040180F8421A5AE0BDF86F
:1024B0000C0000EB400101EB0010BDF8041004EB30
:1024C000001000EB011090F8421A21F0080180F88A
:1024D000421ABDF80C0000EB400202EB0010BDF800
:1024E000042004EB001000EB021005E0FDE339E0EE
:1024F000FCE3FCE3FCE3FCE3C0F8449ABDF80C10F9
:102500000220F7F779FB00204A46BDF80C1001EBDA
:10251000C10303EB012104EBC103BDF8041001EB7F
:10252000411103EB8101014481F8172F401C80B257
:102530001428EAD30020BDF80C1001EBC10303EB13
:10254000012104EBC103BDF8041001EB411103EBC1
:102550008101014400E042E181F8332F401C80B248
:102560000A28E8D3BDF81400401CADF81400BDF8EB
:102570000400401CADF80400BDF80C0000EB400165
:1025800001EB001004EB001090F8170ABDF80410DE
:1025900088423FF66CAF22E1CC46ADF804900FE1E3
:1025A000BDF80000BDF8141008443044007A042837
:1025B00005D005DC58B1012840D0022879D11BE1B3
:1025C00008287FD010287ED0202872D1C1E1BDF824
:1025D0000C0000EBC00101EB002004EBC001BDF8D2
:1025E000040000EB401001EB800090F8480F102829
:1025F00020D1BDF80C0000EBC00101EB002004EB82
:10260000C001BDF8040000EB401001EB800080F831
:1026100048CFBDF80C00F32100EBC00202EB002014
:1026200004EBC002BDF8040000EB401002EB800098
:1026300080F8DD1EBDF81400401CBAE0BDF80C00A7
:1026400000EBC00202EB002004EBC002BDF8040066
:1026500000EB401002EB800080F8DDBEBDF80C00FE
:1026600000EB400101EB0010BDF8041004EB00107A
:1026700000EB011090F8421A21F0080180F8421A8C
:10268000BDF80000BDF8141008443044017ABDF8CC
:102690000C0000EBC00202EB002004EBC002BDF80E
:1026A000040000EB401002EB800080F8481F00207F
:1026B0000AE080E020600020D4120020180A0020E8
:1026C000D442002098E0D1E0BDF80010BDF81420FD
:1026D0001144014431444A7ABDF80C1001EBC103A6
:1026E00003EB012104EBC103BDF8041001EB411120
:1026F00003EB8101014481F8212F401C80B20F2897
:10270000D6D30020BDF80010BDF8142011440144B8
:1027100031440A7EBDF80C1001EBC10303EB01212B
:1027200004EBC103BDF8041001EB411103EB81017F
:10273000014481F8332F401C80B20A28E2D3BDF84F
:102740000000BDF814100844304490F82200BDF891
:102750000C1001EBC10202EB012104EBC102BDF838
:10276000041001EB411102EB810181F8420F0020BE
:10277000BDF80010BDF8142011440144314491F813
:102780002320BDF80C1001EBC10303EB012104EB86
:10279000C103BDF8041001EB411103EB81010144B9
:1027A00081F8432F401C80B20528E1D3BDF8140006
:1027B0002030ADF81400BDF80400401CADF8040052
:1027C000BDF80C0000EB400101EB001004EB001021
:1027D00090F8170ABDF8041088423FF6E1AEBDF844
:1027E0000C00401CADF80C0094F86C09BDF80C10FE
:1027F00088423FF626AE1FE6BDF80C0000EBC00293
:1028000002EB002004EBC002BDF8040000EB401016
:1028100002EB800080F8DDBEBDF80C0000EB40014B
:1028200001EB0010BDF8041004EB001000EB0110E8
:1028300090F8421A21F0080180F8421ABDF8000011
:10284000BDF8141008443044017ABDF80C0000EBC8
:10285000C00202EB002004EBC002BDF8040000EB54
:10286000401002EB800080F8481FE3E6BDF80C0042
:10287000F32100EBC00202EB002004EBC002BDF824
:10288000040000EB401002EB800080F8DD1EBDF874
:102890000C0000EB400101EB0010BDF8041004EB4C
:1028A000001000EB011090F8421A21F0080180F8A6
:1028B000421ABDF80000BDF8141008443044017AF3
:1028C000BDF80C0000EBC00202EB002004EBC002DC
:1028D000BDF8040000EB401002EB800080F8481FB8
:1028E000BDF80000BDF8141008443044417ABDF82A
:1028F0000C0000EBC00202EB002004EBC002BDF8AC
:10290000040000EB401002EB800080F8421F002022
:10291000BDF80010BDF814201144014431448A7AF6
:10292000BDF80C1001EBC10303EB012104EBC10363
:10293000BDF8041001EB411103EB8101014481F862
:10294000432F401C80B20528E2D3BDF81400C01DFF
:102950002FE7BDF80C0000EBC00202EB002004EBF7
:10296000C002BDF8040000EB401002EB800080F8CC
:10297000DDBEBDF80C0000EB400101EB0010BDF81E
:10298000041004EB001000EB011090F8421A21F043
:10299000080180F8421ABDF80000BDF81410084480
:1029A0003044017ABDF80C0000EBC00202EB0020BD
:1029B00004EBC002BDF8040000EB401002EB800005
:1029C00080F8481F0020BDF80010BDF81420114405
:1029D000014431444A7ABDF80C1001EBC10303EB0A
:1029E000012104EBC103BDF8041001EB411103EB1D
:1029F0008101014481F8432F401C80B20428E2D3B6
:102A0000BDF81400401DD4E6A81E0D2190FBF1F086
:102A1000C0B20490ADF80C904446ACE1484686E163
:102A2000BDF80C0000EB400101EB0010BDF80410F4
:102A300004EB001000EB011090F8420A80077DD4EF
:102A400007EB8700BDF8001000EBC70008443044D6
:102A5000007A0021FEF75CFABDF80C2002EB42037D
:102A600003EB0212BDF8043004EB021202EB031276
:102A700092F8402A89EA010342401A435ED1BDF828
:102A80000C0000EBC00101EB002004EBC001BDF81D
:102A9000040000EB401001EB800090F8150F0128B6
:102AA0007DD1BDF800003044407BBDF800103144BA
:102AB000897A40EA0161BDF800003044C07A000420
:102AC00000E0FDE3BDF800203244127B40EA022022
:102AD0000143BDF80C0000EBC00202EB002004EB48
:102AE000C002BDF8040000EB401002EB8000C0F80B
:102AF000E01EBDF800003044007DBDF800103144F8
:102B0000497C40EA0160BDF800103144897CBDF881
:102B1000002009043244D27C41EA02210843BDF876
:102B20000C1001EB410202EB0111BDF8042004EB93
:102B3000011101EB0211C1F8440A00E0F4E0BDF814
:102B40000C0000EB400101EB0010BDF8041004EB99
:102B5000001000EB011090F8421A41F0200180F8BB
:102B6000421ABDF80C100220F7F746F8BDF80C0029
:102B700000EB400101EB0010BDF8041004EB001065
:102B800000EB011090F8401ABDF80C0000EBC002F9
:102B900002EB002004EBC00080F8D11E00E051E001
:102BA000BDF80C0000EB400101EB001004EB00103D
:102BB00090F8160A012804D0022847D0032841D1F2
:102BC00044E0BDF800003044407A10B1012839D10A
:102BD0003AE0BDF80C0000EB400101EB001004EB03
:102BE000001090F81C0A0028BDF80C0000EBC00192
:102BF00001EB002000E0FDE304EBC001BDF80400A0
:102C000000EB401001EB8000D0F8E00E03D0B0F1F3
:102C1000104F03D105E0B0F5100F02D0B52101E04F
:102C2000B0E0C321BDF80C0000EBC00202EB0020B5
:102C300004EBC002BDF8040000EB401002EB800082
:102C400080F8DD1E6BE0FCE3B921EBE7BDF80C007A
:102C500000EBC00101EB002004EBC001BDF8040053
:102C600000EB401001EB800090F8D81EBDF80C007E
:102C700000EBC00202EB002004EBC00090F8D40E81
:102C800081424CD1BDF800003044807BBDF800107B
:102C900000043144C97B40EA0121BDF80000304402
:102CA000007C0143BDF80C0000EBC00202EB0020E9
:102CB00004EBC002BDF8040000EB401002EB800002
:102CC000C0F80C1FBDF800003044417ABDF80C007C
:102CD00000EBC00202EB002004EBC002BDF80400D0
:102CE00000EB401002EB800004E0F0E302E1EFE3D0
:102CF00028E248E080F8DE1EBDF80C00A42100EBBD
:102D0000C00202EB002004EBC002BDF8040000EB9F
:102D1000401002EB800080F8DA1E514682E77F1CEB
:102D20000498FFB2874213D2BDF80400401CADF8EE
:102D30000400BDF80C0000EB400101EB001004EBB7
:102D4000001090F8170ABDF8041088423FF668AEEC
:102D5000BDF80C0000EB400101EB001004EB00108B
:102D600090F8170ABDF8041088420BD8BDF80C0083
:102D7000401CADF80C0094F86C09BDF80C108842AA
:102D80003FF64CAE01E1ADF80C90444642E0ADF8A0
:102D900004901EE0BDF800003044007A0021FEF7E8
:102DA000B7F8BDF80C2002EB420303EB0212BDF8AA
:102DB000043004EB021202EB031292F8402A89EA73
:102DC000010342401A432CD0BDF80400401CADF86A
:102DD0000400BDF80C0000EB400101EB001004EB17
:102DE000001090F8170ABDF804108842D2D8BDF838
:102DF0000C0000EB400101EB001004EB001090F818
:102E0000170ABDF804108842BCD8BDF80C00401C5D
:102E1000ADF80C0094F86C09BDF80C108842B6D8D7
:102E2000B3E0BDF80C0000EB400101EB0010BDF871
:102E3000041004EB001000EB011090F8401ABDF8EC
:102E40000C0000EBC00202EB002004EBC00080F895
:102E5000D11EBDF80C0000EB400101EB001004EBAB
:102E6000001090F8160A012832D0022801D0032859
:102E7000BDD1BDF80C0000EBC00101EB002004EB5C
:102E8000C001BDF8040000EB401001EB800090F899
:102E9000D81EBDF80C0000EBC00202EB002004EBD2
:102EA000C00090F8D40E8142A1D1BDF80C00AA2137
:102EB00000EBC00202EB002004EBC002BDF80400EE
:102EC00000EB401002EB800080F8DA1E514600E073
:102ED000CA21BDF80C0000EBC00202EB002004EB9D
:102EE000C002BDF8040000EB401002EB800080F847
:102EF000DD1E7CE7484640E0ADF804901EE0BDF8DA
:102F000000003044007A0021FEF702F8BDF80C20E2
:102F100002EB420303EB021308EB0312BDF804308B
:102F200002EB031292F8402A89EA010342401A4355
:102F30002CD0BDF80400401CADF80400BDF80C0016
:102F400000EB400101EB001108EB011090F8170AAB
:102F5000BDF804108842D2D8BDF80C0000EB400147
:102F600001EB001108EB011090F8170ABDF80410EE
:102F700088420AD8BDF80C00401CADF80C0098F847
:102F80006C09BDF80C209042B6D85FE1BDF80C008A
:102F9000BDF8042000EB400101EB0010414608EBB6
:102FA000001000EB021090F8402ABDF80C0000EB76
:102FB000C00303EB002008EBC00080F8D12EBDF861
:102FC00000003044407ABDF8002000043244927A78
:102FD00040EA0222BDF800003044C07A0243BDF846
:102FE0000C0000EBC00303EB002001EBC003BDF8B5
:102FF000040000EB401003EB8000C0F80C2FBDF87C
:103000000C0000EB400202EB001001EB001090F806
:10301000160A012841D0022801D003289CD1BDF80E
:103020000C0000EBC00202EB002001EBC002BDF877
:10303000040000EB401002EB800090F8D82EBDF8A1
:103040000C0000EBC00303EB002001EBC00090F884
:10305000D40E824280D1BDF80C00A52200EBC00343
:1030600003EB002001EBC003BDF8040000EB4010AF
:1030700003EB800080F8DA2EBDF80C0000EBC003F3
:1030800003EB002008EBC001BDF8040000EB40108A
:1030900001EB800080F8DDAE5EE7BDF80C0000EBD0
:1030A000C00202EB002001EBC002BDF8040000EBFF
:1030B000401002EB800090F8D82EBDF80C0000EB19
:1030C000C00303EB002001EBC00090F8D40E824255
:1030D000E2D1BDF80C00B22200EBC00303EB0020EC
:1030E00001EBC003BDF8040000EB401003EB8000CF
:1030F00080F8DA2EBDF80C00E52200EBC00303EBEC
:10310000002001EBC003BDF8040000EB401003EB0E
:10311000800080F8DD2E002CBED1BDF8040001280F
:10312000BAD1BDF80C0000EBC00202EB002008EBA6
:10313000C001BDF8040000EB401001EB8000D0F8A6
:103140000C0F09E7BDF800003044007A05287DD255
:10315000BDF800003044007A401EADF80C00BDF808
:1031600000003044407ABDF8001000043144897AF0
:1031700040EA0120BDF800103144C97A0843C11764
:10318000FDF7C6FEBDF80C10444601EB410202EB10
:10319000011208EB0211C1F8100ABDF8000030441A
:1031A000007B0021FDF7B4FEBDF80C1001EB4102DD
:1031B00002EB011204EB021181F8140ABDF80000C1
:1031C0003044407B0021FDF7A3FEBDF80C1001EB5D
:1031D000410202EB011204EB021181F8150ABDF85D
:1031E00000003044807B0021FDF792FEBDF80C10FA
:1031F00001EB410202EB011204EB021181F8160A05
:10320000BDF800003044C07B0021FDF781FEBDF811
:103210000C1001EB410202EB011204EB021181F8E8
:10322000170ABDF800003044007C0021FDF770FE55
:10323000BDF80C1001EB410202EB011204EB02118C
:10324000C1F8180ABDF80000304400E035E2407CC7
:103250000021FDF75DFEBDF80C1001EB410202EB11
:10326000011204EB021181F81C0ABDF80C0000EBFE
:10327000400101EB001104EB011090F8160A06283A
:10328000484655D09CE0BDF80000BDF80410084445
:103290003044807C0021FDF73BFEBDF804204FF058
:1032A0000309B2FBF9F2BDF80C1001EB410303EB8B
:1032B000011304EB031101EB021181F8400A00E055
:1032C00086E3BDF80000BDF8041008443044C07C1B
:1032D0000021FDF71DFEBDF80420BDF80C10B2FB67
:1032E000F9F201EB410303EB011304EB031101EBD2
:1032F000021181F8410ABDF80000BDF8041008442D
:103300003044007D0021FDF703FEBDF80420BDF828
:103310000C10B2FBF9F201EB410303EB011304EBD8
:10332000031101EB021181F8480ABDF80400C01C2A
:10333000ADF80400BDF80C0000EB400101EB0011FA
:1033400004EB011090F8170ABDF8041000EB4000E0
:10335000884298D845E0BDF80000BDF80410084444
:103360003044807C0021FDF7D3FDBDF80C1001EB4B
:10337000410202EB0111BDF8042004EB01115208D7
:1033800001EB021181F8400ABDF80000BDF80410FD
:1033900008443044C07C0021FDF7BAFDBDF80C1094
:1033A00001EB410202EB0111BDF8042004EB011115
:1033B000520801EB021181F8410ABDF80400801C9B
:1033C000ADF80400BDF80C0000EB400101EB00106B
:1033D00004EB001090F8170ABDF80410B1EB400F91
:1033E000B9D3BDF80C100220F6F706FCBDF80C00AE
:1033F000C0B200E0D8E2FEF75FFABDF80C00012190
:1034000000EB400204EB820080F83115B7E2BDF812
:1034100000003044007A444688F86D02BDF8000090
:103420003044407A88F86C02BDF800003044807A5D
:1034300088F86B02BDF800003044C07A88F86A0250
:1034400000E0A2E2BDF800003044007B84F869028D
:10345000BDF800003044407B84F8680204F51A741B
:10346000F6F7E6FAF6F7A2FA2078A4F51A74FF2820
:1034700029D1F6F753FABDF800003044007A84F8F9
:103480006D02BDF800003044407A84F86C02BDF84B
:1034900000003044807A84F86B02BDF800003044AC
:1034A000C07A84F86A02BDF800003044007B84F8DA
:1034B0006902BDF800003044407B84F86802F6F7EA
:1034C000B7FAF6F773FA606D18B10F2002E0F5E075
:1034D000FEE0102084F8250651E21020444688F8CA
:1034E0002506BDF800003044007A88F86D02BDF86A
:1034F00000003044407A88F86C02BDF80000304487
:10350000807A88F86B02BDF800003044C07A84F8F5
:103510006A02BDF800003044007B84F86902BDF8FF
:1035200000003044407B84F8680204F51A74F6F712
:103530007FFA01F0BDFEA060A068A0681FE20E2126
:1035400088F8251688F8619019E24946ADF80C9084
:10355000444638E0ADF8041014E0BDF80C0000EB70
:10356000400202EB0010BDF8042004EB001000EB59
:10357000021090F8420AC00712D1BDF80400401CA6
:10358000ADF80400BDF80C0000EB400202EB0010A7
:1035900004EB001090F8170ABDF804209042DCD824
:1035A000BDF80C0000EB400202EB001004EB001031
:1035B00090F8170ABDF80420904208D8BDF80C0016
:1035C000401CADF80C00BDF80C000428C2D3BDF8B7
:1035D0000C00042869D3FF4A89465170FE49012036
:1035E000C1F88802C1F8880294F86500E8B30D209C
:1035F00084F82506BDF800003044407ABDF800107C
:103600003144097A40EA0120ADF80800BDF8000015
:103610003044C07ABDF800103144897A40EA012074
:10362000508000204FF40073BDF800100144314475
:10363000097B04EB000C8CF86610401C80B29842A9
:10364000F2D3E448408800F2FF3081B20120F5F760
:10365000BFFC50B184F86190DE4841886422514338
:10366000BDF80820B1FBF2F100E01CE084F8601026
:103670000121A1714188491C41804088BDF8081092
:10368000884210D914F85C0F40F0010020702078B7
:1036900020F00600801C2070BDF80800608000212A
:1036A0000120F6F7A9FA484643E1102084F82506E0
:1036B00014F85C0F40F08000207060E1BDF800005D
:1036C0003044017A88F86110112188F8251656E1F6
:1036D0004946ADF80C90444638E0ADF8041014E0CB
:1036E000BDF80C0000EB400202EB0010BDF8042016
:1036F00004EB001000EB021090F8420AC00712D150
:10370000BDF80400401CADF80400BDF80C0000EB4F
:10371000400202EB001004EB001090F8170ABDF80D
:1037200004209042DCD8BDF80C0000EB400202EB14
:10373000001004EB001090F8170ABDF80420904226
:1037400008D8BDF80C00401CADF80C00BDF80C000A
:103750000428C2D3BDF80C0004287DD39D4B002063
:1037600058709D490120C1F88802C1F8880294F878
:103770006500E8B3122084F82506BDF80000304447
:10378000007A84F8610094F86100401EADF80C00E6
:103790000020BDF80010014431444A7ABDF80C10F5
:1037A00001EB410C0CEB011104EB0111014481F818
:1037B0001E2A401C80B20A28EBD3BDF8000030441A
:1037C000007DBDF800103144C97C40EA0120ADF80D
:1037D0000800BDF800003044807DBDF80010314481
:1037E000497D40EA0120588000204FF4007100E03C
:1037F00056E0BDF8002002443244D27D04EB000CB8
:103800008CF86620401C80B28842F0D358889946D4
:10381000BDF80C1000EB8120401E81B20320F5F7AB
:10382000D7FBE8B3B9F80210484664225143BDF80B
:103830000820B1FBF2F184F860100121A171B9F800
:103840000210491CA9F80210B9F80210BDF80820AE
:10385000914242D9002000E091E0BDF80C1001EB4C
:10386000410202EB011104EB011101EB001191F88F
:10387000492A42F0010281F8492A401C80B21028EE
:10388000E9D3BDF80C0000EB400101EB001004EBA4
:10389000001090F8281A41F0010180F8281A00E081
:1038A00046E0BDF80C0000EB400101EB001004EB1A
:1038B000001090F8281A21F00601891C80F8281AB7
:1038C000BDF80810BDF80C0000EB400202EB001040
:1038D00004EB0010A0F82A1A25E04088012827D11F
:1038E0000020BDF80C1001EB410202EB011104EBCA
:1038F000011101EB001191F8492A22F0010281F82F
:10390000492A401C80B21028EBD3BDF80C0000EB14
:10391000400101EB001004EB001090F8281A21F090
:10392000010180F8281ABDF80C100220F6F764F99E
:1039300000202949C1F88802C1F888021FE0D8F8A0
:10394000540044460A21B0FBF1F0BDF800103144A8
:10395000097A884213D1BDF800003044007A18B1CA
:10396000606D0A38606504E0C4F85490102084F853
:10397000250600210520F6F73FF90120A071B8F8CF
:10398000EA04424620B300201EE000200146BDF8B4
:1039900000200244B154401C80B20528F7D3A8F897
:1039A000EA1407B0BDE8F08F0020A4F8EA04F8E7B5
:1039B000BDF800102944014431448978BDF8003035
:1039C0000344F154401C80B2B2F8EA148142EFD8AB
:1039D000444603E0180A002000004242B8F8EA0416
:1039E00000287EF471ACDCE72DE9F74F002084B0AD
:1039F000FE4E019005468046009096F826054FF051
:103A0000000B012876D196F82106012872D108EB27
:103A1000480101EB0810002706EB001A56E00AEBFC
:103A2000071494F8420A00064ED594F8420A40F072
:103A3000040084F8420A94F8420A000744D594F836
:103A4000420A20F0080084F8420AC6F835B008EBB4
:103A5000C80101EB082006EBC00007EB471100EBA3
:103A60008109E24809F6F9611022253004F5246441
:103A7000F4F7EBFBD9F8F10EC6F81900D9F8F50EFA
:103A8000C6F81D0020783076D9F80C0FC6F8210052
:103A9000D648D0F86812C6F83910B0F86C02A6F80B
:103AA0003D006068C6F83F00706D81B20220F5F7F6
:103AB0008FFA00210620F6F79FF8706D401C7065A4
:103AC00000210520F6F798F87F1CBFB29AF8170A74
:103AD000B842A4D841460220F6F78EF808F101005A
:103AE0001FFA80F8B8F1040F91D386F821B60B20A5
:103AF00086F82506BE4F0020387000980DE001F0D2
:103B0000D7FBC6F87002D6F87002C0F300400190EF
:103B1000D6F87002C0F3420000900028EFD096F86B
:103B20002306B3493A31022816D1B24890F8322020
:103B30002AB1002180F8321001F090F969E00725E0
:103B400055200870FD204870AA2088700020C87099
:103B5000087161224A718871F520485500208B4612
:103B6000D6F87012C0F10302D200D1402B1803EB3B
:103B70000B02D170401C80B20428F1D396F82206C3
:103B800030B39D48D0F808123078B8B30020014314
:103B90003CD000205946321892F8A8252B180B4427
:103BA000DA71401C80B21428F5D30020321892F844
:103BB00034262B180B44DA76401C80B20A28F5D341
:103BC0000BEB0501069881F8250005F1260405E0B8
:103BD0000BEB05000699C17105F10804CCB18349CE
:103BE000069881F8E70406981021FF2311287DD05C
:103BF00013DCA0F10B00062822D200E004E0DFE88D
:103C000000F01F1FFF11F4200120C0E7012086F8FB
:103C10002605002007B0BDE8F08FA22810DA122890
:103C20000ED10FE2714880F82516744900205A46DB
:103C300026180B5C9355401C80B20A28F8D30A342E
:103C4000FDE26A4890F85C10C90704D0012080F3B7
:103C50001388FEF711F84FF0000977E100EB4001FF
:103C600001EB091002EB001696F8160A032814D08F
:103C700096F8160A012810D096F8160A02280CD0D9
:103C800096F8160A042808D096F8160A05287DD05A
:103C900096F8160A06287AD054E101200BF80400A1
:103CA000E41CA0B2022302900BF80030401C80B24A
:103CB0001D230BF80030401C84B20020A7E006EB67
:103CC000081292F8400A59460BF80400641CA0B28E
:103CD00092F8424A0BF80040401C84B292F8420A23
:103CE000400709D492F8420A000700E059E103D4E2
:103CF00092F8420A800777D500201F46D2F8443A4E
:103D0000C0F1030C4FEACC0C23FA0CF300EB040CCB
:103D100001F80C30401C80B20428EFD3241DA3B25C
:103D200009EBC90404EB092207EBC20408EB4812B3
:103D3000002004EB8207D7F8F12EC0F10304E40061
:103D4000E240C4180A55401C80B20428F3D31B1D5E
:103D50009AB20020D7F8F53EC0F10304E400E34036
:103D600084180B55401C80B20428F3D3121D92B264
:103D70000020D7F80C3FC0F10204E400E3408418AF
:103D80000B55401C80B20328F3D301E050E080E0E3
:103D9000D21C1FFA82FA0024D7F8F90ED7F8FD1EBC
:103DA000C4F10502D200F4F73EFA04EB0A020BF864
:103DB0000200641CA4B2062CEED30AF106001FFA1E
:103DC00080FA0024D7F8010FD7F8051FC4F10502C7
:103DD000D200F4F728FA04EB0A020BF80200641C84
:103DE000A4B2062CEED30CE00EE062E1D412002067
:103DF000180A0020D44200200000404248910108E7
:103E0000ACE00AF1060084B208F1010080B2FF4B79
:103E100096F8171A804641453FF651AF0298029A2C
:103E2000201A0BEB0201030A01F8023D487089E0F9
:103E300002205E460BF80400E41CA4B223460020D6
:103E400090461AE0421C3255641CA1B23C1894F80A
:103E500005447454491C8CB2002108EB001047182B
:103E600097F8117401EB040C06F80C70491C89B228
:103E70001029F4D31034A4B290B298F80414474631
:103E80008142DFD80BEB0300002100F8021DE11A8C
:103E900057E003200BF80400E41CA7B202200BF843
:103EA0000700781C80B20E210BF80010401C84B271
:103EB00000219646DA463AE006EB011292F8400AF3
:103EC0000AF80400641CA0B292F8424A0AF80040C2
:103ED000401C84B292F8420A000726D509EBC90CAF
:103EE0000CEB09220EEBC20201EB4113002002EBA6
:103EF0008302131893F8173F00EB0408D4460AF81E
:103F00000830401C80B20A28F3D30A34A3B2002040
:103F1000141894F8304F00EB03080CF80840401CCC
:103F200080B20228F4D39B1C9CB2491C89B296F83B
:103F3000170A8842C0D80AEB0700002100F8021DCA
:103F4000E11B417009F101001FFA80F9AF4A92F8B4
:103F50006C19484649453FF681AE70E17878401CBF
:103F600078707878052804D2A84890F85C20D207A9
:103F700007D0A64880F8251690F85C10C90704D031
:103F800005E00D2180F8251601E080F86030788882
:103F9000010A0BF8041079880BEB04004170A41C93
:103FA0004DE19A4F87F8251697F86100DC460BF82B
:103FB00004000022641C38E097F8610002EB42160E
:103FC00000EBC00101EB002007EBC00000EB860016
:103FD00090F80207012826D197F8610000EB400114
:103FE00001EB001007EB001000EB021090F8100935
:103FF0000CF80400641CA3B2002097F8611001EBD8
:10400000C10404EB012107EBC10101EB860101446E
:1040100091F803171C180CF80410401C80B20A28F1
:10402000EBD30A339CB2521C92B297F8610000EBBA
:10403000400101EB001007EB001090F8E7089042F8
:10404000BAD8FCE07878401C7870787805280CD2D3
:104050006E4A92F8610000EB400606EB001002EB9E
:10406000001090F8F808C0070FD0684A82F82516AB
:1040700092F8610000EB400101EB001002EB001030
:1040800090F8F808C00704D005E0122082F8250651
:1040900001E082F860305D4890F861100BF8041080
:1040A00079880BEB0400090A417079888170E41C5F
:1040B000C5E0DFF85881012188F80610D8F85410BF
:1040C0000A22B1FBF2F259460BF80420D8F854004A
:1040D000641C0A2801D90A2001E0D8F85400002203
:1040E0000292814608552220641C08551646DA467D
:1040F000641C9DE0D8F8540038B1D8F85400801BF7
:10410000401E81B20220F4F7F7FE98F818005146DD
:104110000AF80400641CA2B20020D8F81930C0F1DB
:104120000304E400E34084180B55401C80B20428CB
:10413000F3D3121D92B20020D8F81D30C0F1030451
:10414000E400E34084180B55401C80B20428F3D3EC
:10415000121D92B20020D8F82130C0F10204E40010
:10416000E34084180B55401C80B20328F3D3D21CC3
:1041700097B20024414651F8250F4968C4F1050261
:10418000D200F4F750F8E2190AF80200641CA4B255
:10419000062CEFD3BF1DBFB20024414651F82D0FAE
:1041A0004968C4F10502D200F4F73DF8E2190AF8B3
:1041B0000200641CA4B2062CEFD3BF1D98F83E3059
:1041C000B8B2414652460AF80030401C98F83D30DB
:1041D00080B20AF80030401C98F83C3080B20AF8EF
:1041E0000030401C98F83B3080B20AF80030401C88
:1041F00091F83A3080B21354401C91F8393080B2B3
:104200001354401C83B2002002E00000D4120020AE
:10421000D1F83F40C0F10307FF00FC40C718D45558
:10422000401C80B20428EFD31B1D761C9CB2B6B292
:1042300002990020B6EB09028841FFF65BAF661BCE
:104240000BEB0500320A8046427086700023D94687
:104250000AE0E91801EB0907F879DDE90021F5F733
:1042600047FCF8715B1C9BB29E42F2DC164D95F840
:10427000670228B1B1B2404600230422F6F77EFB64
:10428000B1B24E464046F5F717FA010A3155641CA3
:10429000A1B27054491C95F823068CB202280AD1A9
:1042A000601F010AF170307181B2701D01F047F991
:1042B0003055641CA4B2054804600121001FF5F7C5
:1042C00051FA2046A6E40000D4120020BC6402404B
:1042D00070B5164C40F224452946204603F053F8A9
:1042E000002821D02946204602F0EAFF104D002187
:1042F0002846F5F737FA61102846F5F71DFA0D49FB
:10430000012081F824062088A088281D0268C2F5B3
:10431000FA62A1F8EA244FF4FA6101602846BDE888
:1043200070400121F5F71EBA70BD00000010014079
:1043300088640240D412002010B5074C054920467D
:10434000F5F7FAF900212046F5F70CFA03490120A8
:10435000087010BD00800028B8640240180A0020D0
:104360002DE9F04301218FB0880500F0F7FEDFF85A
:1043700094904846F5F700FA402005010390002488
:10438000CDE90545C60207940894CDE909464FF0EA
:1043900000681E480B940C940D941B4FCDF80080C0
:1043A0000E94CDE9017069464846F5F78DFA012271
:1043B00010214846F5F772FADFF84890A9F1300964
:1043C0004846F5F7D9F94FF4FA60CDE90340CDE955
:1043D000054507940894CDE909460D480B940C94C3
:1043E0000D94CDF800800E94CDE9017069464846E1
:1043F000F5F76AFA01214846F5F7B4F90FB0BDE8C0
:10440000F0830000B864024004100140520A00200A
:10441000206000207CB50121032000F09FFE134D99
:10442000072206212846F5F7DBFF0722114628461A
:10443000F5F7D6FFC020022100908DF8051000246A
:104440008DF8064001208DF807008DF804106946AC
:104450002846F5F789FF072000908DF804408DF875
:10446000074069460248F5F77FFF7CBD0004024023
:104470000000024070B50024FFF7CCFFFFF770FF8B
:104480004FF4E13000F086F800F066F8012140209A
:1044900000F07CFE012000F0FDFE2D490B2081F88C
:1044A0002506002581F8145581F8165581F8155513
:1044B00081F817554FF47A70C1F81C0581F824551E
:1044C000012381F8263581F8253581F82735C2008A
:1044D000C1F82C2581F8FC5481F8FE3481F8FD34B4
:1044E00081F8FF34C1F8040581F8085581F80A35D0
:1044F00081F8093581F80B354210C1F81025154AAD
:10450000157095705370D37042F21076966042F633
:10451000F82604EB440201EB820282F8305582F85F
:10452000325582F8313582F83355C2F83865641C4B
:10453000042CEED391F8202622B191F82026521EA9
:1045400081F8222604F0D8FBBDE8704000F022B9C3
:10455000D41200200443002038B546208DF8000016
:1045600002208DF8010001248DF802408DF80340EF
:104570006846FDF745FB25208DF800008DF80140C9
:1045800000208DF802008DF803406846FDF738FBE7
:1045900038BD00001FB504460121102000F01AFEAE
:1045A0000020ADF804000094ADF80600ADF8080056
:1045B000ADF80C000C200D4CADF80A006946204601
:1045C00002F018FF0121204602F07DFE012240F298
:1045D0002441204602F0F6FE1021204602F070FE33
:1045E0000122C021204602F078FE1FBD00100140CC
:1045F0002DE9F04F8DB034225F496846F3F725FE70
:104600005E4D002695F8220600287CD0DFF870B1B8
:104610000121CBF888124FF0000985F82496594FF4
:10462000594C02E0B85DA055761C5648F3F72BFEB6
:10463000B042F7D8DFF85481C8F800600121A8F132
:104640000400F5F78FF84FF4FA7004F055FB85F885
:104650002496DFF830A100260AF1750A03E01AF863
:104660000600A055761C47487530F3F70CFEB042A3
:10467000F5D8C8F8006045480121001FF5F772F829
:104680004FF47A7004F038FB4E46A94685F824664C
:10469000DFF8F0A000250AF1020A03E01AF805008D
:1046A00060556D1C3748801CF3F7EDFDA842F5D826
:1046B000C246C8F8005035480121001FF5F752F8EE
:1046C0004FF47A7004F018FBB04689F8246600268F
:1046D00002E0B85DA055761C2A48F3F7D4FDB0423D
:1046E000F7D85546CAF80060DFF8A0A00121AAF16A
:1046F000040A5046F5F736F84FF47A7004F0FCFAE5
:104700002349684600E034E0F3F7B1FD1D496846EF
:10471000891DF3F7ACFD4F4689F824860026E9464B
:1047200003E019F80600A055761C6846F3F7ABFDC8
:10473000B042F6D82E6001215046F5F713F84FF439
:104740007A7004F0D9FA464687F824860D4900208D
:104750000A310A5C2254401C0728FAD3401E286004
:1047600001215046F4F7FEFF642004F0C5FACBF8AF
:1047700088620DB0BDE8F08FC0960108D412002009
:1047800000004242E4930108520A0020BC64024047
:10479000901800202DE9F04FDFF8F48389B0002451
:1047A00098F8220600287DD0FA480125C0F88852E2
:1047B00098F8231608F27650F74E0090022904D09C
:1047C000A34688F824B6F54FEDE000203055641C70
:1047D000642CFBD3814688F82406F04900209631EA
:1047E0000A5C3254401C0828FAD3002708F2E4542B
:1047F00006E008EB070090F8E405F11908727F1C49
:104800002046F3F740FDB842F3D82C20F119087286
:10481000002408F20C6B093706E008EB040090F85E
:104820000C0639197054641C5846F3F72CFDA0424D
:10483000F3D8DBA1D848F3F71AFDD748F3F723FDE7
:10484000DFF860B3CBF800000121ABF10400F4F70E
:1048500089FF4FF47A7A474605E0012004F04CFACC
:10486000641C54457ED897F824060028F5D0CE481D
:10487000D0F81802C949B331C8B100204A463254B1
:10488000401C6428FBD3B84687F824260024085D22
:104890003055641C0E2CFAD30098F3F7F4FC000496
:1048A000000C00E073E032D00024414629E0B84615
:1048B00087F82496002404E0B848B330005D3055F2
:1048C000641CB648B330F3F7DEFCA042F4D8CBF852
:1048D0000040B4480121001FF4F744FF464605E0BC
:1048E000012004F009FA641C5445BBD896F824064C
:1048F0000028F5D015E00A1992F8762533199A7335
:10490000641C8442F7D3A6A1A348F3F7B0FCA248E5
:10491000F3F7B9FCCBF80000A2480121001FF4F71F
:1049200021FF564697F8240690B3A048A0494C466C
:10493000006808609D48001D006848609B4808307A
:104940000068886000203A1882F8A845401C1428A6
:10495000F9D3087A04AECD7A8B7A4A7A86E82D00AC
:10496000CD7900E012E108798B794A798DE82D0044
:104970008B780A788FA19A4802F0A4FD00210320C9
:10498000F5F73AF9002802D08248C0F888424BE295
:10499000FFE7012004F0B0F9641CB442C2D93BE245
:1049A000385D3055641C7D48F3F76DFCA042F7D8A4
:1049B0007C4804600121001FF4F7D4FE4FF4FA7024
:1049C00004F09AF95846DA46C34688F82406DFF818
:1049D000CC81002408F1750803E018F80400305574
:1049E000641C6E487530F3F74EFCA042F5D86D4854
:1049F00004600121001FF4F7B5FE4FF47A7004F053
:104A00007BF9D046D9468BF824A6DFF890A1002484
:104A10000AF1020A03E01AF804003055641C5F48EA
:104A2000801CF3F730FCA042F5D8DFF878A1CAF873
:104A300000400121AAF10400F4F794FE4FF47A70CB
:104A400004F05AF989F82486002402E0385D3055D4
:104A5000641C5248F3F717FCA042F7D85746CAF82F
:104A6000004050480121001FF4F77CFE4FF47A709B
:104A700004F042F9C24689F82486DFF82081002438
:104A800008F16A0803E018F804003055641C434834
:104A90006A30F3F7F8FBA042F5D8BB463C604148CA
:104AA0000121001FF4F75EFE4FF4FA784F4605E04F
:104AB000012004F021F9641C444567D897F82406C6
:104AC0000028F5D0D14687F824A6DFF8D0A000242E
:104AD0000AF1390A03E01AF804003055641C2F4823
:104AE0003930F3F7D0FBA042F5D8DA46CBF80040D6
:104AF0002C480121001FF4F735FE05E0012004F0E9
:104B0000FBF8641C4445D8D897F824060028F5D053
:104B100087F824962448D0F818022049113168B14A
:104B200000200A5C3254401C0D28FAD30098F3F799
:104B3000AAFB0104090C1BD0002013E000248B46C3
:104B400003E01BF804003055641C14481130F3F7DF
:104B50009AFBA042F5D80FE03A1892F87625331860
:104B60005A73401C8842F7D30DA10B48F3F77FFB23
:104B70000948F3F788FB0446CAF8004009480121B8
:104B8000001FF4F7EFFD4FF47A7B31E0BDE0000049
:104B9000D412002000004242520A0020E49301088F
:104BA0000D0A0000BC64024000004342107AFF1F5F
:104BB000F067002025303278253032782530327881
:104BC00025303278253032782530327825303278E9
:104BD00025303278253032782530327825000000B3
:104BE0007C1800200A2004F087F8641C5C458AD8F1
:104BF00097F824060028F5D087F824960024DFF8DB
:104C000038B203E01BF804003055641C8A48F3F7FF
:104C10003AFBA042F6D8CAF8004001218748F4F7D1
:104C2000A1FD05E0012004F067F8641C4445DED8CE
:104C300097F824060028F5D087F82496DFF8F8B115
:104C400000240BF1110B03E01BF804003055641C29
:104C500079481130F3F717FBA042F5D8D346CAF8CC
:104C6000004001217548F4F77DFDC24605E00120B2
:104C700004F042F8641C544547D897F824060028ED
:104C8000F5D0C84687F824966B4800243730015D7C
:104C90003155641C0C2CFAD3601ECBF800000121A6
:104CA0006648F4F75FFD05E0012004F025F8641C78
:104CB00054452AD897F824060028F5D060A1624808
:104CC00004F0BAF9D8B1604A002143181344914660
:104CD0005B797C1884F86135491C1429F5D397F861
:104CE000BD0568B359495A48F3F7C1FA52495848C3
:104CF0004239F3F7BCFA87F8248600240AE0012041
:104D000003F0FAFF641C5445D8D985E05048005D93
:104D10003055641C4E48F3F7B6FAA042F6D8CBF8EB
:104D2000004001214548F4F71DFD05E0012003F096
:104D3000E3FF641C54456FD897F824060028F5D08B
:104D4000642003F0D9FF002087F8240604463A487F
:104D50004330B046025D3255641C0B2CF9D3601E03
:104D6000CBF8000001213548F4F7FCFC05E00120F8
:104D700003F0C2FF641C54454ED897F8240600285F
:104D8000F5D034A1304804F057F9061E37D064201E
:104D900003F0B2FF00200446391881F8A845401CF2
:104DA0001428F9D30020494632180A4452783B1897
:104DB00083F8AD25401C0F28F6D300210320F4F71B
:104DC0001BFF10B12448C0F88842642003F094FF10
:104DD00087F824461849002440463E390A5D0255AA
:104DE000641C072CFAD3611ECBF800100121134874
:104DF000F4F7B8FC642003F07FFF564610E0012072
:104E000003F07AFF641C5445BBD905E0012003F090
:104E100073FF641CB44203D985F31388FCF72CFF9D
:104E200097F824060028F1D00B490020C1F8880229
:104E300009B0BDE8F08F00002C940108B86402406E
:104E400049434349443A0000206000209018002064
:104E5000200A0020493A0000000042422DE9F047B4
:104E60000020574E01463154401C6428FBD3554D59
:104E7000884685F82416544900200A5C3254401CA8
:104E80000828FAD3002705F2E45405E0E81990F861
:104E9000E405F11908727F1C2046F3F7F4F9B842D3
:104EA000F4D82C20F1190872002405F20C69093796
:104EB00005E0281990F80C0639197054641C48460E
:104EC000F3F7E1F9A042F4D840A13D48F3F7CFF958
:104ED0003B48F3F7D8F93E4F3860A7F1040A0121A7
:104EE0005046F4F73FFC05E0012003F005FF641C89
:104EF000642C03D895F824060028F5D03548D0F85E
:104F0000180231491D31B8B1002042463254401CCC
:104F10006428FBD3A84685F824260024085D305574
:104F2000641C0E2CFAD32C48F3F7ADF90004000CE6
:104F300031D00024414628E04046A84685F82406A2
:104F40000024894603E019F804003055641C1E480B
:104F50001D30F3F798F9A042F5D83C600121504686
:104F6000F4F700FC464605E0012003F0C5FE641C92
:104F7000642C1FD896F824060028F5D01AE00A19E8
:104F800092F8762533199A73641C8442F7D30FA1E3
:104F90000B48F3F76CF90A48F3F775F9386001210B
:104FA0005046F4F7DFFB05E0012003F0A5FE641C8A
:104FB000642C03D895F824060028F5D0BDE8F087C6
:104FC000520A0020D41200207A9401080D0A000031
:104FD000BC640240000043424A1800202DE9FC5FF7
:104FE0000121592000F0BAF800248DF80440022075
:104FF000DFF894B04FF47C578DF8070000976946AE
:105000005846F5F7B1F9FC20DFF8809000908DF854
:10501000044001258DF8075069464846F5F7A4F984
:10502000DFF86CA04FF440468DF8044000968DF8F0
:10503000075069465046F5F797F90720DFF8548086
:1050400000908DF804408DF8075069464046F5F70A
:105050008BF907214046F5F7DCF931465046F5F764
:10506000D8F939465846F5F7D4F9FC214846F5F702
:10507000D0F90948D0F828120848012902D0047054
:10508000BDE8FC9F0570FBE70010024000180240DD
:10509000000C02400000024000004242D4120020F6
:1050A00010B5FFF79BFF642003F026FE1048D0F8F0
:1050B0003C12104819B1002180F8221610BD0E498B
:1050C000D1F8182292B1012280F82226D1F80822C4
:1050D000D1F80C1242EA4101C94380F8231690F836
:1050E000231601F0030180F8231610BD0222EBE71E
:1050F00000804142D4120020000043427CB50121CF
:10510000102000F02BF84CF20400012400908DF8E0
:10511000044000208DF8060003208DF80500084D9E
:105120008DF8074069462846F5F71EF90421284600
:10513000F5F76DF90348C0F8B842C0F8BC427CBD31
:105140000010024000004242FFF7D8BF4FF4006158
:105150000148F5F755B9000000040240044A00294F
:10516000116801D0014300E08143116070470000E5
:1051700030380240044A0029116801D0014300E0A0
:10518000814311607047000010380240044A002932
:10519000116801D0014300E08143116070470000B5
:1051A00034380240044A0029116801D0014300E06C
:1051B000814311607047000040380240044A0029D2
:1051C000116801D0014300E0814311607047000085
:1051D00020380240044A0029116801D0014300E050
:1051E000814311607047000044380240044A00299E
:1051F000116801D0014300E0814311607047000055
:105200002438024070B5204B1968204C11F00C0175
:1052100004D06610042903D0082903D004601BE0E1
:10522000066019E0184A121F1168C1F38055116811
:1052300001F03F0115B1B6FBF1F101E0B4FBF1F172
:1052400014681268C4F388146143C2F30142521C0B
:105250005200B1FBF2F1016019680F2202EA11114C
:105260000B4A545C0168E14041601C68072505EA6F
:105270009424145D21FA04F484601B6805EA533316
:10528000D25CD140C16070BD083802400024F400F7
:105290000000002005490028086802D040F0040002
:1052A00001E020F00400086070470000000806508C
:1052B00001480068704700000808065070B50120DA
:1052C00080F310880C4D10212846F5F7A0F808212E
:1052D0002846F5F79EF8D720F3F732FFFF20F3F7C3
:1052E0002FFF044610212846F5F793F8002181F39B
:1052F0001088204670BD00000000024070B50120FB
:1053000080F31088194C0020A080FFF7D7FF00061B
:1053100009D4012003F0F0FCA088401C80B2A080DA
:10532000C828F2D31EE0A088C8281BD2104D102137
:105330002846F5F76CF808212846F5F76AF89F200B
:10534000F3F7FEFEFF20F3F7FBFEFF20F3F7F8FE76
:10535000607010212846F5F75CF8002080F3108873
:10536000607870BD002080F3108870BD221200208C
:105370000000024070B5012188B08803FFF712FFDA
:1053800001210220FFF7EAFE00244FF400602F4EB7
:105390008DF8044000908DF8074069463046F4F7D8
:1053A000E3FF01218DF8041002258DF80550080354
:1053B0008DF806408DF80710009069463046F4F7E6
:1053C000D3FF05220D213046F5F70AF805220E21FC
:1053D0003046F5F705F805220F213046F5F700F8BD
:1053E0004FF4604000908DF8045003208DF80500C4
:1053F0008DF806408DF8074069463046F4F7B4FF53
:10540000134D284600F04AF8ADF810406815ADF885
:1054100012001820ADF814000720ADF81800ADF800
:1054200008404FF48270ADF80C40ADF80A00ADF8BA
:105430000E40ADF8164002A9284600F064F801219C
:10544000284600F021F808B070BD000000040240BA
:105450000038004070B50B4C05460221204600F094
:1054600047F80028F9D02946204600F04AF80121E3
:10547000204600F03DF80028F9D0204600F03FF823
:10548000C0B270BD003800400029018802D041F050
:10549000400101E021F0400101807047114910B541
:1054A00088420AD1841401212046FFF79FFE20463E
:1054B000BDE810400021FFF799BE0B49884202D198
:1054C0000121041404E0094988420AD10121C413CE
:1054D0002046FFF773FE2046BDE810400021FFF78D
:1054E0006DBE10BD0030014000380040003C00405F
:1054F0000246002012890A4200D0012070478089AC
:1055000070478181704730B502884C8802F441535E
:105510000A88CD8822438C882C4322430C8922435D
:105520004C8922438C892243CC8922431A4302802E
:10553000828B22F400628283098A018230BD024696
:10554000002003E012F8013B1844C0B2491E89B2A2
:10555000F8D2704770B501218D070024284601F06C
:105560008BFBE8B3F5F7FAF90020264B3BE003EBA1
:105570008401D1F840261278012AD1F8402603D0C0
:105580005278012A08D02AE01070D1F840265070D5
:10559000D1F84026907030E0D1F840269278F2B9E8
:1055A000D1F840265668761C5660D1F840265268DD
:1055B000D1F84066B668B24211D3D1F840660122F4
:1055C000B270D1F84026D278012A16D0D1F8402600
:1055D0005070D1F840265060D1F84016C87000E0F5
:1055E00005E0641CE4B293F83E16A142BFD82846F9
:1055F000BDE87040012101F089BAD1F84016486039
:10560000EDE70000D41200200CB5002225490092DD
:105610000192086840F4803008604FF4A063086885
:1056200000F4003001900098401C0090019810B9DF
:1056300000989842F3D10868800330D5012001908A
:1056400018484030026842F08052026016480268F2
:1056500042F4804202601348083002680260026827
:10566000026002680260031F104A1A600A6842F072
:1056700080720A600A689201FCD50D4A40F2056109
:105680001160016821F003010160016841F002012D
:1056900001600168C1F381010229FAD10CBD0192B8
:1056A0000CBD000000380240007000400854400764
:1056B000003C02407CB500229FED170A00928DED60
:1056C000010A6D4601AC16E0835CA3F13006102E92
:1056D00005D2009B1B010093865C303E07E0413BF6
:1056E000062B0CD2009B1B010093865C373E1E43A9
:1056F000521CD2B200968A42E6D3002006E0BFEEEA
:10570000000A7CBD2A5C2254401CC0B2B0EB510F91
:10571000F8D39DED010A7CBD0000000030B50546C0
:105720000022104611E0AB5CA3F13004102C02D231
:1057300044EA001007E0A3F14104062C08D204015A
:10574000A3F137002043521CD2B28A42EBD330BDC2
:105750004FF0FF3030BD00002DE9FC414E4D4FF0C1
:10576000380895F86A02002105F51A75FBF7D0FB99
:1057700001240826CDE90064024618200023414692
:10578000FCF79EFC071D07EB47004006000E0823B0
:105790002D2241460094FCF725FC687800217F1CEF
:1057A000FBF7B6FB024607EB4700CDE90064400675
:1057B000000E00234146FCF783FC074407EB47003B
:1057C0004006000E08232D2241460094FCF70AFCF7
:1057D000287800217F1CFBF79BFB024607EB470064
:1057E000CDE900644006000E00234146FCF768FC4A
:1057F000074407EB47004006000E082320224146DD
:105800000094FCF7EFFB687900217F1CFBF780FB1D
:10581000024607EB4700CDE900644006000E002376
:105820004146FCF74DFC074407EB47004006000EDD
:1058300008232D2241460094FCF7D4FB287900214F
:105840007F1CFBF765FB024607EB4700CDE90064D0
:105850004006000E00234146FCF732FC074407EBEC
:1058600047004006000E08232D2241460094FCF715
:10587000B9FBE87800217F1CFBF74AFB024607EBE7
:105880004700CDE900644006000E00234146FCF7C6
:1058900017FCBDE8FC810000D41200200249C8704A
:1058A0000120887170470000D41200202DE9FC5FB0
:1058B00000252C46F4F7BCFBF94FB87900287DD0C1
:1058C000A94687F80690FCF7E7F9F8780223DFF895
:1058D000D4B301264FF008084FF0100A0F286ED2FB
:1058E000DFE810F00F008300EC007A01BE01E50252
:1058F00038045C05A505F405870649079207C60725
:105900001908F5F71BF801280AD0022808D0042846
:1059100006D0082804D10220FFF7C0FF87F8609066
:10592000CDE900A600211523DFA20846FCF765FC9F
:1059300097F8610010B3CDE9008644460523DFA245
:1059400014210020FCF759FCCDE9004697F86120AE
:10595000002314211E20FCF7B3FBCDE9004697F885
:1059600061000A2300EB400101EB001007EB00127D
:105970001421282002F6EE02FCF73FFC97F86000A5
:10598000FF2825D017F8600FCDE900060A2364220E
:105990001E211846FCF7A4FACDE900863A780023C8
:1059A0002D213220FCF78CFB00EB4001322000EB74
:1059B000410008232522C0B22D2101E0D3E30FE3EB
:1059C0000096FCF70FFB17F86009642807D007E37F
:1059D000CDE9008615232D21BAA2142044E287F8D0
:1059E00060900220FFF75AFFF1E7F4F7A7FF0128C4
:1059F0000BD0022809D0042802D0082805D101E0E4
:105A0000082000E00320FFF749FF97F8210638B18E
:105A100097F8220638B1012808D0022811D108E0F1
:105A20001523ACA207E01523ADA204E01523B0A214
:105A300001E01523B1A2CDE9008600210846FCF75C
:105A4000DCFBB878012802D002280CD101E0AF4875
:105A500001E0AE481230CDE9000609231A460A21BA
:105A60000020FCF77DFBA94818234838CDE9000643
:105A70001A4600216820FCF773FBCDE900864446F6
:105A80001523A3A21A210020FCF7B7FBCDE900469D
:105A90001523A5A224210020FCF7AFFBCDE9004689
:105AA0007A6D002324215420FCF70AFB786D10B98D
:105AB0000220FFF7F3FEFFF74FFE88E7F4F73EFF03
:105AC000012806D0022804D0042809D0082818D1BB
:105AD0000EE097F85C0020F0800087F85C0010E092
:105AE00097F85C0020F0800087F85C00082006E052
:105AF00097F85C0020F0800087F85C000320FFF737
:105B0000CDFE97F8210638B197F8220668B1012832
:105B10000ED0022814D118E0CDE90086002115230B
:105B200085A20846FCF769FB15E015236CA201E08D
:105B300015236FA2CDE9008600210846FCF75DFB26
:105B400097F8E7040F2803D005E015236BA2F1E7CF
:105B50000120FFF7A3FEB878012802D002280CD15B
:105B600001E06A4801E069481230CDE900060923E6
:105B70001A460A210020FCF7F3FA97F8600010B1EA
:105B80000020FFF78BFE614818234838CDE9000656
:105B90001A4600216820FCF7E3FACDE900A6544636
:105BA000102367A214212820FCF727FBCDE90086EB
:105BB000152365A224211220FCF71FFB97F85C0037
:105BC00000067FF578AFCDE90046102363A22E21B1
:105BD0000020FCF712FB6EE7F4F7B0FE012806D0B8
:105BE000022809D004280ED008281ED121E03879D7
:105BF000D8B13879401E04E03879032815D23879B5
:105C0000401C387111E0387930B1012806D00228E3
:105C100006D0032809D105E0042004E0052002E0B5
:105C2000062000E00720FFF739FEF878032805D0AA
:105C3000CDE60220FFF732FE4846E2E73348042271
:105C40000021243000F000FFCDE900A938792F4968
:105C5000243101EB001238790007010E1023F1E323
:105C6000F4F76CFE082802D10320FFF717FEF8783E
:105C70000428DDD1254804220021643000F0E4FE30
:105C800097F8220620B1012875D0022872D198E039
:105C90001023CDE9008612A21946002083E06AE0B5
:105CA000D4120020000042424669726D776172652D
:105CB000446F776E6C6F616400000000506F727407
:105CC0003A000000446F776E6C6F61642046616932
:105CD0006C2100004E6F205369676E616C000000FC
:105CE000547970653A53746174696F6E00000000F6
:105CF000547970653A436C6F75640000547970652F
:105D00003A436C6F75642D546573740048B3010891
:105D10004F66666C696E65205265636F72642055CC
:105D2000706C6F61640000005265636F7264206E76
:105D3000756D6265723A00004F66666C696E65004B
:105D4000424C5545534B5900454E455247592054F6
:105D50004543484E4F4C4F475900000055706772FD
:105D60006164652045525220436865636B20477526
:105D70006E00000019E044461023AFF28C02CDE91A
:105D8000008619460020FCF738FACDE900461023BA
:105D9000F5A238210020FCF730FACDE900461123A6
:105DA000F34A38211E20FCF728FA97F8230600B39F
:105DB00097F8230601281CD097F82306022854D010
:105DC00005E6CDE9008610234446EAA219460020E4
:105DD000FCF713FACDE900461023E3A23821002096
:105DE000FCF70BFACDE9004611233821E54A1E20C5
:105DF000D9E7781990F8610518B96D1CADB2152D69
:105E0000F7D3CDE9008644461023DFA21A210020F3
:105E1000FCF7F3F9CDE900467A1910231A21202066
:105E200002F26152FCF7E9F9CDE900461023D8A24D
:105E300024210020FCF7E1F9CD4ACDE900462421D8
:105E4000102339320846FCF7D8F9CDE90046102373
:105E5000D1A22E210020FCF7D0F9C54ACDE9004699
:105E60000F232A322E2124202FE3CDE90086444639
:105E70001023CBA21A210020FCF7BFF9BC4ACDE9C0
:105E80000046102361321A211E20FCF7B6F9CDE935
:105E900000461023C0A224210020FCF7AEF9B44A2A
:105EA000CDE90046142325322E2100200DE3F4F71E
:105EB00045FD012804D0022807D008280FD10BE0A7
:105EC000387960B13879401E04E03879032806D269
:105ED0003879401C387102E00320FFF7DFFCF878C6
:105EE00005287DD104220021AF4800F0ADFDCDE9A9
:105EF00000A63A79BA46012300213E20521CFCF745
:105F0000DFF8CDE9008647461023A8A200214820EB
:105F1000FCF773F9DFF890820823A8F1F408CDE9C3
:105F200000861A4600217820FCF71AF9CDE90076A0
:105F30001023A1A208214820FCF75FF908231A4684
:105F400019467820CDE90089FCF70AF9CDE90076F9
:105F500010239CA219460020FCF74FF99AF8040080
:105F600000EB400101EB00110AEB011090F81D0A53
:105F70004FF01003012840D094A2CDE90076102103
:105F80001E20FCF73AF9CDE90076B046102391A225
:105F900018210020FCF731F99AF8040000EB4001C9
:105FA00001EB00100AEB001090F8160ACDE900781A
:105FB00005289AF8040000EB400101EB00100AEB01
:105FC00000101CD090F8160A7749403101EB0012FE
:105FD0000C2318213620FCF710F9C346B84600E020
:105FE00024E2CDE9007B10237DA220210020FCF7D4
:105FF00004F909274FF0200A9EE07CA2BDE790F843
:106000001C0A6949B031E1E707EB47014FF07A0913
:10601000B9EB410F02D2641CA4B20027307900EB27
:10602000400101EB001006EB001000EB051090F8AA
:10603000420AC009CDE90080307900EB400101EB54
:10604000001006EB001000EB051090F8402A0AEB58
:10605000C400C1B207EB47004006000E0023FCF766
:106060002FF8384487B207EB4701B9EB410F02D252
:10607000641CA4B20027307900EB400101EB001052
:1060800006EB001000EB051090F8420A0823C00947
:1060900000900AEBC400C1B207EB47004006000EB7
:1060A0002D22FBF79FFF7F1CBFB207EB4701B9EB27
:1060B000410F02D2641CA4B20027307900EB4001EA
:1060C00001EB001006EB001000EB051090F8420AFF
:1060D000C009CDE90080307900EB400101EB0010F0
:1060E00006EB001000EB051090F8412A0AEBC40003
:1060F000C1B207EB470040065646000E0023FBF7EF
:10610000DFFF384487B207EB4701B9EB410F02D2FA
:10611000641CA4B2002706EBC400C1B207EB470021
:106120004006000E08233B22CDF800B0FBF75AFFD3
:106130007F1C6D1CBFB2ADB22E4E307900EB40011A
:1061400001EB001006EB001090F8170AA8423FF68A
:106150005BAF6BE1F4F7F2FB01284DD0022850D081
:10616000082858D154E0F1E355524C3A00000000A1
:1061700057180020547970653A436C6F75642D543C
:1061800061737400029401084943434944000000CC
:1061900041504E203A000000494D45493A00000068
:1061A000535349443A000000ECB301084F6E4C6968
:1061B0006E65203A200000004F66664C696E653AB5
:1061C00020000000547970653A00000052533438C2
:1061D0003500000050726F746F636F6C3A000000FE
:1061E00047756E2D416464723A0000004C4F524175
:1061F00000000000D4120020387940B13879401EE8
:1062000004E03879032806D23879401C387102E05E
:106210000320FFF743FBF87806289AD10126BE71C8
:1062200004220021F94800F00FFCCDE900A63A79DC
:10623000012300214020521CFBF742FFCDE90086DC
:10624000C3461023F2A214210020FBF7D6FF092633
:1062500096E006EB46024FF07A09B9EB420F02D204
:10626000641CA4B200264FF0010ACDE900BA0879F7
:10627000884600EB400202EB001001EB001000EB3F
:10628000051090F8402A142707EBC400C1B206EBB2
:1062900046004006000E0023FBF712FF304486B292
:1062A00006EB4601B9EB410F02D2641CA4B20026F2
:1062B00007EBC400C1B206EB46004006000E0823FF
:1062C0002D22CDF800A0FBF78DFE761CB6B206EBB2
:1062D0004601B9EB410F02D2641CA4B20026CDE9FD
:1062E00000BA98F8040005EB451100EBC00202EB80
:1062F000002008EBC00000EB810090F8140F64212F
:1063000010FB01F0020A07EBC400C1B206EB460025
:106310004006B846000E0023FBF7D2FE304486B29A
:1063200006EB4601B9EB410F02D2641CA4B2002671
:1063300008EBC400C1B206EB460040065746000E0B
:1063400008232522CDF800A0FBF74CFE761CB6B240
:1063500006EB4601B9EB410F02D2641CA4B2002641
:1063600008EBC400C1B206EB46004006000E08234D
:106370003B220097FBF736FE761C6D1CB6B2ADB221
:10638000A649087900EB400202EB001001EB001077
:1063900090F8170AA8423FF65CAFE4E2F4F7CEFAB1
:1063A000082802D10320FFF779FAF8783C4607283D
:1063B000F3D1964804220021403000F045FBCDE99E
:1063C000008647461023964A14210020FBF715FF4C
:1063D000A14605EB450000EB051109EB01108046D5
:1063E00090F8280AC0071DD005EB8501142000EBAA
:1063F0004104CDE90076E1B205238AA20020FBF733
:10640000FCFECDE90076E1B201236A1C1E20FBF7F9
:1064100057FECDE9007608F61E22E1B20A232A20B3
:10642000FBF7EBFE6D1CADB2042DD2D39BE2F4F76B
:1064300085FA012807D002280CD0042812D0082899
:106440002AD12DE040E0387910B13879401E1EE0A5
:1064500005201CE03879052802D23879401C16E066
:10646000484614E03879062816D2DFE800F0030524
:1064700007090B1209200DE00A200BE00B2009E0B0
:106480000C2007E00D20FFF709FA97F82006387175
:1064900002E00E20FFF702FAF878082804D062E242
:1064A0000220FFF7FBF9DBE73879584C04228034EF
:1064B00004EB0010002100F0C7FACDE900A93879FB
:1064C000102304EB00120021002021E2F4F736FA39
:1064D000012806D0022809D004280ED0082849D166
:1064E00045E0387978B33879401E04E038790328DC
:1064F00040D23879401C38713CE0387900EB4001DB
:1065000001EB001007EB001090F81D0A01280AD0DB
:10651000387900EB400101EB001007EB001090F818
:106520001D0A88B126E038794C4600EB400101EBAA
:10653000001007EB001080F81D9A39790220F3F75C
:106540005BFBCBF8884215E0387900EB400101EBAA
:10655000001007EB001080F81D6A3879FBF7ACF9E2
:10656000CBF8886239790220F3F746FB02E0082075
:10657000FFF794F9F878092891D1042200212B48DB
:1065800000F062FACDE900864446152328A21421C2
:106590002820FBF732FECDE900463A790123142189
:1065A0004620521CFBF78CFD387900EB400101EBD3
:1065B000001007EB001090F81D0A01280AD0387966
:1065C00000EB400101EB001007EB001090F81D0AF2
:1065D00018B10AE0152318A201E0152319A2CDE98C
:1065E00000461E210020FBF708FE152318A23221C9
:1065F00006E1F4F7A3F91B4C012835D002283ED060
:10660000042849D008285BD14BE00000CCB4010835
:1066100047756E2D525353493A000000D4120020A2
:1066200048910108506F72742D000000DCB501081C
:10663000504F52543A000000545950453A4C4F5272
:1066400041000000545950453A5253343835000047
:106650005061737320456E746572204368616E6784
:1066600065000000D4420020387948B394F849000E
:1066700010B13879FBF720F93879401E0AE03879F3
:1066800003281DD294F8490010B13879FBF714F9AA
:106690003879401C387113E084F8496084F83D6013
:1066A0000EE00820FFF7FAF884F83C6094F84900FF
:1066B00030B1CBF8889284F849903879FBF7FCF830
:1066C000F8780A282FD104220021AA4800F0BCF94A
:1066D00045461523AFF2A802CDE9008612212820F5
:1066E000FBF78BFDCDE900563A79012312214620B4
:1066F000521CFBF7E5FCCDE9005615239EA21C2198
:106700000020FBF77AFDCDE900561523A0A2262133
:106710000020FBF772FDCDE900561523A2A230211F
:106720000020FBF76AFD94F8490001284FD1BE71A3
:1067300094F83E0078B1CBF8889284F83E9038798E
:106740000121FBF787F9CDE9008615239BA23821AB
:106750000020FBF752FD94F84800C0B384F848903D
:10676000CDE90086152399A238210020FBF745FDCD
:10677000CBF88862F7E0F4F7E1F8012813D002289B
:1067800011D0042802D008280DD109E0F2F754FEF8
:10679000142802D087F8679205E087F8676202E064
:1067A0000820FFF77BF8F8780B2810D171480422F5
:1067B0000021403000F048F9CDE900864446152319
:1067C00086A21A210020FBF718FD152300E0A1E0A6
:1067D000CDE9004686A224210020FBF70EFDCDE97D
:1067E0000046152386A22E210020FBF706FD97F810
:1067F00067024FF0150308B187A200E08CA2382190
:10680000CDE90046002083E0F4F798F8012806D08F
:1068100002280BD0042812D0082821D11DE0387995
:1068200010B13879401E08E03B7119E0387903282F
:1068300002D23879401C00E04846387110E03879BF
:1068400087F8200600210320F3F7D6F940B1022093
:10685000FFF724F8FDF70EFE02E00820FFF71EF810
:10686000F8780C287FD1434804220021803032E0A0
:10687000F4F764F8012806D002280BD0042812D0BF
:10688000082821D11DE0387910B13879401E08E080
:106890003B7119E03879032802D23879401C00E0B6
:1068A0004846387110E0387987F820060021032027
:1068B000F3F7A2F940B10220FEF7F0FFFDF7DAFD91
:1068C00002E00820FEF7EAFFF8780D284BD12948AE
:1068D00004220021C03000F0B7F8CDE900A697F8F7
:1068E00020065446554D102305EB00121946002092
:1068F000FBF783FC97F820063979884233D0CDE93D
:10690000004638790C2305EB001220210020121DCF
:10691000FBF773FC27E0F4F711F801281AD00228DE
:1069200018D0042802D0082814D110E0F3F7BAF9DF
:1069300086F31388BFF34F8F41490868414A00F43A
:10694000E06010430860BFF34F8FFEE70FE00820C0
:10695000FEF7A4FFF8780E2805D13848042200215C
:10696000403000F071F8BDE8FC5FFBF7FFBABDE80E
:10697000FC9F00001CB60108313A4469702073770F
:10698000697463682031616E6432204F4E000000EC
:10699000323A496E7365727420736C617665206D4E
:1069A0006F64756C65000000333A50617373204565
:1069B0006E74657220537461727400005374617454
:1069C000653A53656E64696E6700000053746174C4
:1069D000653A436F6D706C6574650000496E736550
:1069E000727420552D4469736B204669727374006C
:1069F0005468616E205061737320456E7465720037
:106A0000466F726D61743A46415433323B4D415882
:106A10003A3332470000000046696E6420552D4429
:106A200069736B2C4F7574707574696E6700000024
:106A300053746174653A49646C6500001CB70108C1
:106A40000CED00E00400FA052DE9F84F0025924610
:106A500088468146012715E000242E0109EB040138
:106A600001EB081000EB051000970278E006F1B288
:106A7000000E1023FBF7B6FA641CE4B2102CEDD321
:106A80006D1CEDB25545E7D3BDE8F88F06480021EF
:106A90000172817201214172C172642202618171AD
:106AA0000220FEF7FBBE0000D4120020124810B5F1
:106AB000016841F4700101601048016841F0010172
:106AC00001600E4A00210832116002680C4B1A4026
:106AD0000260031D0B4A1A60026822F480220260E1
:106AE00006480C300160FEF78FFD03494FF000604F
:106AF0008039086010BD000088ED00E000380240D9
:106B0000FFFFF6FE10300024FEF724BDC9430182CA
:106B100070470029018802D041F0010101E021F015
:106B20000101018070470000464910B5884206D136
:106B300001210846FEF75AFB002101205BE0B0F17D
:106B4000804F09D0404988420DD101210220FEF733
:106B500035FB0021022070E001210846FEF72EFBE4
:106B60000021012069E03949884206D10121042031
:106B7000FEF724FB002104205FE03549884206D15E
:106B800001210820FEF71AFB0021082055E03149B9
:106B9000884206D101211020FEF710FB00211020B1
:106BA0004BE02D49884206D101212020FEF706FB4B
:106BB0000021202041E02949884206D101210220FC
:106BC000FEF714FB0021022015E02549884202D17E
:106BD00001210C040AE02349884202D101214C041E
:106BE00004E0214988420AD101218C042046FEF7A5
:106BF000FDFA00212046BDE81040FEF7F7BA1B4918
:106C0000884206D101214020FEF7D8FA0021402019
:106C100013E01749884206D101218020FEF7CEFA01
:106C20000021802009E0134988420AD184150121FE
:106C30002046FEF7C3FA00212046BDE81040FEF7CB
:106C4000BDBA10BD00000140000400400008004033
:106C5000000C0040001000400014004000040140FF
:106C6000004001400044014000480140001800403D
:106C7000001C00400020004002460020138A928938
:106C80000B4202EA010202D0002A00D00120704724
:106C9000002A828901D00A4300E08A43828170473A
:106CA00030B50288164C174DA0420DD0A8420BD02B
:106CB000B0F1804F08D0144B984205D0134B984246
:106CC00002D0134B984203D122F070034A881A4332
:106CD000104B984206D0104B984203D022F44073D8
:106CE0000A891A4302804A68C2620A880285A04261
:106CF00001D0A84201D1897A01860121818230BD6B
:106D00000000014000040140000400400008004071
:106D1000000C0040001000400014004010B5FEF7C9
:106D2000BFF9FEF711FA00F0A9F9F3F75BF8154C7B
:106D300014F85C0F20F001002070207840F006006D
:106D400020700020608001460120F2F755FFF3F724
:106D500045FDF2F77DF9F2F7E1FDF3F707FEFBF7EA
:106D600011F8FFF793FEF3F7A7F9FAF725FCFDF703
:106D700081FB4FF4FA6024F8460C012004F8480C1B
:106D800010BD0000D41200202DE9F0410024F3F7DB
:106D900043FBB94E96F8F2040025012805D186F888
:106DA000F254F2F703FE0120B0713AE104EB440023
:106DB00006EB800090F83215012901D180F8325598
:106DC00090F83115002979D190F8A2190129FAD14A
:106DD00004EB440101EB041106EB011292F8161AC0
:106DE00000296BD080F8A25992F8160A072864D2BD
:106DF000DFE800F0EC04376591E1E10004EBC4004A
:106E000000EB042006EBC00090F8D31E012909D046
:106E100090F8D21E01EB411100EB810191F8D81ED0
:106E200000294AD190F8D21E491C80F8D21E90F851
:106E3000D01E29B190F8D01E80F8D21E80F8D05E06
:106E400090F8D21E01EB411100EB810191F8D81EA0
:106E5000052932D090F8D21E01EB411100EB8100E0
:106E6000A6E004EBC40000EB042006EBC00090F8A1
:106E7000D31E012909D090F8D21E01EB411100EB7D
:106E8000810191F8D81E002917D190F8D21E491C13
:106E900080F8D21E90F8D01E29B190F8D01E80F84C
:106EA000D21E80F8D05E90F8D21E01EB411100EBAB
:106EB000810191F8D81E0F29CCD187E0AFE004EB17
:106EC000C40000EB042006EBC00090F8D31E01299B
:106ED00008D090F8D21E01EB411100EB810191F82E
:106EE000D81E71BB90F8D21E491C80F8D21E90F8B3
:106EF000D01E29B190F8D01E80F8D21E80F8D05E46
:106F000090F8D21E01EB411100EB810191F8D81EDF
:106F100007299FD15AE004EBC40000EB042006EBE4
:106F2000C00191F8D30E012808D091F8D20E00EBE1
:106F3000401001EB800090F8D80E10B991F8D20EF5
:106F400019E037E091F8D23E02EB031393F8413A8F
:106F500002EB001797F8517ABB4205D091F8D20E98
:106F6000401C81F8D20E0AE091F8D23E5B1C81F8F9
:106F7000D23E401CC0B292F8173A8342E2D891F850
:106F8000D00E28B191F8D00E81F8D20E81F8D05EE3
:106F900091F8D20E00EB401001EB800090F8D80E73
:106FA000052813D091F8D20E00EB401001EB8000C1
:106FB00080F8D85E0AE004EBC40000EB042006EB86
:106FC000C00090F8D21E491C80F8D21E04EBC40009
:106FD00000EB042006EBC00090F8D21E92F8172AAE
:106FE000914201D380F8D25E90F8D11E51B190F851
:106FF000D21E80F8D01E90F8D11E491E80F8D21EF5
:1070000080F8D15E90F8D21E01EB411100EB8101B6
:1070100091F8DD2E90F8D21E2046F8F755FE641C3C
:10702000E4B296F86C09A0423FF6C0AE96F822068C
:1070300020B196F8FE04012807D010E096F80A0562
:1070400001280CD186F80A5501E086F8FE5496F81E
:10705000252696F8211696F82206FCF7C5FCF3F7CC
:107060006DFD96F8240618B186F82456FBF714F93E
:10707000BDE8F041FEF71ABCD4120020FEB5012194
:1070800000240846FEF78EF8A720ADF80000002681
:1070900040F2E73001904FF08045ADF80260ADF866
:1070A000086069462846FFF7FBFD724981F83E6695
:1070B00004EB440001EB800091F83E3600F5A66237
:1070C00001EB8303C3F8402691F83E26521C81F859
:1070D0003E2691F83E3600F51A6201EB8303C3F8B1
:1070E000402691F83E26521C81F83E2691F83E3605
:1070F00000F5176201EB8303C3F8402691F83E26A2
:10710000521C81F83E2691F83E2600F5405001EBD6
:107110008202C2F8400691F83E06401C81F83E0605
:1071200004EBC40202EB0422002001EBC20300EBDB
:10713000401291F83E6603EB820201EB860602F6EE
:10714000E462C6F8402691F83E26521C81F83E269D
:10715000401CC0B21028EAD3641CE4B2042CA7D3AC
:10716000454891F83E2601EB8202C2F8400691F8AC
:107170003E06401C81F83E063F4891F83E262838DE
:1071800001EB8202C2F8400691F83E06401C81F8ED
:107190003E06394891F83E261C3801EB8202C2F8BF
:1071A000400691F83E06401C81F83E06324891F8B0
:1071B0003E26103801EB8202C2F8400691F83E06E6
:1071C000401C81F83E062D4891F83E2601EB8202D4
:1071D000C2F8400691F83E06401C81F83E06284859
:1071E00091F83E2601EB8202C2F8400691F83E0675
:1071F000401C81F83E06204891F83E26343801EBC9
:107200008202C2F8400691F83E06401C81F83E0614
:107210001C4891F83E2601EB8202C2F8400691F824
:107220003E06401C81F83E06124891F83E26083082
:1072300001EB8202C2F8400691F83E06401C81F83C
:107240003E06104891F83E260C3801EB8202C2F847
:10725000400691F83E06401C81F83E060121284672
:10726000FFF757FC012211462846FFF711FD00F0F9
:107270000BF8FEBDD4120020F8170020FC180020E7
:10728000341C00201043002008B51C208DF800009D
:1072900001208DF8010002218DF802108DF8030005
:1072A0006846FAF7ADFC08BDF9F7A0BEF9F7BEBE17
:1072B000FDF70EB8F9F774BEF9F7D6BEF3F7AAB921
:1072C000C943018070470029818902D041F40051EF
:1072D00001E021F4005181817047002A828A01D0A7
:1072E0000A4300E08A438282704700001C4910B5BF
:1072F000884206D101211020FDF778FF00211020DF
:1073000028E01849884202D101214C0410E01649B6
:10731000884202D101218C040AE01449884202D13A
:107320000121CC0404E0124988420AD101210C0554
:107330002046FDF743FF2046BDE810400021FDF741
:107340003DBF0C49884209D101212020FDF74EFFA5
:1073500000212020BDE81040FDF748BF10BD00000F
:10736000001001400044004000480040004C004034
:1073700000500040001401400246002012880A42DA
:1073800000D00120704770B501F01F0501260024D0
:10739000C1F3421306FA05F2012B0FD0022B0FD0D6
:1073A000838A4FEA11210088134206FA01F600EAA7
:1073B000060001D000B10124204670BD8389F0E7AA
:1073C000038AEEE710B5C1F3421301F01F04012157
:1073D000A140012B07D0022B07D01430002A0268ED
:1073E00005D00A4304E00C30F8E71030F6E78A4392
:1073F000026010BD7FB50446008A0D46C98820F49E
:10740000405001432182A08941F20C618843A98840
:107410002A8911436A8902431143A181A08A20F479
:107420004071A8890843A0826846FDF7EBFE1A4820
:10743000844202D01948844201D1039800E00298A6
:10744000A189090400EBC00101EB0010296801D5F6
:10745000490000E08900B0FBF1F06422B0FBF2F1DA
:1074600009010B096FF018056B4300EB8300A3893A
:107470001D044FF0320306D503EBC000B0FBF2F061
:1074800000F0070005E003EB0010B0FBF2F000F0A5
:107490000F00084320817FBD00100140001401400F
:1074A00070B50024064DFDF751FE20B1641CAC42BE
:1074B000F9D3FA2070BDBDE87040F1F7EBBF0000D2
:1074C000404B4C000FB4084B10B504A902AA039816
:1074D00001F0E2F9044602A9002001F008FC204670
:1074E00010BC5DF814FB0000EF8C010803B4019898
:1074F0004100009850EAC12018BF04204A0D18BF6F
:1075000040F0010040F2FF72B2EB515F08BF40F063
:107510000200012808BF052002B0704700000000EB
:1075200030B583B0044601F093F99FED090B054691
:107530008DED000B002221466846F1F72EF9284612
:1075400001F09CF99DED000B03B030BD0000000080
:10755000000000000000000070B5D94B00242DEDA4
:10756000020B2DED108BDDE91010984205DA20F0AA
:1075700000429A4201D809D141B19DED100BBDECFA
:10758000108B02B0BDE8704001F01EB9B0F5801F4D
:1075900026DA11430BD0002813DA012001F06EF92E
:1075A000BDEC108B02B0BDE8704001F021B90220A3
:1075B00001F064F901F0F0F851EC100B81F000419A
:1075C0009EE06FF035049FEDC00B53EC102B9DED4A
:1075D000100B51EC100BF0F713FFCDE9100108462A
:1075E00004EB2051C0F31304B948A1F2FF31204449
:1075F00000F4801080F07F6282F04052224301EB61
:1076000020559FEDB50B119253EC102B9DED100BF7
:1076100051EC100BF0F7EEFE41EC180BA01CC0F380
:1076200013009FEDAFDB9FEDB0EBB14E7E4403281E
:107630006CD296ED000B51EC180B53EC102BF1F7BC
:10764000EDFB1DD1002D01BF96ED000BBDEC108BA5
:1076500002B070BD2846F1F77EF941EC180B53ECEF
:107660001D2BF0F7CDFE41EC190B53EC1E2B51EC0A
:10767000180BF0F7C5FE53EC192BF0F71AFE3FE09C
:107680009FED9D0B51EC180B53EC102BF0F7B8FE4F
:107690009FED9B1B53EC112BF0F7AFFE41EC190B48
:1076A00053EC182B51EC180BF0F7AAFE53EC192BE6
:1076B000F0F7A6FE41EC190B002D04BF53EC192B7B
:1076C00051EC180B1AD02846F1F745F941EC1A0B8A
:1076D00053EC1D2BF0F794FE53EC192BF0F78DFEB5
:1076E00053EC182BF0F786FE41EC180B53EC1E2BD5
:1076F00051EC1A0BF0F784FE53EC182BF0F77AFEDE
:10770000BDEC108B02B041EC100B70BD9FED7E0BF9
:1077100051EC180B53EC102BF0F7CBFD41EC100B98
:1077200051EC180B53EC102BF0F7DCFE41EC190B6D
:107730002846F1F710F941EC1B0B53EC192B51ECD7
:10774000190BF0F75DFE41EC1A0B714853EC1A2B44
:10775000261851EC1A0BF0F753FE41EC1F0B6D4845
:10776000C4F1510404F5D724B0EE4F0AF0EE6F0ACD
:107770000321784400F094FF53EC1F2B51EC100BC5
:10778000F0F73EFE41EC1C0B6348B0EE4F0AF0EE02
:107790006F0A0421784400F083FF53EC1A2B51EC5C
:1077A000100BF0F72DFE344353EC1C2BF0F781FD4A
:1077B00041EC1C0B002C4CDD9FED510B51EC180BD8
:1077C00053EC102BF0F71CFE53EC182BF0F718FEBF
:1077D00041EC1A0B55B353EC1D2B51EC1B0BF0F77E
:1077E0000FFE41EC1D0B53EC1C2B51EC1A0BF0F768
:1077F00060FD53EC192BF0F703FE53EC1D2BF0F753
:1078000058FD53EC1A2BF0F7F8FD53EC182BF0F75A
:10781000F1FD41EC180B53EC1E2B51EC1B0BF0F758
:10782000EFFD53EC182BF0F7E5FD69E753EC1C2B4B
:1078300051EC1A0BF0F73DFD53EC192BF0F7E0FD7E
:1078400053EC1A2BF0F7D9FD53EC182BF0F7D5FDBC
:1078500056E735B353EC1D2B51EC1B0BF0F7D0FD65
:1078600041EC1A0B53EC1C2B51EC180BF0F7C2FD3A
:1078700053EC192BF0F7C4FD53EC1A2BF0F7BAFDBB
:1078800053EC182BF0F7B6FD41EC180B53EC1E2B04
:1078900051EC1B0BF0F7B4FD53EC182BF0F7AAFDDD
:1078A0002EE753EC1C2B51EC180BF0F7A3FD53EC17
:1078B000192BF0F7A5FD53EC182BF0F79EFD1FE7F1
:1078C0000000F07F000000000000000000005043B6
:1078D000645F090000000000000000000000F03FAD
:1078E000763C7935EF39EA3D0000E0FE422EE63F76
:1078F0003042000000000000555555555555D53F04
:10790000000000000000E03F000000000000004018
:1079100086EBF9FFB2400000A84000000000000024
:1079200070B5414A00252DED020B2DED048BDDE9EC
:107930000404944205DA24F00041914201D809D1AF
:1079400040B19DED040BBDEC048B02B0BDE870406E
:1079500000F03ABFB4F5801F26DA08430BD0002CA4
:1079600013DA012000F08AFFBDEC048B02B0BDE801
:10797000704000F03DBF022000F080FF00F00CFFDF
:1079800051EC100B81F0004146E09FED290B6FF0A8
:10799000350553EC102B9DED040B51EC100BF0F75B
:1079A0002FFDCDE904010C4605EB2450A0F2FF3079
:1079B000C10F40F2FF32521A62F31F540844F0F72D
:1079C000CAFF05949DED040B41EC180B51EC100B14
:1079D00001F0C6FA9FED181B53EC112BF0F710FDC8
:1079E0009FED170B41EC190B53EC102B51EC180BBE
:1079F000F0F706FD53EC192BF0F75BFC9FED120B33
:107A000041EC190B53EC102B51EC180BF0F7F8FC70
:107A100053EC192BF0F74DFCBDEC048B02B041EC9C
:107A2000100B70BD000000000000F07F000000009F
:107A300000000000000050430EE526157BCBDB3F25
:107A4000362BF111F3FE593D00609F501344D33F94
:107A50002DE9F04D2DED040B2DED0E8B96B0DDE9EB
:107A60002550279CDDF890A025F0004624F0004822
:107A7000BAF1000F14BF0121002101EB4502FC49BE
:107A800053184A1093422AD3002814BF012300231D
:107A900003EB44030B44F7498B4220D358EA00011F
:107AA0009FEDF59B76D0DFF8D8B35D4503D1BAF1F1
:107AB000000F05D188E0BAF1000F08BF002100D007
:107AC000012101EB450111F5001F08D8002814BF62
:107AD0000121002101EB440111F5001F0BD99DED9F
:107AE000261B9DED240B16B0BDEC0E8B04B0BDE83B
:107AF000F04D00F073BE0027002DBCBFE149884562
:107B000021DAE1498845A8BF02271CDAC3451ADCFF
:107B1000DE4901EB2851142908DDC1F1340220FAB5
:107B200002F101FA02F282420DD108E058B9C1F126
:107B3000140228FA02F101FA02F2424503D101F0DF
:107B40000101C1F1020756EA0A0124D1002C22DA10
:107B5000002D18BF022F01D0012F0AD0022000F003
:107B60008DFE16B0BDEC0E8B04B0BDE8F04D00F0FC
:107B700013BE022000F082FE00F00EFE51EC100B4E
:107B800081F0004141EC100B16B0BDEC0E8B04B03F
:107B9000BDE8F08D18E09FEDBEAB9FEDBF8B0028D8
:107BA00071D1B848804522D105F1804010F5801090
:107BB00008BFBAF1000F07D0B3450ADC002CA8BFFC
:107BC0009DED260BE0DA0DE0B0EE490AF0EE690A11
:107BD000DAE7002C06DA9DED260B51EC100B81F054
:107BE00000416FE0AE48784490ED000BCCE7D845FB
:107BF0004DD1002C48DA2EB186423AD1BAF1000FAD
:107C000042D126E0BAF1000F13D0022000F036FE78
:107C100000F0FEFD8DED020B9DED240B8DED000BB4
:107C200010EE900A039961F31E0003909DED020B84
:107C3000AAE78DED02AB9DED240B1AEE901A10EE23
:107C4000900A8DED000B61F31E0003909DED020B79
:107C50009AE78DED028B9DED240B18EE901A10EE35
:107C6000900A8DED000B61F31E0003909DED020B59
:107C70008AE709DA9DED240B51EC190B53EC102B1C
:107C8000F0F730FC1EE020E09DED240B7CE78642FF
:107C90001BDAB4F1804F0DD0A4F10050B0F1FF50C9
:107CA00013D1002D11DB9DED240B51EC100B01F0D5
:107CB000E2F907E09DED240B53EC102B51EC100B77
:107CC00000F0C2BC41EC100B5EE79DED240B51ECC3
:107CD000100B01F039F8BAF1000FCDE90E0142D1D5
:107CE0009FED710B46B3A6F1E040B0F17F600CD080
:107CF0005E4538D1002D00DAA7B3022F0CBF01205A
:107D00004FF0FF30F0F727FEDCE7002D01DD002CFF
:107D10000DDA002D01DD002C1FDB002D16DA002C02
:107D200014DB012F08BF9FED620B3FF42DAFB0EEC7
:107D30004A0AF0EE6A0A27E7022F18BF002D0CD07E
:107D4000012F0AD1002DFFF61FAF06E0002DB8BFAE
:107D5000002C08DA012F3FF417AFB0EE480AF0EE1E
:107D6000680A11E71BE0012000EBE57050EA07010B
:107D700015D0791EB0EE498AF0EE698A084308BF33
:107D80009FED4D8B4E480025804570DD4D494E4896
:107D9000884514DDB0420DDB002C19DB2FE00120FB
:107DA00000F06CFD16B0BDEC0E8B04B0BDE8F04DDC
:107DB00000F01EBDB34502DC002C09DC1FE086424A
:107DC00002DA002C1BDA03E05E452BDD002C16DD09
:107DD000022000F053FD00F01BFD8DED020B53EC73
:107DE0001A2B51EC180BF0F70BFBCDE900010399AE
:107DF000019861F31E0003909DED020BC4E6022082
:107E000000F03CFD00F014FD10EE901A18EE900A00
:107E10008DED020B8DED008B61F31E0003909DED47
:107E2000020BB1E69DED0E0B53EC192B51EC100B30
:107E3000F0F7E0FA9FED260BCDE9080153EC102B8B
:107E40009DED080B51EC100BF0F7DAFA9FED221BB9
:107E500053EC112BF0F7D1FA9DED081B53EC112BCD
:107E6000F0F7CEFA9FED1E1B53EC112B3CE08CE09B
:107E7000FFFF1F00FFFF0F00000000000000F03FA9
:107E80000000F03F0000F07F0000404301FCFFFFD6
:107E9000000000000000F07F000000000000000073
:107EA000763C0000000000000000000000000080A0
:107EB000000000000000F0FF000000000000F0BF24
:107EC0000000E0410000F043FFFFEF3F0000000032
:107ED000000000000000D03F555555555555D53F81
:107EE000000000000000E03FF0F787FA9DED080B6E
:107EF00041EC1A0B53EC102B51EC100BF0F780FAFD
:107F000053EC1A2BF0F77CFA41EC1A0B9FEDFE0BA9
:107F100053EC102B9DED080B51EC100BF0F770FAA1
:107F200041EC1B0B9FEDFA0B51EC1A0B53EC102B91
:107F3000F0F766FA41EC1A0B9FEDF70B53EC102BA0
:107F40009DED080B51EC100BF0F75AFA53EC1A2B7D
:107F5000F0F750FA41EC1A0B51EC1B0B53EC1A2BB7
:107F6000F0F7A7F90690CDE906519DED060B53EC0D
:107F70001B2B51EC100BF0F73DFA53EC1A2BF0F7DA
:107F80003CFA41EC100B00F0A1B90020B6F5801FBF
:107F90000EDA9FEDE30B53EC102B9DED0E0B51EC25
:107FA000100BF0F72DFACDE90E016FF034000E46FC
:107FB00000EB2650A0F2FF37C6F31300DA4940F079
:107FC0007F6646F040568842D8BF002408DDD74976
:107FD0008142C8BF012403DC0024A6F580167F1C63
:107FE000D348784400EBC4000F9690ED00CB9DED94
:107FF0000E0B53EC1C2B51EC100BF0F7FBF99DED25
:108000000E0B41EC1B0B53EC1C2B51EC100BF0F73F
:1080100050F941EC100B51EC190B53EC102BF0F70D
:1080200061FA41EC1D0B51EC1B0B53EC1D2BF0F7CF
:10803000E7F941EC1A0BBF488DED10AB7844109571
:1080400090ED000B4FF0005040EA660000EB8440DA
:108050008DED080B00F5002009909DED080B53EC09
:108060001C2B51EC100BF0F7C5F99DED0E1B53ECDA
:10807000112BF0F7C2F941EC100B53EC102B9DEDD6
:10808000100B51EC100BF0F7BBF99DED080B41EC18
:108090001C0B53EC102B9DED100B51EC100BF0F75B
:1080A000AFF953EC1B2BF0F7A8F953EC1C2BF0F7AE
:1080B000A1F953EC1D2BF0F7A3F941EC1C0B53EC89
:1080C0001A2B51EC1A0BF0F79BF941EC1B0B9A4859
:1080D0000621B0EE4B0AF0EE6B0A784400F0E0FAAD
:1080E000B0EE401AF0EE601AB0EE41DAF0EE61DA6E
:1080F00053EC1B2B51EC1B0BF0F782F953EC1D2BAF
:10810000F0F77EF99DED100B41EC1B0B53EC1A2B95
:1081100051EC100BF0F7CDF853EC1C2BF0F770F985
:1081200053EC1B2BF0F7C5F89DED100B41EC1B0B2E
:1081300053EC102B51EC100BF0F762F941EC1D0BD6
:108140009FED7FEB53EC1E2BF0F7B3F853EC1B2B9A
:10815000F0F7AFF80890CDE908519DED080B53EC0E
:108160001E2B51EC100BF0F745F953EC1D2BF0F7DB
:1081700041F953EC1B2BF0F740F99DED080B41EC56
:108180001D0B53EC102B9DED100B51EC100BF0F769
:1081900037F941EC1B0B53EC1A2B51EC1D0BF0F78C
:1081A0002FF99DED080B41EC1A0B53EC102B51EC01
:1081B0001C0BF0F725F953EC1A2BF0F77AF841EC89
:1081C0001A0B51EC1B0B53EC1A2BF0F772F80C90B6
:1081D000CDE90C519DED0C0B53EC1B2B51EC100B0E
:1081E000F0F708F953EC1A2BF0F707F941EC1B0BE9
:1081F0009FED550B53EC102B9DED0C0B51EC100B20
:10820000F0F7FEF841EC1A0B9FED510B51EC1B0BF4
:1082100053EC102BF0F7F4F841EC1B0B9FED4E0BD9
:1082200053EC102B9DED0C0B51EC100BF0F7E8F814
:1082300053EC1B2BF0F73DF841EC100B4848784409
:1082400000EBC40090ED001B51EC100B53EC112B14
:10825000F0F72FF841EC1B0B3846F0F77CFBCDE92B
:10826000080153EC1B2B51EC1A0BF0F722F841ECF0
:10827000100B3C48784400EBC40090ED00CB51EC6F
:10828000100B53EC1C2BF0F714F89DED081B53EC6E
:10829000112BF0F70EF80690CDE906519DED080B75
:1082A00053EC102B9DED060B51EC100BF0F7A2F8E0
:1082B00053EC1C2BF0F79EF853EC1A2BF0F79AF8BE
:1082C00053EC1B2BF0F799F841EC100B9DED261B9E
:1082D00053EC102B8DED001B00959DED260B51EC02
:1082E000100BF0F78DF89DED000B41EC1A0B53ECE1
:1082F000102B9DED260B51EC100BF0F77BF89DED4C
:10830000061B53EC112B2FE0000000604715F73FD0
:10831000FE822B654715F73F44DF5DF80BAE543EF8
:1083200000000000000040438E9803007AB60B0066
:10833000BA37000020380000F236000000000000CC
:108340000000000000000840000000E009C7EE3F08
:10835000FD033ADC09C7EE3FF5015B14E02F3EBE9A
:108360007E35000038350000F0F74AF853EC1A2B40
:10837000EFF79FFF9DED060B41EC1A0B53EC102B12
:108380009DED000B51EC100BF0F73AF8CDE90C0124
:108390009DED0C0B51EC1A0B53EC102BEFF789FFF2
:1083A000CDE902010C46AA498C422FDB611A084331
:1083B00018D19DED0C0B53EC102B9DED020B51ECE5
:1083C000100BF0F717F841EC1B0B9FEDA30B51ECD2
:1083D0001A0B53EC102BEFF76CFF53EC1B2BF0F741
:1083E000CBFA2DD2022000F049FA00F011FA10EE7B
:1083F000901A18EE900A8DED020B8DED008B61F353
:108400001E0003909DED020BFFF7BEBB944A24F0C3
:108410000041914214D39349214408437FF4EFACC7
:108420009DED0C0B53EC102B9DED020B51EC100B42
:10843000EFF7E0FF53EC1A2BF0F79EFA7FF6DFAC74
:1084400024F000408849894A002601EB20518242ED
:108450002BDA481C4FF4801121FA00F02044844AA2
:10846000C0F30A517A44A1F2FF3192ED000B814A28
:108470008DED080BCA4020EA0202C0F3130040F45D
:108480008010C1F1140120FA01F60992002CB8BF46
:1084900076429DED080B53EC102B9DED0C0B51EC2F
:1084A000100BEFF7A7FFCDE90C019DED0C0B51EC84
:1084B0001A0B53EC102BEFF7FCFE9FED6F0B08909F
:1084C000CDE9085153EC102B9DED080B51EC100B2E
:1084D000EFF796FF41EC1B0B9FED690B53EC102B54
:1084E0009DED080B51EC100BEFF78AFF9DED0C0B87
:1084F00041EC1C0B53EC102B9DED080B51EC100BB9
:10850000EFF778FF53EC1A2BEFF777FF9FED5E1B29
:1085100053EC112BEFF774FF53EC1C2BEFF7C9FE54
:1085200041EC1A0B51EC1B0B53EC1A2BEFF7C1FE6D
:10853000CDE902019DED020B53EC1B2B51EC100B0E
:10854000EFF758FF53EC1A2BEFF757FF9DED020B97
:1085500041EC1A0B53EC102B51EC100BEFF750FFC2
:10856000CDE908014A489DED080B0521784400F04B
:1085700097F89DED081B51EC100B53EC112BEFF706
:108580003FFF9DED021B53EC112BEFF736FFCDE9BA
:1085900006019DED020B53EC1A2B51EC100BEFF77B
:1085A0002FFF53EC1A2BEFF784FE9FED3B0B41ECB2
:1085B0001A0B53EC102B9DED060B51EC100BEFF743
:1085C00019FF9DED060B41EC1B0B53EC102B9DEDA1
:1085D000020B51EC100BEFF713FF53EC1B2BEFF7D3
:1085E00081FF53EC1A2BEFF705FF9DED021B53ECB7
:1085F000112BEFF7FFFE53EC192BEFF7FEFECDE941
:10860000020101EB065001150029C8BF039015DCDB
:108610009DED020B324651EC100BF0F785F9FEF799
:1086200065FF042808BF00F003F932469DED020BF8
:1086300051EC100BF0F778F9CDE902019DED020B3A
:1086400051EC180B53EC102BEFF7DAFEFFF73ABBA7
:108650000000904000000000FE822B654715973C0B
:1086600000CC904000346F3F01FCFFFF0000E03F72
:10867000F8330000FFFF0F0000000000432EE63F2C
:10868000396CA80C615C20BEEF39FAFE422EE63F41
:1086900090320000000000000000000000000040D8
:1086A00070B504462DED028B4D1E00EBC500B0EEFB
:1086B000408AF0EE608A90ED000B35F0060017D08E
:1086C00053EC182B51EC100BEFF79AFE41EC100B0A
:1086D0006D1E04EBC50090ED001B51EC100B53EC2C
:1086E000112BEFF7E6FD41EC100B35F00600E7D15A
:1086F000022D36D0042D1CD0062D1CBFBDEC028BE4
:1087000070BD53EC182B51EC100BEFF779FE94ED84
:108710000A1B53EC112BEFF7CCFD53EC182BEFF7A2
:108720006FFE94ED081B53EC112BEFF7C2FD41ECEB
:10873000100B53EC182B51EC100BEFF761FE94ED7E
:10874000061B53EC112BEFF7B4FD53EC182BEFF78E
:1087500057FE94ED040B53EC102BEFF7AAFD41EC00
:10876000100B53EC182B51EC100BEFF749FE94ED66
:10877000021B53EC112BEFF79CFD53EC182BEFF77A
:108780003FFE94ED001B53EC112BEFF792FDBDEC77
:10879000028B41EC100B70BD9FED070B10B553EC35
:1087A000102B9FED070B51EC100BEFF79BFE41ECEC
:1087B000100B10BD000000000000000000000000D1
:1087C000000000000000F03F10B553EC102B51ECFE
:1087D000100BEFF76EFD41EC100B10BD10B553EC14
:1087E000112B51EC100BEFF764FD41EC100B10BD99
:1087F0009FED050B10B553EC102B51EC100BEFF760
:1088000071FE41EC100B10BD0000000000000000E4
:108810009FED050B10B553EC102B51EC100BEFF73F
:10882000EFFD41EC100B10BD0000000000000070D7
:108830009FED050B10B553EC102B51EC100BEFF71F
:10884000DFFD41EC100B10BD000000000000001027
:108850000148006870470000D012002002E008C8FC
:10886000121F08C1002AFAD170477047002001E0AA
:1088700001C1121F002AFBD17047000001490860A6
:1088800070470000D012002030380A2801D20120A1
:1088900070470020704700002DE9FF4F8DB00F4654
:1088A0000546002606E025280BD0DDE90F1290478B
:1088B0006D1C761C28780028F5D111B03046BDE833
:1088C000F08F0024A246A1460122E94900E00443BA
:1088D00015F8013F203B02FA03F00842F7D128784F
:1088E0002A2810D06FF02F022878A0F13001092932
:1088F00014D80AEB8A0102EB410144F0020400EBB8
:10890000010A6D1CF0E701CF5FEA000A03D544F4C9
:108910000054CAF1000A44F002046D1C28782E2885
:1089200017D115F8010F44F004042A280ED06FF077
:108930002F022878A0F1300109290AD809EB890112
:1089400002EB410100EB01096D1CF2E757F8049BB3
:108950006D1C28786C280FD006DC4C2817D06828AE
:108960000DD06A2814D104E0742810D07A280FD1D1
:108970000DE044F400140AE044F4801401E044F4EF
:1089800040146978814202D104F580146D1C6D1C7D
:1089900028786E281ED00CDC632830D004DC002838
:1089A0008BD0582811D19FE0642867D069280CD15A
:1089B00064E073282DD004DC6F2872D0702804D1B5
:1089C00094E075286ED078286DD0DDE90F129047BD
:1089D000761C4BE1C4F30250022806D0032809D0CC
:1089E000042801CF09D0066040E101CFF117C0E9AA
:1089F00000613BE101CF068038E1067036E117F8EF
:108A0000040B8DF8000000208DF80100EB460120DA
:108A100003E057F804BB4FF0FF3061074FF000014F
:108A200002D40DE008F10101884649450FDA80457E
:108A3000F8DB1BF808100029F4D108E008F1010167
:108A400088468142FADB1BF808100029F6D1DDE9DF
:108A50000F23AAEB08008146214600F031F930448B
:108A600000EB080604E0DDE90F121BF8010B90474C
:108A7000B8F10108F7D221464846F2E00A21C4F3D2
:108A800002524FF0000B0891022A04D001CFC11707
:108A9000032A09D00AE0FF1D27F00707F7E80201C3
:108AA00008E02CE01EE01FE000B2C117042A01D14B
:108AB00040B2C117021E71F1000206DA0023D0EBAA
:108AC000030063EB01012D2202E0220504D52B22D5
:108AD0008DF82420012203E0E20701D02022F7E7ED
:108AE000904653E00A210BE0102109E010214FF0DD
:108AF000000B44F004044FF00809089103E008213A
:108B00004FF0000B0891C4F30252022A04D001CFA7
:108B10000021032A06D006E0FF1D27F00707F7E82B
:108B2000020103E080B2042A00D1C0B24FF0000875
:108B300022072BD52A78702A07D0DDF820C08CF0C8
:108B4000100C5CEA0B0C05D00EE040228DF82420BE
:108B5000012208E050EA010306D030238DF82430CA
:108B60008DF8252002229046089B83F0080353EAE3
:108B70000B030BD150EA010201D1620706D5302266
:108B80008DF824204FF00108A9F101092A78582A0C
:108B900004D038A20B9208AA0A920BE03AA2F9E795
:108BA0005B46089AEFF78EFD0B9B9B5C0A9A521E60
:108BB0000A92137050EA0102F2D10A98ADEB00005C
:108BC00000F1200B600702D524F4803401E04FF05F
:108BD0000109D94502DDA9EB0B0000E0002000EB04
:108BE0000B0141440890AAEB010AE00306D4DDE939
:108BF0000F232146504600F063F806444FF0000969
:108C000008E009A911F80900DDE90F12904709F100
:108C10000109761CC145F4DBE0030CD5DDE90F2327
:108C20002146504600F04CF8064404E0DDE90F12FE
:108C300030209047761C0899481E08900029F5DCE2
:108C400008E00A980A990078491C0A91DDE90F1298
:108C50009047761CBBF10001ABF1010BF1DC214622
:108C60005046DDE90F2300F019F806446D1C21E69B
:108C700009280100303132333435363738396162F2
:108C800063646566000000003031323334353637B6
:108C90003839414243444546000000002DE9F04187
:108CA000044600251E461746880404D405E03946CC
:108CB0002020B0476D1C641EF9D52846BDE8F08120
:108CC0002DE9F041044600251E469046C80301D513
:108CD000302700E02027880404D505E041463846C7
:108CE000B0476D1C641EF9D52846BDE8F0810A68BE
:108CF000531C0B6010707047002806D04DF6BC2343
:108D00001946491EFDD2401EFAD17047002100EBE2
:108D1000800002E000BF491CC9B2B1EB400FF9D39B
:108D20007047000010B502460020064C07E012F81C
:108D3000013B4340DBB234F8133083EA1020491E74
:108D4000F5D210BD1608002082B0CDE9000121F057
:108D5000004001909DED000B02B051EC100B7047EC
:108D600010B50E4C10212046F1F751FB206840F45D
:108D70008060206020212046F1F749FB0220FFF7A8
:108D8000C5FF10212046F1F744FB0220FFF7BEFF8C
:108D90002046BDE810401021F1F739BB0014024015
:108DA00010B50E4C10212046F1F731FB206840F43D
:108DB0008060206020212046F1F72BFB0220FFF786
:108DC000A5FF10212046F1F724FB0220FFF79EFFAC
:108DD0002046BDE810401021F1F719BB00140240F5
:108DE0002DE9F041154E07460024306820F440601C
:108DF0003060254610213046F1F709FB0220FFF7CD
:108E000085FF10213046F1F704FB6006040E202197
:108E10003046F1F7F5FA08B144F001040120FFF7FC
:108E200075FF6D1CEDB2082DE4D317B1FFF798FF65
:108E300001E0FFF7B5FF2046BDE8F08100140240D5
:108E400070B5164E05463046316841F48061316098
:108E50001021F1F7DCFA002428064FF020013046FB
:108E600002D5F1F7D6FA01E0F1F7D1FA6806050E5E
:108E70000220FFF74BFF10213046F1F7CAFA02201B
:108E8000FFF744FF10213046F1F7C1FA0220FFF747
:108E90003DFF641CE4B2082CDED370BD0014024018
:108EA00010B50B4C206840F48060206020212046E3
:108EB000F1F7AFFA10212046F1F7ABFA0420FFF7E3
:108EC00025FF2046BDE810402021F1F7A0BA0000A0
:108ED0000014024010B50B4C206840F48060206004
:108EE00020212046F1F793FA0420FFF70FFF10210D
:108EF0002046F1F78EFA2046BDE810402021F1F718
:108F000088BA00000014024070B5144D002428688F
:108F100020F44060286020212846F1F77AFA0120E9
:108F2000FFF7F4FE10212846F1F773FA0120FFF74E
:108F3000EDFE07E0641CE4B2FA2C03D9FFF7CAFF88
:108F4000012070BD20212846F1F75AFA0028F1D1FE
:108F500010212846F1F75BFA002070BD0014024092
:108F600010B541EC100BFEF7F7FA51EC100B10BDE9
:108F700070B5FCF7FFF9062000F0BEF8552000F0B0
:108F8000DBF800F0AFF8124E04464FF48055294646
:108F90003046F1F73CFA29460E48F1F73AFAAA2C86
:108FA00011D1152000F0A8F8062000F0C5F8142013
:108FB000FFF7ACFE00F096F8044629463046F1F77C
:108FC00028FA512C01D0FA2070BD142070BD000089
:108FD00000040240000C02404FF400410803F8F77F
:108FE00041FE4FF08040FDF79FFD0F48FEF77EF9F0
:108FF0000E48F0F7C1FB0D483030F0F7BDFB0C48D0
:10900000F1F740F90B48F1F73DF9F1F7A7FC002023
:1090100080F310884FF47A70FFF76EFEFDF77EFE46
:10902000FDF7B2FEFCE7000000100140886402403A
:1090300000000240000402402DE9F04104460E46C3
:1090400000250846EFF71FF907000ED10120BDE803
:10905000F0816D1C3178ADB2884205D13A46314677
:109060002046EFF717F920B1641C20780028F0D1D2
:10907000EDE72846EBE700B52DED048B83B041EC1E
:10908000190BEFF779FE41EC180B18EE100A18EEE9
:10909000901A8DED008B002818BF0120084320F0A6
:1090A0000040C0F17F6000F1E040C00F14D019EE25
:1090B000101A19EE900A8DED009B002918BF0121AE
:1090C000084320F00040C0F17F6000F1E040C00F95
:1090D00004BF0120FFF7D2FB51EC180B03B0BDEC2D
:1090E000048B00BD10B50120FFF710FEBDE8104055
:1090F000FF20FCF7AFB9000070B50D4E04464FF4E9
:10910000805529463046F1F784F90320FFF7FEFD2C
:1091100029463046F1F77BF929460648F1F779F9F7
:109120002046FCF797F9BDE870400320FFF7EEBD3D
:1091300000040240000C024010B5FCF78BF9BDE8BA
:1091400010400120FFF7E2BD5458485F56312E32DF
:109150002E32003880250000010000000A000000C7
:1091600000000000000000000000000000000000FF
:1091700000000000000000000000000000000000EF
:1091800000000000010100000000000000000000DD
:1091900000000000020300000000000000000000CA
:1091A00000000000030500000000000000000000B7
:1091B00000000000040700000000000000000000A4
:1091C0000000000005050000000000000000000095
:1091D0000000000006060000000000000000000083
:1091E0000000000007070000000000000000000071
:1091F000000000000808000000000000000000005F
:10920000000000000909000000000000000000004C
:10921000000000000A0A000000000000000000003A
:10922000000000000B0B0000000000000000000028
:10923000000000000C0C0000000000000000000016
:10924000000000000D0D0000000000000000000004
:10925000000000000E0E00000000000000000000F2
:10926000000000000F0F00000000000000000000E0
:1092700000000000101000000000000000000000CE
:10928000000000006A6F796675656C2E6A6F7966FA
:1092900075656C696E672E636F6D2C3730313100E8
:1092A00000000000000000000000000000000000BE
:1092B00000000000000000000000000000000000AE
:1092C000000000000000000000000000000000009E
:1092D000000000000000000000000000000000008E
:1092E000000000000000000000000000000000007E
:1092F00000004B46422D322E344700000000000093
:10930000000000000000000000000000000000005D
:10931000000000000000000000004B4642313233E4
:10932000343536000000000000000000000000009E
:10933000000000040000000000000000539101083C
:1093400020430020371300206400000002000100C9
:10935000000000003093010820430020301300205B
:1093600066000000050001000100000054910108A2
:1093700020430020E41C00206B00000031010400A9
:109380000200000084920108204300204A180020B7
:109390002F050000AC000100030000002F9301081E
:1093A00020430020401C0020DB05000002000100DB
:1093B00004000000349301082043002028130020FB
:1093C000DD050000050001000500000038930108DC
:1093D000204300202C130020E205000005000100BE
:1093E0000600000061002B2B2B000D0A00004154E9
:1093F0002B530D0A0041542B534F434B413D5443D3
:10940000502C746573742E6A6F796675656C696E1D
:10941000672E636F6D2C373031310D0A0041542BAC
:10942000574B4D4F443D4E45540D0A0041542B556A
:10943000415254464C3D343039360D0A0041542BCC
:109440004845415254454E3D4F46460D0A00415451
:109450002B453D4F46460D0A0041542B454E544D79
:109460000D0A0041542B49434349443F0D0A004132
:10947000542B494D45493F0D0A0041542B5749464D
:10948000493D4B46422D322E34472C4B4642313219
:10949000333435360D0A0041542B536F636B6574BA
:1094A0003D302C302C746573742E6A6F7966756547
:1094B0006C696E672E636F6D2C373031310D0A0089
:1094C00000C1814001C0804101C0804100C1814094
:1094D00001C0804100C1814000C1814001C0804184
:1094E00001C0804100C1814000C1814001C0804174
:1094F00000C1814001C0804101C0804100C1814064
:1095000001C0804100C1814000C1814001C0804153
:1095100000C1814001C0804101C0804100C1814043
:1095200000C1814001C0804101C0804100C1814033
:1095300001C0804100C1814000C1814001C0804123
:1095400001C0804100C1814000C1814001C0804113
:1095500000C1814001C0804101C0804100C1814003
:1095600000C1814001C0804101C0804100C18140F3
:1095700001C0804100C1814000C1814001C08041E3
:1095800000C1814001C0804101C0804100C18140D3
:1095900001C0804100C1814000C1814001C08041C3
:1095A00001C0804100C1814000C1814001C08041B3
:1095B00000C1814001C0804101C0804100C18140A3
:1095C00000C0C101C30302C2C60607C705C5C40463
:1095D000CC0C0DCD0FCFCE0E0ACACB0BC90908C8D3
:1095E000D81819D91BDBDA1A1EDEDF1FDD1D1CDCC3
:1095F00014D4D515D71716D6D21213D311D1D01033
:10960000F03031F133F3F23236F6F737F53534F422
:109610003CFCFD3DFF3F3EFEFA3A3BFB39F9F83892
:1096200028E8E929EB2B2AEAEE2E2FEF2DEDEC2C82
:10963000E42425E527E7E62622E2E323E12120E0F2
:10964000A06061A163A3A26266A6A767A56564A4E2
:109650006CACAD6DAF6F6EAEAA6A6BAB69A9A86852
:1096600078B8B979BB7B7ABABE7E7FBF7DBDBC7C42
:10967000B47475B577B7B67672B2B373B17170B0B2
:1096800050909151935352929656579755959454A2
:109690009C5C5D9D5F9F9E5E5A9A9B5B9959589812
:1096A000884849894B8B8A4A4E8E8F4F8D4D4C8C02
:1096B0004484854587474686824243834181804072
:1096C00041542B41504E3D000000000000000000BE
:1096D000000000000000000000000000000000008A
:1096E000000000000000000000000000000000007A
:1096F0000000380000000000000000000000000032
:109700000000000000000000000000000000000059
:109710000000000000000000000000000000000049
:109720000000000000000000000000000000000039
:10973000F2960108FC6700203813002000000000AA
:109740000200010000000000F2960108FC67002002
:109750003A1300200100000001020008010000008F
:10976000F3960108FC670020EC12002001080000BD
:109770003C00D00702000000F2960108FC670020C0
:109780003A130020D10F0000010200100300000076
:1097900000000000000000000000000000000000C9
:1097A00000000000000000000000000000000000B9
:1097B00000000000000000000000000000000000A9
:1097C0000000000000000000000000000000000099
:1097D0000000000000000000000000000000000089
:1097E0000000000000000000000000000000000079
:1097F0000000000000000000000000000000000069
:109800000000000000000000000000000000000058
:109810000000000000000000000000000000000048
:109820000000000000000000000000000000000038
:109830000000000000000000000000000000000028
:109840000000000000000000000000000000000018
:109850000000000000000000000000000000000008
:1098600000000000000000000000000000000000F8
:1098700000000000000000000000000000000000E8
:1098800000000000000000000000000000000000D8
:1098900000000000000000000000000000000000C8
:1098A00000000000000000000000000000000000B8
:1098B00000000000000000000000000000000000A8
:1098C0000000000000000000000000000000000098
:1098D0000000000000000000000000000000000088
:1098E0000000000000000000000000000000000078
:1098F0000000000000000000000000000000000068
:109900000000000000000000000000000000000057
:109910000000000000000000002F00000000070011
:10992000070000147F147F1400242A7F2A1200628B
:109930006408132300364955225000000503000037
:1099400000001C224100000041221C000014083EBF
:1099500008140008083E0808000000A06000000885
:1099600008080808000060600000002010080402D9
:10997000003E5149453E0000427F40000042615197
:109980004946002141454B31001814127F10002731
:1099900045454539003C4A494930000171090503F4
:1099A00000364949493600064949291E0000363625
:1099B0000000000056360000000814224100001488
:1099C0001414141400004122140800020151090665
:1099D00000324959513E007C1211127C007F4949E6
:1099E0004936003E41414122007F4141221C007F17
:1099F00049494941007F09090901003E4149497A25
:109A0000007F0808087F0000417F4100002040419E
:109A10003F01007F08142241007F40404040007F0A
:109A2000020C027F007F0408107F003E4141413E4E
:109A3000007F09090906003E4151215E007F091996
:109A400029460046494949310001017F0101003F93
:109A50004040403F001F2040201F003F4038403F13
:109A60000063140814630007087008070061514977
:109A7000454300007F41410000552A552A5500000A
:109A800041417F0000040201020400404040404088
:109A9000000001020400002054545478007F484420
:109AA000443800384444442000384444487F003857
:109AB0005454541800087E0901020018A4A4A47C80
:109AC000007F080404780000447D4000004080844A
:109AD0007D00007F102844000000417F4000007C92
:109AE00004180478007C080404780038444444389E
:109AF00000FC242424180018242418FC007C0804EA
:109B0000040800485454542000043F444020003CC2
:109B10004040207C001C2040201C003C4030403C49
:109B2000004428102844001CA0A0A07C00446454D9
:109B30004C4414141414141400000000000000001D
:109B4000000000000000FC00000000000200000017
:109B5000000C020C020000000000000090D0BCD0FD
:109B6000BC900003000300001824FE448C00030294
:109B7000070201001824D8B04C8000030001020144
:109B8000C038E438E00001020201020208060000C9
:109B90000000000000000000000000F804020000C7
:109BA00000010204000204F80000000402010000A9
:109BB0009060F86090000000010000002020FC2070
:109BC0002000000001000000000000000000080666
:109BD00000000000202020202000000000000000E5
:109BE0000000000000000002000000000080601C77
:109BF0000200040300000000F8040404F80001025D
